:20000000003B012085330100A1C10310A1C10310A1C10310A1C10310A1C10310A1C103100D
:1C002000A1C10310A1C10310A1C10310A1C10310A1C10310A1C1031079C10310B9
:20004000DFF800C32DE9F04FADF1440D9CF8AF049CF840730F90BC4807B9017881210F9F08
:200060000170022F02D1B949FF200870B84C0F9DB949B84ADFF8E482002003461E46277815
:20008000A081012D0C93098816702069A77012D0007A801E85B2A942C0F2AD83216A04F13D
:2000A00018000422083157F0D1FB0426A17E607EE27EA68129E0467A027A06F0070302EBD6
:2000C000032295B2720938BF2D1F06D3427A057A02F0070205EB0225AD1E36F07F06ADB2FB
:2000E00040F08983A942C0F286830A30294610F05DFE216A04F118000522083157F0A6FB3A
:200100000526A681227FE17EA07E04F11A0300EB01200B93C1F3011B60818A49227191F813
:200120004013ED1EADB2002908BFBBF1020F00F06283BBF1020F00F35E83DFF8B49261B1C0
:2001400010F0070F00F0578349460978862904D100F00701022940F04E83011301F00201FF
:20016000022944DA637800F00700022831D1D8F804A0181C2DD1216A09A801228919083158
:2001800057F064FB771CB8B2A081D0470746D8F808106C4899F800304568CDF828800E466C
:2001A000862B02D03846884710E09DF9240017F0B5FD9DF9243068770020A8773846EB7724
:2001C000B047608900F0100011F06EFE17F010F815E399F800000C9E862808BF0126CDF82F
:2001E00028803EB10C9813F0BFFFA77801E0CDF8288063788FB183B9012F00F0F9826089BB
:20020000022F03D110F0070F40F0F282032F05D100F00701032901D0EAE26089010909D387
:2002200010F4405F00F0E482464991F86474002F00F0DE82011301F00201022902DA810ABC
:2002400080F0D6820F99012905D0BC4ABB49921C89780B9201E0B949C978C1F381098E11D8
:20026000B9F1010F00F0C482012E00F0C182BD49BBF1020F09D08A5D11F809108918CFB265
:20028000AEB1C10913D3BF1E0BE072184944127909798918CFB2C10905D259EA060306D07E
:2002A000BF1CFFB203E059EA060308BF0227C0F300217A1A61719542C0F29A82ED1B0009A3
:2002C0000D44A9B2218124BF25200C900C984018743080B216F008FD65786061002800F079
:2002E00087820021742211F073FA0020E070B4F80A804FF0FF0A1DB9164908F0200008701D
:200300000025144B60790D951D780E90002D41D000283FD108F00708B8F1030F06D0B8F1F4
:20032000010F25D1074890F8AE0408B30F98012816D0A34805789DB117F074F9FE2815D088
:200340000EE0C04610010020B9350020091F0020FC330020BB3500206C1E0020D818002009
:2003600016F00EF910B915F0CDFE08B10420E0700F98012808D1B94890F8400310B1BBF1C8
:20038000020F01DA16F0D0FA6079B4F80A800E90E0780D90636903F1740058609865258968
:2003A0001D812089A3F85C005FEA181016D30F9D0E98012DC0F1030082B2A3F85C2019BF4E
:2003C0005E49491CB3F85C200B99986D57F03EFA6369B3F85C10986D401898650F98A3F843
:2003E0000C80012806D055490B980078497805E0BD35002051480B99C07809780D9DC0F3AE
:20040000011001F07801014345EA0100187483F80EA00E9920790C9001B1002083F830607F
:2004200083F83A9083F84900A089002FA0EB010085B2A58100F0D1818848BB46216A90F84C
:20044000AF94E7805A464919CDF840906846083157F0FCF97F19BDB2A581B9F1010F07BF8B
:200460003648C0780B98007861690F7C4E46012E07F0400AC0F301100F9007BF2F48C0787A
:200480000B9800786E46C0F38107002F44D00F980023022802D1BAF1000F0BD19DF80120FC
:2004A0009DF8000000EB0220A1F844000DF10206A1F84200DFF83493B1F84400B9F86A2016
:2004C000824203D04FF6FF72824222D1032F11D07278307800EB022082B24A86B9F8681039
:2004E000B61C0120914213D04FF6FF71914218BF181C0DE0CC4800683146323057F01EFC1D
:20050000C948006809F15F01323057F0FFFB08360346002B00F064811098012807BF0748F8
:20052000C0780B980078831124D00F996069022906D0017CC90906D30CE0C04614340020EC
:200540005AEA070706D172783178B61C01EB0221A0F84210032B07D07178327802EB01226C
:20056000028507E030AC0100AF4800683146283057F0E4FB08F00708B8F1030F07D0B8F19A
:20058000010F39D1354890F8AE04002834D033486669D0F880704FF00009E7B17B7E33F060
:2005A0007F0314D096F8300002280BD003280ED107F1700006F1280157F0A8FB38B11BE0B2
:2005C0007C1E0020B7F87000318D884214D057F80C7C002FE2D1B9F1000F0DD1934F484616
:2005E000E0700B9BF878C0F301111878CDF8349000F0780008433074109801285BD1174804
:2006000090F8400310B10F98022854DA88480078002850D00E9800284DD10D980F4E074684
:20062000DFF8F8A1DFF8F8910C9D96F8AF04012816D02846524600250223D570911C0B7034
:2006400017B143F010030B7003228870484680F84720816416F068F92AE0C04610010020FA
:20066000E9200DF1260114F07DF89DF82660052336B95046072200F10C010A70082204E05C
:20068000504600F10C010B7018224273881C022200260270CE701FB1027842F010020270BE
:2006A0000D71C9F8DC10A9F8D030032110F07EFBA589B4F806B0606981890909C0F08D809F
:2006C000806D5A46694657F0C1F86169886D58448865276AB1F85C0001225844A1F85C004C
:2006E0000DF125007919083157F0B0F86E1CB5B2A58161699DF82500896D087061699DF8B5
:2007000025709DF82530886D401C8865B1F85C00401CA1F85C0007F0070081F82400C3F375
:20072000C10781F8257091F8246020898146002E56D03C497F183A78121D1646E28086428F
:200740004EDC216A05A84919083157F07FF838789DF817209DF814304019001D80B23D782C
:20076000A08103EB026061699DF8163000EB03409DF8153000EB032088616DB12A4800686C
:200780006D1E06A92A461C3057F060F8387861696844C07D81F82600886D324605A957F060
:2007A00055F86169886D80198865B1F85C004FF0FF3706EB0642C9EA0040A0FA42F01FFA1C
:2007C000A0F217FA80F0A1F85C2082B22281B1F85C000A818018A1F85C0000F001FC0EE022
:2007E00017F074F912F0B2F809E0C0462018002016F0D6FF03E016F0D3FFCDF828800A9DE8
:2008000068688047216A0A680023137109682162A968884711B0BDE8F08FC046C81B0020DB
:200820007C130020FC9D01001034002014340020BB3500202DE9F047044660784FF0000ADB
:20084000ADF1200D42280DDC422800F09783401E0E2813D92F38082821D9103844D0401E3B
:2008600037D07CE3433825D0401E00F083830C3800F07C83401E00F0758370E3DFE810F0BB
:200880005F035703A20338039E039A039203D302C6026F036F038E038A03B802B002DFE817
:2008A00010F0A7017C006C0075035F00540046002C007103A088022838BF272407D3A06821
:2008C000024657F0CAF9911C16F0E0FD044643208CE2A08828B9C549182055F085FCC4B290
:2008E00000E02724412081E2A08818B916F068FE044600E02724402078E2A088CDF800A0E8
:20090000012818BF27240CD1A068CA4902786B46182055F069FC0099C4B20DF1110057F022
:200920006EF98DF810403720052104AADAE2A088012818BF272406D1A068C7490278182080
:2009400055F052FCC4B2362050E2A08828B9C349182055F049FCC4B200E02724352045E212
:20096000A088082818BF272405D1BD49A268182055F03AFCC4B2342038E2A088022818BF57
:20098000272408D1A06857F068F9B6490246182055F02AFC5446322028E2A1880329C0F09E
:2009A0002281A06890F800804046713800F00881401E012840F215815E3800F0E480401E45
:2009C00000F0C380401E00F0AB80401E00F09080401E5DD0401E3ED040468138022810D9C4
:2009E000001F01280DD9801E09D0401E09D0401E012804D9801E14BFFF20022002E00820FB
:200A000000E00120C91E814240F0ED8015F064FC071C00F0BF80A06841468139022900F172
:200A2000030015D9091F012912D9891E0AD0491E0ED0491E012905D9891E6FD157F00DF91F
:200A400038806BE001683A4611604068506065E00078387062E0072940F0C580052015F06B
:200A60003BFC071C00F09680A068401C10F8021B397010F8011B797010F8011BB97010F882
:200A8000011BF9700678524606B10122384677E0182940F0A8801C2015F01EFC071C79D0AC
:200AA000A3685B1C13F8020B3870184657F0D5F89E1CB880304657F0D0F8B51CF880294653
:200AC00007F1080016F0E4FF05F1080313F8010B514600B1012107F1100502263976184669
:200AE00057F0AAF81B1D761E45F8040BF7D115E0172978D1182015F0EFFB071C4AD0A5683E
:200B00006D1C15F8020B102229463870781C0FF02FF805F1100057F08FF87861384630E0F4
:200B2000052960D1042015F0D7FB071C32D0A068401C10F8011B397010F8011B797010F8F0
:200B4000011BB9700078F870E8E706294BD1052015F0C2FBF0B1A168491C11F8012B0270B9
:200B600011F8012B427011F8012B827011F8017B524607B10122C2700F78524607B1012243
:200B8000027107461AE00D292DD10C2015F0A4FB071C01D11A2427E0A068401C10F8011BD5
:200BA000397010F8011B79700268BE1C326045687560037A337210F8091FF972384602E00A
:200BC000032910D15046A060A368C849424618201F4655F009FBC4B237B1384615F074FF94
:200BE00002E0F42400E027243120FFE0296C0100A088032840F0F180A0680678451C1A24F1
:200C000030467138022840F2E6805F3816D0401E09D0401E10D0401E09D0401E05D0401E39
:200C200018BF08200BD1052009E01C2007E0182005E0C04625030100042000E00C2015F027
:200C40004BFB071C00F0C5803046D03802280BD9C01E02280AD90BE0C9AC000079C90000DD
:200C600005B80000B12901006878787028783870CE491820324655F0B7FACD4985B232464A
:200C80003B46182055F0B0FAC4B2002C40F09E80681C80B215F020FB5FEA000800F0958090
:200CA0008146304609F8014BD03870D0401E5FD0401E51D0401E40D0401E23D0401E57D012
:200CC000E8B24E46012818D0E8B202280FD0E8B2042807D0EAB2304639460EF049FFE8B224
:200CE00036180DE03968484656F089FF03E03988484656F0ACFF064602E0387806F8010BB1
:200D0000304656E03978484600F8011BB98856F09EFFF98856F09BFF07F1080116F0B8FE92
:200D2000397E022607F1100500F8011B55F8041B56F065FF761EF9D13BE038784D46791C4C
:200D4000102205F8010B28460EF012FF796905F1100056F054FF2CE03978484600F8011BFB
:200D6000797800F8011BB97800F8011BF9781EE03978484600F8011B797800F8011BB97831
:200D800000F8011BF97800F8011B39790FE03978484600F8011B7978BE1C00F8011B32684D
:200DA000026075684560337A0372F97A093000F8011BA0EB0900C1B242463020491C16F023
:200DC00097FE404615F080FE00E01A24384615F07BFE1CB9F9E0F42400E02724302005E035
:200DE000A088012814BF272426240F2021469BE0A088012818BF272106D1A06875490278A2
:200E0000182055F0F1F9C1B20E208DE0A088002808BF272105D0A1680878491C16F046FAF5
:200E20000146092080E00A202727ADF80C00A6888DF81870012E0CD1A0680478452C05D1A7
:200E400065491820462203AB55F0CEF9BDF80C0038B99DF8180000283DD1BDF80C00401CD8
:200E60003AE0BDF80C00401C80B215F035FA071C2ED0452C07D0791C204603AA14F000FFC1
:200E80008DF818000DE0452001A90DF10E0214F0F7FE0199BDF80C208DF81800781C0EF008
:200EA00067FE9DF8180038709DF81800002806BFBDF80C00401C0120ADF80C00BDF80C101E
:200EC0003A46082016F014FE384615F0FDFD7CE01A208DF818000120ADF80C00BDF80C10FF
:200EE00006AA082016F004FE6FE0C046E1700000A088042818BF272115D1A06801788DF80D
:200F00000810401C10F8011B8DF8091010F8011B8DF80B103149007802AA8DF80A00182072
:200F200055F062F9C1B2042016F044FC4DE0A08800280CBF54462724022021460DE0A08869
:200F4000012818BF272107D1A1680978504601B1012016F03FFB014601200C4646E74FF018
:200F6000260A32E0204612F091FA2EE0204612F0E9FC2AE0204612F00FFD26E0204613F0F4
:200F8000CDF822E0204610F071FE1EE020460EF0C7FB1AE0204612F0B5FF16E020460DF022
:200FA000D9FA12E0204611F00BFB0EE0ED3F0100CD900000204610F045FC06E020460AF09A
:200FC00097FB02E020460BF063FC504608B0BDE8F087C046C978010065470100D77B01002B
:200FE0002DE9F04FC04C60692689216AA589806DADF1440D32464919083156F027FC61693D
:20100000886DAD1980198865B848216A0678ADB2012249190DF13E00083156F017FCB44FD1
:201020006D1CADB2022E09D1216A38460122401C4919083156F00AFC6D1CADB2216A04A830
:2010400004224919083156F001FC2D1DA8B29DF813109DF810309DF81220A08103EB016024
:201060009DF81110636900EB024000EB0120049016F032FBD863049816F020F8A3F840001E
:20108000EA2016F006F9BA48DFF8E8A20221022E01700AD1B848801C007830B1387810B9D1
:2010A0007878FF2801D00420E0706569E078297C084328749DF93E0016F030FE85F8460057
:2010C00005F17407AF6529899DF93E006E6885F84800B5F85C004FF0000B401A80190146DD
:2010E0006860A88985F847B0820A18D2020950D310F0070F07D000F00700032812BF081CDB
:201100006868401C41E06968C87800F00702401000F0380000EB42004018001D35E0696878
:201120004878C7112BD12E89696658464B780A7803F07F035B0003EBE2137E2B0DD07F2BCF
:2011400009D002F07F0280188918801C891C80B28642EBDC09E0594600E0012185F8601091
:201160002989801C80B2814201DA584605E06968091869602989091A2981A5F86800686EB9
:2011800010B1B5F86800B0B168686861A889000918D295F86000002800F0FC80284613F069
:2011A00009F86569E86C002800F0F480B5F85000002840F0EF8004F1140016F0A9FD584669
:2011C00060610CE258465E46059095F82470069005A906AA07AB0796284605F07DF9002824
:2011E00040F0CD80B5F85C106869009101902E896968401A311A88B202900698001D03901F
:201200000598AB6DA9693A4615300BF0F1F8002840F0B580B94895F860302E89C15D701A54
:20122000288113B1284612F0C5FFAE8906F00706032E02D168680078E87395F80F8073207D
:2012400009A915F071F8832010A907F03FFFD94659460AE0C278012A03D1002F08BFDC200A
:2012600028D0001D491C0990C9B29DF84000884240F3848009988278032E07D00378B342F7
:201280000DD09AF840330BB1022E08D0032EE8D10378032BE5D103465B784345E1D1BB103E
:2012A000B3EBA20F05DA02F0030207F003039A42D0DD58468446059895F80FE090F81480E6
:2012C000594601E0491CC9B288454FDD07694B00032E07EB03020DD1FB5C032BF2D15278E2
:2012E0007245EFD10FE0C046FC330020BF050020081F00201278B24205D09AF84023002A96
:20130000E0D0022EDED10698077D002F08BFBCF1DC0F33D0A869B0F1FF3F25D0712008A964
:2013200015F002F8089B5846AA6905998B4206D10699814601EB8901C968914212D8401CF2
:201340002C330228F1DB0698521CB2F1FF3F00EB8900C26002D107980121817085F801B002
:2013600058460DE0DB200BE0DB2008E0DC2006E0B9350020100100207A1E0020DD2068706B
:2013800065696870A8696F7868651FB1F22015F080FF65699AF84003002800F09E80A98971
:2013A000914E01F00702022A5FD16778002F5CD16F78002F59D16169D8460DF136008DF8DC
:2013C0003F80283156F0BAFC61690BA80A22283156F03CFA06F1100167690888DAF86433AA
:2013E000401C0880786E0DF13F020421984704F11409354630B9DAF8040018B19DF83F10E7
:2014000080F86810676997F83000022811D1D9F800000AF22C410E4602222830203115F0E1
:20142000CBFA30B906F116010DF1360056F086FC67696E480078862807D1688A401C688238
:20144000B88900F0100010F02FFD9AF8400320B1DAF8881309B160698847484616F058FCD2
:201460005846606115F0C4FEBBE0614A17785FB3C1F30131022927D16878002840F0AF80EF
:20148000E7789DF83E105F48B38A05F128021C35002F017003F10100B0820CBF594608215B
:2014A000544B5846186000910195BAF85234117A0D2004F005FF10B915F036FA01E015F084
:2014C00035FE4D486569007838B1DAF8881321B12846884765699AF84003AF890A9507F028
:2014E000070778B1A87BFF2875D0032F08D1284640680078042805DD6DE0C046009E01008D
:20150000012F68D1381C3AD0401E4FD0801E62D1A889C0F30130022803D16868007807282C
:201520002BD02889002856D0284641684A1C42600F78AC46C7739CF824606EB9002F4AD057
:201540000A2F48DA2D490089C95D814209D0082F41D1082805D03EE0C07B00283BD00A2863
:2015600039DA28460189491E0181C17B0B3101700A99C87B401CC8731AE0322017E09AF83C
:2015800039040F280CD016F0CFF848B90A988189091301F00201022902DADAF810108847A9
:2015A0009AF86F040A9D2874152000E0162028700A990AF1840056F093F8114D6868804718
:2015C0009AF88C10491C8AF88C10A9688847202016F0C2F944E70AA813F074FE40E711F0FF
:2015E000B5F911B0BDE8F08F481D0020BD350020BB350020D01B002050040020079E01008C
:20160000D81800207A1E00202DE9F04FADF18C0D1C9104461D920DF15700D1491E93082286
:2016200056F014F92046694614F085F81F90002804BF0020229000F0098202200027A41CD1
:20164000DFF824B32090C74E2297204602A912F0C8FA5FEA000900F0F68122990DF13900DE
:20166000162256F00FF99DF809707F1E00F088807F1E40F0E081B9F10B0FC0F2E781A41C75
:2016800004A80422214656F0E1F8241D05A80222214656F0DBF842F20B000DF1160112F00A
:2016A0007FFCBDF81600BDF81410884200F3CE81A41C14F8010B0DF1390214F8017B8DF8E1
:2016C000390014F8015B8DF83A7014F8011B8DF83B50204606F048FCC34909780028044465
:2016E00000F0B4811F9D012905F1020500F09C814FF400500DF14F0112F052FC0DF14F0057
:201700000DF15701082215F057F940B11C990DF14F00082215F050F9002840F0858142F2F7
:20172000010004A906F0CCFD42F20B0005A906F0C7FD42F205000DF1390106F0C1FD0DF172
:201740003A0142F2060006F0BBFD0DF13B0142F2070006F0B5FD0FA942F2090006F0B0FDB1
:201760009DF83C0028B1022840F05E8142F2030001E042F20D000DF13D0106F0A1FD53E129
:20178000B9F1050FC0F26281A41C14F8010B0DF1390214F8017B8DF8390014F8015B8DF8B2
:2017A0003A7014F8011B8DF83B50204606F0DCFB0028044400F04A811C9806A906F01CFF75
:2017C0009DF83600002840F011819DF83C0000287DD1B6F84E70002F00F00481B6F85200FD
:2017E000874207D0308B718B884201D10AF09AFAB06D21E0B76D4FF400500DF15F0112F033
:20180000CFFB15F0E1F94FF6FF78229D2190AA46B6F84E00A84243DCB06D4FF6FF714145A6
:201820000AD04FEA480707EB88073818808813F02DF9B06D3F1823D1B6F84E300746002B38
:2018400008BF229D19D05846229D40681946D846BF1FBF1DFA782AB1491E05F10105F8D164
:20186000BF1D0AE08047B6F85210491CA6F85210D8F808108847B6F84E30AB4200F099808D
:201880001C980BF05FF9B8800120F870FD788DF83650B888ADF83700229B8DF82330A5E0CA
:2018A000B88812F017FA014608220DF15F0015F083F840B138880104219816F001FA824550
:2018C0003CBF8246A8466D1CBF1DADB2A0E7B6F84C70002F00F08680B6F85000874207D0DF
:2018E000308B718B884201D10AF01CFA706D20E0776D4FF400500DF1670112F051FB15F078
:2019000063F94FF6FF78229D2190AA46B6F84C00A84250DC706D4FF6FF71414509D008EB5B
:2019200048173818B0F81F0013F0B0F8706D3F1829D1B6F84C300746002B08BF229D20D040
:20194000DBF80400229D1946D846213F2137BA7F62B1491E05F10105F8D1213711E0C046F5
:2019600054A50100C00E0020D81800208047B6F85010491CA6F85010D8F808108847B6F8D2
:201980004C30AB4215D022993846212255F07AFF1C980BF0D7F8A7F81F000123FF203946C1
:2019A0002122BB770546787206A8FD7255F04EFF1CE0612060E0B7F81F0012F08BF9014676
:2019C00008220DF1670014F0F7FF38B17968219816F076F982453CBF8246A8466D1C21372D
:2019E000ADB293E7642047E0120100209DF836000DF13901162240F004008DF8360008A856
:201A000055F024FF1F9D9DF83C00AD1C48B19DF84E700DF13D00394611F030FC3F1A8DF8F7
:201A2000357006A810F0E6FA209809EB0007BF1CB8B2209003E01F9D4C44A41CAD1C20985B
:201A400085423FF702AE2098022803DC229A672011460DE01F9F01460220C0EA014207EB8B
:201A60000741A1FA42F21FFAA2F110FA82F222981D9B19801E990A8023B0BDE8F08F70472B
:201A8000D6482DE9F04F14300168ADF11C0D31B1CD480078012814BF002001208847DFF80D
:201AA00034B3CA4DCA4FCC4C9BF8AF042979012861D0E86801290CD158B1002011F0C0FF75
:201AC000386A4168E8688847D748012101700020E86002214FF00108297138B9386A016A7F
:201AE00005F1140088474FF4FA70E88413F00EF9F8698069006860639BF96E040FF01AFF57
:201B00004FF6FF71814218BF60860026668404F12D016662087868F30300087015F0CAFF71
:201B200030B9D548D94A102114230170501C0370E86858B9386A0668F96AD04804F12002C1
:201B400005F11403B0472F46044612E0304611F077FF8DF80C6033468DF80D60386A029350
:201B6000066D08228DE80C00E8682034214602AAB047FC607CE1E86802290CD158B100205F
:201B800011F05EFF386A4168E8688847A648012101700020E860012129714FF00008CDF8CC
:201BA00010808DF814808DF81580A8B9B448006812F068FA012812BF85F801800120687048
:201BC000386A016A05F1140088474FF4FA70E884AC4EAE620623EB6213F098F8AA49786A1E
:201BE0004DC88A468AE84D009BF8AD64F86981F8008026B980690068C4F8FC0005E0C0694D
:201C00000068C4F8FC0015F083FA632006A912F0A9FD9BF87F94484614F0C2F804F1EE0271
:201C2000014610780123B9F1800F63F30200107005DDB9F1840F1FDBB9F1860F10DB0F202E
:201C400004F1F70284F8F000107868F303001070887B052814BF2420292084F8F40019E0CB
:201C60000F2084F8F000292684F8F46004F1F700027868F303020CE00F2084F8F000212616
:201C800084F8F46004F1F700027822F00F0242F00802027004F1F5021078B9F1800F68F335
:201CA0008710107002DDB9F1840F1ADB8E7A86B904F1F5039DF818001A78401E60F30502D1
:201CC00004F1F6001A70027822F03F0242F0180216E004F1F5029DF81830107863F30500D4
:201CE00006E004F1F502107820F03F0040F00200107004F1F600027822F03F0242F020027D
:201D00000270887B8A890A2604F1EE03401D504390FBF6F21E8862F3CD061E80888919220A
:201D200004F1F006800390FBF2F3326863F31C2204F1F8033260FA69187892F8246066F3BB
:201D40000200187092F8240004F1F806C310307863F3C30030704AF63F33A4F8FA3008891B
:201D60004B680E68401E434306EB53004FF47A73B0FBF3F0166AA4F800013078A4F8E28091
:201D8000C4F8E48004F1ED0284F804011078012666F30300107015F08DFE30BB8889364E23
:201DA000B9F1020FB3FBF0F0C1B238483170B3FBF1F2427014D0B9F1840F16DBB9F1860FB2
:201DC00013DA05225C210DE0BF0500202C1C002020180020100100207C1300203C1800208D
:201DE0000222A8212A4B1A700170E8683E6A70B3404611F025FEA8789BF87F14884215D1CB
:201E0000E9789BF8AD243E6AE868914210D1022142468DE80600366DE034434604AA2146D6
:201E2000B047FC601EE0C0463E1F00203E6AE86871688847012117483B6A01701E680F48BA
:201E400004F1E002514605F11403B04707E004F1E0020A48346805F114035146A047E86091
:201E6000786AB8629BF87F04A8709BF8AD74EF7007B0BDE8F08FC046701D00202030002027
:201E800094120050E168010088350020781E0020481D00203E1F00202DE9F04FCE4CADF160
:201EA0003C0DDFF838A3DFF83893DFF83CB3D04F0C90616894F8AF04012800F081800120C1
:201EC00052464E4610703278012A02D001F026FA61680D894E6894F86F040BF0F5FE01F0AB
:201EE00091FBC04CDFF8048304F1380908F1040089F80F500068A6640025658780478246C7
:201F00005A4607F120000C9B0668106833F0010335D104F1A00104F138024D8004F1AD0318
:201F2000C4F8A4201A7822F00F0242F002021A7004F1AC031A7865F303021A7004F1B703E0
:201F40001A7822F00F0242F004021A70658749F64043C4F8BC3004F144031A7865F3030289
:201F60001A708DF814500495B64B8DF8155008248DE83000346D04AAA0474C460FE08DF85D
:201F8000145038348DF815502A466580AD4B049208218DE80600356D04AA2146A847AA4967
:201FA00046460880B16800280A4607D4A74991F90000FC60401C0870504638E1504639E198
:201FC0004FF0000808894A68A14ECDF82480C500127830781035920906D340F6485292FB12
:201FE000F0F2AD1805F5AF750E7D68438500352E0CBF46464FF4FA560DF12E01E82012F0DD
:20200000B1FB9DF82E00032808BF44F620666068007DAD19352803D1D4F8A40380474543A1
:2020200002205E468DF828003068089508A90CF093FE4E46012051460870317887F800804E
:20204000012901D001F06AF960680589466814F08BFEDFF800B23088BA46000942D394F8B5
:2020600040736168002F3DD04B6A4F6E986AB0F1FF3F26D02FB3421C9A628862030E07F829
:202080000139606890F82A0007F80109606890F8290007F80109606890F828003870626817
:2020A000106A00950190801B281A80B20290916A506A92F88C203346153009F031FD0746C2
:2020C00000E0DB27D4F8841367B119B9E4200EF073F904E0604880F80080E4208847002FDD
:2020E00040F0AC80294630460EF060FE64200BA912F038FB594894F84073007837B994F802
:202100006F040BF0E1FD012805D094E00BF0DCFD012840F09080524BA81C87B20DF12D01FE
:20212000E9201F8012F01EFB9DF82D00012805D13D46C5F3022040F0180005E02D1DADB2E8
:20214000C5F3022040F0080006F8010D06F8015D244D9DF82C00A5F8C2800028C5F8DC60D3
:202160000CBF40484048CDF8188002238DF81D8005F168068DF81C3005F1C009A6F80280CC
:2021800005F17501C5F81801184FC9F81800087820F00F0040F003000870786880470D902F
:2021A000284B0C98012825D0042823D088B105280DD0032808D194F87F0413F0F1FDC07B49
:2021C000022818BF4E4617E005F1C00614E0274B12E005F184060FE0100100202F1E002052
:2021E0003D1F00207C130020381C0020D81800202018002005F16806DAF82000046D41468A
:2022000002208DE80300DBF80C0006AA3146A047BE680D490028324608800AD40B4991F9D7
:202220000000C035401C08700D98CAF80C50904704E00D9890471A200EF0BEF80FB0BDE889
:20224000F08FC046E9660000C81B0020361E0020701D00202C1C0020BD3500207B1E002053
:202260004C1400204E9055550E7A555511E300002DE9F04F064692F80890307D09AF88463A
:20228000ADF1240D04933528039205D0114606F170000A2255F0DAFADFF8D4C238F07F05F5
:2022A00006BF604600884FF6FF700590F08A800934BF002008203076F08AC00834BF102099
:2022C00080207076F08A400903D260460E30007800E00020B076F08A41082CBF2024002448
:2022E000000928BF44F010047368002108F07F08307D06915B1E02280EDB0D2808DA0C2810
:2023000003D1022044F40854069044F0030404E00D280CBF02200120044396F88C0008B121
:2023200044F00804210900D320B1B34D95F8642412B908B1DF204EE1210973D306F124013C
:20234000DFF8A8A296F88DB0079100EB0A011AF80B300A7999183389491DCAB29918A44B44
:202360001A8808908A42C0F23881002851D0049A039906F184000BF0DBFB079900280860ED
:2023800044D0806AB0F1FF3F3ED07068BBF1000F4FF00003A0F1010012D096F88E10524645
:2023A00000F8011912F80B10491EC9B241B18A1992F88320491EC9B2002900F80129F6D14E
:2023C000079970660968896AB162090E00F8011996F82A1000F8011996F82910089A00F8AC
:2023E000011996F828100BF0030B00F8011902F0070141EACB0101707168091ACAB231894E
:2024000070608918318105E0DB2700E0F3277770E4E00023F08A7370C00828BF44F0100496
:2024200073685B1E326DA2B9B26D92B995F87D14012903D13089B0F5EE7F06DA200904D21E
:2024400002290AD144F4005401E044F48054012002E044F4085402200690A87801280CD089
:2024600095F8400348B196F86B00042805D1022024F48054069044F4005444EA8834B8F1D5
:20248000020FA4B20CD0B8F1030F12D1A3F1070A05F58E61504655F051FCAAF1010308E01E
:2024A000B5F85604001203F8010995F8560403F80109069802280CD0B8F1000F15D0B9F127
:2024C000000F0CD004990598814208D144F040040BE0B9F1000F08D1B8F1000F05D005991B
:2024E000081203F8010903F8011944EA8924B9F1020FA4B20BD0B9F1030F10D10399A3F114
:202500000708404655F01AFCA8F1010307E003990888001203F80109087803F80109B9F1D5
:20252000000F05D00498011203F8011903F801093878F8B92F480178307D0D2814D068B9B6
:20254000306D28B995F84004411C85F840140AE095F86504411C85F8651404E095F84E0408
:20256000411C85F84E14014603F8011904E0C0466205002044F48074201203F801091C7063
:2025800070683789C01AC1B2736078183081200920D3B06D00B1306295F8400310B1307D88
:2025A0000D2817D1706A816A4A1C82623289306AB162C71A0092D21B019090B20290706AE8
:2025C00096F88C20153009F0ABFA00281CBF7070071C07D10020707005E0E5277770F32015
:2025E00014F057FEF8B209B0BDE8F08FFC9D01006C1E00200034002010010020B1482DE923
:20260000F04F8846ADF1140DB14DAF4903920078AE4A9A4601286AD001230B70C848039B63
:202620004FF0E04600240227884616EA0A060068147007EA030708BF002F34D14FF4803134
:202640001A4614EA0A0501EA020108BF00291AD122464FF4003112EA0A0501EA030108BFA7
:2026600000290CD14FF4800112EA0A0201EA030108BF00290AD0047110F068F906E004719E
:2026800011F0C0FF02E00471FDF7DAFC03992546202015EA0A0500EA010008BF002813D047
:2026A00014F044FD10E095F90010AB4A491E297092F90010491E117095F900500DB9A7493B
:2026C0000C80047110F042F9A34991F9000028B1002E0CBF002F91F9000004E0A04804707D
:2026E000204600F01BFE0094CDF804802DE10120002316460191DFF86CB29C4C08702027B2
:202700001A460399009317EA0A07327003EA010008BF002876D108464FF0E047104017EA4D
:202720000A0708BF002843D14FF48601039BBBF80A01DFF83CC2CDF808B012EA0A0701EA15
:20274000030108BF002919D1874912EA0A0701EA030108BF002970D004F13801A4F808804D
:2027600099466081BAF1000F81E8000604BF4946B1F1806F61D102285FD111E004F13801E2
:20278000A4F8088099466081BAF1000F81E8000604BF4946B1F5803F4FD1B0F5505F4CD1E4
:2027A0002046006A6746436938684146984742E0264695F90000B6F90870401EB8452870B4
:2027C00017D1728906F1380003C8002904BFB0F5803FB2F5505F08D0002904BFB0F1806F22
:2027E000022A02D010F0B2F803E011F00BFF14F0F9FD594A92F90000401E10706FF00101DC
:20280000318116E05E4E6FF0010004F1080196F8407308806FB157480078832802D05649EA
:20282000812008702646316919B1184688474146E6E7CDF808B0BBF80A010399464E00279C
:202840004FF0020917EA0A0309EA010108BF00295FD043F2014181423CD0C91C814239D015
:20286000B4F9083095F900109845A1F10101297004D043F60401814237D134E004F13800AD
:2028800003C84FF4820217EA010302EA000208BF002A13D104F1380090E800183B464FF45D
:2028A000003213EA0C0302EA0B0008BF002802D110F04CF819E011F0A5FE16E0FDF7C0FB9B
:2028C00013E0C046BF0500203D1F0020301E0020371E0020A07895F90030401CA070581E04
:2028E000287010F033F814F04BFC0298244A39466FF00103A0F80A1192F84003238110B1FB
:202900001E4804780CB914F06DFD96F90000401E307095F9000010B911483946017096F9E6
:20292000000078B103994FF0E047484617EA0A0700EA01000CBF002896F9000005E0C04674
:202940000C340020384600F0E9FC0198009905B00170BDE8F08FC046361E0020B6140020E4
:202960002E1E00207C13002000000C8C20180020381C0020BD350020B9350020BB350020A8
:20298000100100202DE9F84FDFF844830F460646F80B80F05B81C24DCB4CDFF81C932878CF
:2029A000B90F80F0EA80B90880F0DD80DFF8F8A2DFF810B3F90A80F0B380B90B80F09E80E4
:2029C000DFF8E082790B50D2380C40D23809C0F0608113F0C3FB002834D0554644460321BA
:2029E00028682170783015F067F90CF0FFF8AF48007818B92868403015F07CF9022012F0D8
:202A000039FF11200BF092FA2868007C10B90E200BF08CFAA649087820B100200870052045
:202A200012F028FFA34815F003F800224846B0F91410B0F916002270814214BF02200720D5
:202A40000DF0FCFE27F0080710F07EFA21E14846416889684E88002EFAD04168896849887E
:202A60000129F5D027F40047EEE720B1042012F001FF0020287012F017FF0146002001B150
:202A80000120002540B1B0696FF480712A464FF0007384463046E047884889492A4615F0F2
:202AA00019F9B0684146022203880A70A3F602032BB141F21E015B1A18BF183000D11030CB
:202AC000018821F47C7141F434710180757420685C46006B2668804752467C4912680B68F3
:202AE000934214BF01222A1C26B1801B01EB8201000B886027F480572560A5E7404615F063
:202B0000F5F8011C09D0486838B14A68C868B1F92C10202314460022A04727F40057B8E0C1
:202B200015F0D2F88046484615F0E0F8061C14D05546286810B1783015F0BEF82068F1685F
:202B4000006B296080475C462060624814F070FF61484FF4006115F0D5F8404615F0B6F922
:202B600027F4806795E008F01DFC4846103015F0BDF808B927F002078BE0584A116841F0AD
:202B80008001116020B1042012F074FE0020287015F09AF88046B0680188A1F602052DB1A8
:202BA00041F21E016D1A18BF183000D1103001884B4D21F47C7141F434710180286808B343
:202BC000606D0068014604208847D8B120682C68006B8047F168001B728AF060F068000B8C
:202BE000F060F0688018F060F068884203D240184008F060F06840F6C41181422CBFB0F5A8
:202C0000FA7FF160404615F061F912F04DFE90B1B0696FF4807100224FF000730446304676
:202C2000A047484615F062F8002808BF47F0020701D010F089F9706900214FF080630446D8
:202C40000A463046A04727F0005722E015F03CF80146404615F04AF8061C15D0356AA808B4
:202C600012D225EA05003062084615F02FF9706868B165B17168B6F92CC0F06800232A46E9
:202C80008E466146F04702E0084615F01FF927F480471FB11048394615F034F8BDE8F88F4F
:202CA00082340020B03500206C34002080340020813400201DBA000034350020C434002058
:202CC00095930000743400208C010010003300203C35002071AA00006C330020CC21084074
:202CE00070340020B0B50446C6480768ADF1480D002F00F085812078401E112800F28081AA
:202D0000DFE810F063014F013501200119010301F100E300C300B2008D005D0053004200FB
:202D20007E012A001C001200F86B002800F06881684621460DF054FEF96B5FE1386C002884
:202D400000F05E816846002101220EF041FD60788DF80000396C51E1F86A002800F05081F7
:202D6000684600210E220EF033FDA11C684614F0F1FAA57BA1890022ADF80A1005B10122C8
:202D80008DF80C20F96A3AE1B86B002800F038816846002102220EF01BFDA5788DF8015014
:202DA00060788DF80000B96B28E1786B002800F02781684621460DF013FE796B1EE1386B3D
:202DC00008B36846002114220EF002FDA5788DF80150A3680193A289ADF80820A17B8DF80B
:202DE0000A1060788DF80000E57B8DF80B50237C8DF80C3094F911208DF80D2061690491ED
:202E0000396B684688476068002800F0F9800146F22008700020487012F092F8F0E0B86A11
:202E2000002800F0ED806846002124220EF0D0FC6078A11C8DF800000DF1020014F08AFA8C
:202E400004F10C0103A814F085FA257EE08A04F119018DF818500B22ADF816000DF119003A
:202E60000CF086FEB96AC9E0786A002800F0C8806846002102220EF0ABFCA5788DF8015039
:202E800060788DF80000796AB8E0386A002800F0B7806846002112220EF09AFC658862790A
:202EA0006078ADF8025023798DF80520E11D8DF80000A5798DF804300B220DF107008DF8EC
:202EC00006500CF055FE396A98E0F869002800F097806846002101220EF07AFC60788DF8DF
:202EE0000000F9698AE0B86910B1204610F0D2FDA07820B9A069002800F0828002E0A069F0
:202F000000287DD013F0C0FD7AE07869002877D06846002113220EF05BFC6D46A01C0168A1
:202F2000406829600B22686004F10A0102A80CF01FFE796962E03869002861D020460CF028
:202F400065F85DE0F86800285AD0684600210E220EF03EFC6078A11C8DF800000DF10200D4
:202F600014F0F8F9A089ADF80C00F96846E0B868002845D06846002114220EF029FCA01CBA
:202F800001686D46296040686860A07A0B2204F10B018DF808000DF109000CF0E9FDB9683D
:202FA0002CE0786860B36846002110220EF010FC60786588211D8DF800000B22ADF802505B
:202FC00001A80CF0D5FD796818E03868C0B16846002119220EF0FCFBA01C01686D46296030
:202FE00040686860A07A02A912F001FA0B220DF10E0004F10B010CF0BBFD39686846884793
:2030000012B0B0BD201E00202DE9F04FBF4DDFF80493C14C4FF000084FF0010AADF11C0DEF
:20302000E0694FF0FF3114F04DFFD9F8040080476789E688A288A4F80A802189A4F8068072
:20304000114347EA010246EA0201A180D9F80810A4F808808847A188080A03D34FF67F7073
:203060000840A08008200927ADF80000D9F80010ADF8027068468847DDF808B00028CDF8FC
:203080000CB039D120789DF80620616A904233D139B1A078401E02D0401E02D126E058466F
:2030A000884758460DF062FA071C25D00C2013F027F9061C1DD0D9F804008047B7603B786E
:2030C00083465BB92069314614F0F8FEA08840F01000A080E06914F0EDFE05E0304613F0FB
:2030E00003FD384613F000FDD9F808105846884702E0384613F0F8FCA38858092ED320698F
:2031000014F0D4FEE8B9D9F8041014F0A3FCC0B988470646206914F0C5FE071C0DD0B868AC
:203120004068A061B968486849880DF067FAB86813F0DAFC384613F0D7FCD9F8081030463A
:203140008847206914F0B2FE20B9E06914F0B2FEA38803E0A38823F01003A3809808C0F0BB
:20316000968080E004A8514612F050FB287800286DD0401E71D0401E5ED0401E47D0401E46
:203180001ED0401E6FD19DF810006978A8706F68A868C91CCEB20590314614F083F99DF898
:2031A0001010814205D147B1059930464246B84703E05748006813F0A7FC85F8008052E004
:2031C000AF68E8789DF81010C019C170E878401CC3B2EB7013F038FD6978C6B2C91AB142C6
:2031E0000CDBD8193146C01C12F010FBE87869788019C0B2E870814224D034E0DB1989B2F9
:20320000DB1C184612F002FB6878E8701AE09DF8100085F803809DF810706870F81C13F07F
:2032200033F80028A86008BF85F8008020D06978017085F800A016E09DF81000A96888706C
:20324000687810B9052028700DE00420FBE79DF81000FE2807D10320F5E79DF81000A968BD
:20326000487002272F7013F0EFFC00287FF47AAFA38813F0E9FC30B94FF6FD70184023F003
:203280000203A08003E0E06914F014FEA388180927D3606914F006FE071C15D0216A69B103
:2032A000607858B1401E02D0401E0AD103E0B86811F06CFC216AB868884702E0B86811F0DB
:2032C00065FC384613F010FC606914F0EFFD20B9E06914F0EFFDA38803E0A38823F00803DE
:2032E000A380D808FFF49CAE4FF6FB701840A080206914F0DBFD00287FF492AEA08840F0CE
:203300001000A080E06914F0D5FD89E6581E0020601E0020D8180020580B00202DE9F04FD3
:20332000B74C05466068ADF1340D8047DFF87CB2A24FAC4E012D0B9000F0C4809BF8390414
:203340009F4D0F2850D09A4890F9000010F1020F05D1984890F9000010F1020F44D0964C66
:2033600020783B68099003F13C0000688047099F61680023401AB900B0FBF1F2E768A0688E
:203380000A9704F1180787E80C000A9F98464146BA4271EB080102DA3946884206D807463E
:2033A0004146BA4271EB08011EDA0A90B9469A4604F11801B9EB02097AEB030A81E8000616
:2033C000099A04F1180003C81346DB1714F08EF8183440F6B832D317801A9941002984E83E
:2033E0000300BCBF0120287014F014F8002864D074480078002860D17348007800285CD115
:2034000072480078002858D171480078002854D12878002851D16F48007800284DD16E4896
:203420000078002849D16D480078002845D1002054F02CFA002840D1694F9BF8AF94387866
:2034400000283AD1684C206A436CF068022106AA98479DF8180080B3DFF85481226AF068D2
:2034600098F90010002511F1020F18BF01254FF0010A2DB1926B98F900109047226AF068F5
:203480004C4D95F9001011F1020F03D0926B95F9001090476FF00100287088F8000087F8A6
:2034A00000A0002013F026FE206AC169F0688847B9F1010F04BF0020607051490B988968AF
:2034C000884770E0012054F0E1F921460B9889688847464800780F280DD008F0A3FB386874
:2034E0000C36436C3068022107AA98479DF81C00002856D057E03A4D9BF8AF842878012844
:203500004FD1012013F0F6FD394F97F8C2000028FBD1354C206A436CF068022108AA9847E1
:203520009DF8200050B197F8C20038B92878012837D10020287013F079FF32E0304840685D
:2035400080472C4B814602210022B8F1010FF068297003F11007256A274E7A8009D00492FF
:203560008DF8141001238DF815308DE8060004AA09E002928DF80C108DF80D2003F11007B0
:203580008DE8060002AA2D6D39463346A8471B491B4E91F90000401C0870B168E76048466A
:2035A000884713F0AFF90DB0BDE8F08F100100202C1E00202D1E0020701D00204018002085
:2035C000BC350020B9350020BB350020BD350020BA3500202E1E00202F1E0020301E002054
:2035E0003E1F00202C1C00202018002049050020203000207C1300204D4D0100361E0020F2
:20360000D81800202DE9F04FAA4C6068ADF12C0D8047A94A1178A94D08911278A168012A20
:203620000BD0A54A01241470884728780795012805D02046FFF772FE01E088470795AA4DFF
:203640009F4CDFF8888295F8AF14E068012900F0B080DFF870B29BF9000028B19A4890F9EB
:203660000000002840F0AF80924840688047099000268DF8146004964FF001098DF81590B5
:2036800008F59C7AC8F8406108F5A271AAF80260087808F5A27766F303000870387808F28E
:2036A000531369F3C7103870187808F2531269F300001870107808F2531769F341001070ED
:2036C000387808F2531366F382003870187808F2531266F3C3001870107866F3041010704F
:2036E00098F8530108F5AA7140F0600088F85301F42011F037F8206A754A076D764B7548EB
:2037000031468DE803001068514604AAB8476949A08000288968AF78069148D46A496F4BCC
:2037200091F90000401C087093F90000002F00F1010018709BF90000C4F80CA000F1010008
:203740008BF8000014BF8021311CB4F85C004FF67F7208F5A876024011430843A4F85C00F3
:20376000307867F3C7103070B5F85204B5F85634082204F15F0705F58E663146A4F86A00A6
:203780003846A4F8683054F061F8B5F852040822B5F85644A8F86A013146A8F8684108F59E
:2037A000B07054F053F80699099888476CE0B146FAE708F5847108F58477814205D142481A
:2037C00090F9000008B100265FE03A48406880470026824695F84033A8F80A61002B07BF67
:2037E0004FF48600311C3E482021B1463D4A8DF80D601378CDF808909B0904D21278120975
:2038000038BF012200D302228DF80C20226A166D314B2F4A8DE803001068394602AAB047D0
:20382000244900288E68A0802CD427492B4B91F90000AA78401C087093F90000E760002A7A
:2038400000F1010018700CBF4F468027B4F85C00B5F852344FF67F71082201400F4338433F
:2038600005F58E61A4F85C00B5F85674A4F86A3004F15F00A4F8687053F0E8FF5046B0473B
:20388000012602E05046B0474E460A48406880470849896816B9084B089A1A70884707983F
:2038A0000078012802D00020FFF738FD30460BB0BDE8F08FD81800202E1E00203D1F0020FD
:2038C00020180020381E0020371E00207C130020381C002020004300FD250000361E002089
:2038E00000004F8CBA35002010010020B3492DE9F04F09781346ADF1240D814240F05A81E5
:2039000058781F789E780690FB2F079680F23A8100F01E004FF001090A2880F22F81069857
:20392000A74900F01F0051F82060002E089600F02581069ADD1CADF80C70079E8DF8082051
:2039400028468DF8096032F07F04049000F01281002F4FF0040A00F0F78001781B798DF8DA
:203960000B1021F007048DF80A30083C00F0E580DFF85082083C4ED0083C07D0083C40F01E
:20398000D980032F08BF4FF0000ADDE0032F40F0DB80841C04944446257DADF80C90002746
:2039A000012D30D1257F95422AD1627FB24227D1E27F514011F0070F22D1A17F99421DD1B0
:2039C0008078A8B1401E12D0401E032818D9001F02D0401E14D008E0607D1B1AB3F1FF3FCD
:2039E00006D007200FF006FFA2E008270EE0B94602A849460CF00AF9074604E0032705E0B0
:203A000007200FF0F7FE002F00F092803A4602A8202100278AE0042FC0F296808346A81CD6
:203A200054F01BF94446054620783F1FFEB2002701282BD19DF80810227A914223D19DF8C2
:203A40000910627A91421ED19DF80A10A27A914219DB9DF80BC0E37A9C4512D1A3899D4291
:203A60000DD1914206D0A1788E420DD0A1888E4205D109E002202070A1788E4204D0574635
:203A800002E0022700E00327216927B99DF80A30042808D020E0084613F006F8504620705F
:203AA0009DF80A30A372ABB902A90EC904F1080080E80E00284612F0FBFB2061002804BFF7
:203AC0002078062708D000206070A670A580A581207005E007B90327042823D002281DD063
:203AE0002169A0789DF80A20884612FB00F080B2324640180BF104010CF03AF89DF80A00CA
:203B0000A072A088801B86B2A68036B9CDF81080ADF80C500627D14602E02078042801D072
:203B20004E46267004F1080018213A4612F02CFBBA4609E04FF0050A06E07F1E401CADF8C1
:203B40000C704FF0060A0490D146B9F1060F15D1089902A888478146049878B101901A48B1
:203B600008210527ADF800100168ADF802706846884703E0089902A888478146B9F1000FC1
:203B800002D10FE04FF004090698079F8DF81490002103228DF8150005AB8DF8167060208F
:203BA00004F0C2FE09490888401C08800020022153F0C6FF09B0BDE8F08FC046580B0020DA
:203BC000201D0020D4330020D8180020841900202DE9F04FAF4C0746201DDFF8B482006845
:203BE0008946ADF13C0D4FF0000B017DADF80CB0252900F00781703005A904F0FDFC0028BD
:203C000018BFC0B240F0418101A804A90DF046FF13F0B8FB00280CBF41F2081543F2C825B6
:203C200004A901A80DF03AFF98F82B0201993B684FF47A7A10FB0AF00AFB1100C01A85420B
:203C4000C0F2DD80D8F80422521A0AFB02F1C91A8D4200F3D480854208DD002806DD95FBBB
:203C6000FAF04FF4916110FB013038609DF81F0000285DD042F204000DF1360110F090F952
:203C800012F082FF0699441A42F206000DF1350110F086F99DF835009DF81D10FF2804BF41
:203CA0000A208DF83500FF2908BF0A219DF835609DF81C507848B4FBF0F2701884B2564630
:203CC000A81054437043A04298BF041C41F20810241805A812F0DFFC9DF81C103D68B0FB67
:203CE000F1F24A43821A11FB06F192B206FB02F3CA1AC91A521B491B8C4201D900290CD531
:203D00006142914216D2002A14D53968B4FBF6F24FF4916312FB031508E061003C684FF46E
:203D20009163B1FBF6F18AB203FB02453D6001E03D68584606460DF1120102A80DF0AEFE0A
:203D40000298D8F804125C46B5FBFAF280180290814203D998F82B32834202D998F89871B6
:203D60002FBB9DF81C00B6180004B04298BF361A9DF81F00002808BF9DF8200024D09DF85C
:203D80001C00B6FBF0F085B2BDF833000FF0A2FF9DF831200146284610F058FC054612F07B
:203DA00067FC024608A9284610F00CFB0CE0814204D8BDF81200401CADF81200BDF8120006
:203DC00098F89B110EF000F889F80000314F88F8F5017868007D052812D1384690F855046E
:203DE00070B999F8000003A9ADF80C0042F20C0004F066FABDF80C00A8F8F00100E065245D
:203E0000204642E013F0BEFA00280CBF41F2081443F2C824214800784FF47A7510FB05F1E8
:203E20003868091BA1F5FA62824206D2A1F57A61B0FBF1F24A43801A386068460DF10E01B7
:203E40000DF02CFE3868009998F82B6205FB0102009216FB05F18A1A944211DCA1F5FA61F1
:203E60009142BCBF00F5FA60386098F89B11B8F878010DF0A9FF0146584689F8001002E0AB
:203E800099F80010652088F8F5110FB0BDE8F08FC00E002010010020A0860100EB10002032
:203EA0002DE9F04F002898461446ADF12C0D00F0F38011F47C1F40F0EC8011F00F0F00F0C8
:203EC000EB8007460591002006900A904FF0000A0990554608954FF0010BCDF810B005460F
:203EE00050460790059805990BEA000021EA0B014FEA4B0B401E059100F0AB80401E70D012
:203F0000801E5DD0001F40F0BE8042F205000DF10E0110F045F89DF80E00002800F0B380D8
:203F20001CB1276694F86B0006900720152607F8010B022301A907F8016B42F2010007F8BF
:203F4000013B10F02DF8684603A90DF0A7FD069810F000F80146019A00983E464018009089
:203F6000824206D8801ABDF80C300090581CADF80C00009B50085146814609041804030CD6
:203F800019430004534610EB090041EB0A0102F0B5FE0090BDF80C309DF80C009DF8002071
:203FA0009DF8011006F8010B181206F8010B9DF8023006F8012B9DF803200935BF1D42E038
:203FC0000220152607F8010B042307F8016BB8F1000F07F8013B0CBF099898F800002D1DAE
:203FE0004EE01CB1E76594F86B00069005201526049B07F8010B0DF10F0107F8016B42F236
:20400000040007F8013B0FF0CBFF02A810F05EFD06980FF09FFF02999DF80F609DF80F30E5
:20402000069AED1D4018000200EB6600B0FBF3F03E4602903F1D06F8012B9DF808109DF8BF
:2040400009309DF80A2006F8011B06F8013B327018E00320152607F8010BB8F1000F07F85A
:20406000016B034607F8013B04BF0A9807F8010B05D098F8000007F8010B98F801006D1D55
:2040800007F8010BADB2059800287FF42BAF2E4661E011F00F0F01D000205DE080468A460C
:2040A00002264FF4803908F1020509EA0A002AEA090A4FEA4909B0F580301AD0B0F5803099
:2040C00014D0B0F500300ED0B0F5802009D0B0F5002004D0B0F580102AD1072404E0062429
:2040E00002E0052400E00424002704E00224012701E001242746A81C214600F08FF947B146
:2041000004F00F04C0F30A0141EAC42141F4004105E004F07F0400F0FF0141EA042105F8BB
:20412000011B0912871929702D18B81C6D1C86B2BAF1000FB9D1022ED8BF00260BDDB01E4E
:204140004FF6FE7708F8010BF019C0F3022040F0A00088F8000030460BB0BDE8F08F70475F
:204160002DE9F04FAA4C07466068ADF1340D80470B900AA9822004F0A9FFA64EBDF82800DC
:2041800038BB00244FF6FF75ADF8284017E0ADF80450BDF82800ADF80650FF210822ADF88B
:2041A000000002A853F06EFB8DF81840D420694602F096FFBDF82800401CADF82800301D4F
:2041C000BDF8281000888842E1DC82200AA902F087FFDFF844920020B246ADF828009DF8EF
:2041E000280000268DF8000069468DF80160D02004F06CFFB0460126F0B99DF80B30012B46
:2042000007D19DF80A0020B90DF1020013F032F990B97D7B002D0CBF0522092246469D422A
:204220000AD10DF1020007F10E0153F0D3FA002818BF4FF0010809D1002E40F0D780B8F10D
:20424000000F03D1787F002800F0D080564600240CE06F490B98896888471A20D4E0BAF8B5
:2042600004006D1CADB24BE0641CA4B2B088A04242DD9DF82800ADF8224008A98DF82000FE
:20428000D12004F023FF0028EED19DF82400FF28EAD0ADF800006946D42004F017FF00281C
:2042A00037D102A8391D082253F094FA0028DBD038887D88ADF80400B8F1000FADF8065007
:2042C00008D0387BBDF82810BD698DF818000DEB81010D61D420694602F002FFB8F1000F6D
:2042E0000AD0387F9DF82510884205D08DF8250008A9D12002F0F4FEB088A04276D100250E
:20430000A84270DDADF80050D420694604F0DEFE28B13F490B9889688847192074E00DF1AF
:20432000080B584613F0A6F8002300B101233C1D181C06D158462146082253F04BFA0028F0
:204340008DD07B8838883A7BADF80630B8F1000FADF80400BDF828308DF818200DEB830106
:2043600001F110010CBF0020B86908220860214602A853F06BFA99F8400330B1D9F89023AA
:204380001AB1BDF8001020469047002401E0641CA4B2B088A0427FF762AF9DF82800ADF872
:2043A000224008A98DF82000D12004F08FFEE82803D09DF82400FF28E9D19DF8000000229F
:2043C0008DF824003B7F8DF8262069468DF82530D42002F085FE08A9D12002F081FEB08872
:2043E000A0427FF73CAFA8423FF433AFBDF82800401C80B20228ADF82800FFF6F0AE044939
:204400000B988968884700200DB0BDE8F08FC046D8180020641E002010010020F0B5044660
:204420000846ADF16C0D401E70D0401E0DD0801E00F00981401E00F0EF80401E00F0E180BA
:20444000401E00F0AD80002042E142F2010007A90FF0A6FD42F20B0008A90FF0A1FD42F256
:2044600006000DF165010FF09BFD42F207000DF166010FF095FD42F2050019A90FF090FD83
:2044800004A80BF05DF806460DF1670142F209000FF086FD9DF86700002808BF002503D0CC
:2044A000022011F052FD0546204607A9042253F0CDF9241D08A90222204653F0C7F9A71CB8
:2044C0009DF864009DF865309DF866109DF8674007F8010B9DF8672007F8013B2B4607F8A0
:2044E000011B610706F0070444EA916005F0030404AD40EA8410314607F8010B0124009571
:204500003846019407F006FE0A309AE042F206000DF165010FF044FD42F207000DF166015B
:204520000FF03EFD42F2040019A90FF039FD04A80BF006F805460DF1670142F208000FF081
:204540002FFD9DF86700002808BF002303D0012011F0FBFC03469DF864009DF8657004F88D
:20456000010B9DF8666004F8017B9DF867209DF86770790704F8016B03F0030705F00706ED
:2045800046EA916004AE40EA8710294604F8010B002700962046019707F0BCFD001D50E058
:2045A00042F2150011A90FF0FBFC13AF42F2160039460FF0F5FC15AD42F2170029460FF00C
:2045C000EFFC17AE42F2180031460FF0E9FC204611A9082253F03AF9083408222046394679
:2045E00053F034F904F1080708223846294653F02DF9082207F10800314653F027F9202083
:2046000066E042F214000DF122010FF0C9FCBDF8221002200A1258E009A80021202253F073
:2046200031F942F2130009A90FF0BAFC09A853F02BF9024609A9204653F008F909A853F0F2
:2046400023F980B244E042F20E0002A90FF0A8FC0DF10A0142F20F000FF0A2FC0DF10B0165
:2046600042F20A000FF09CFC03A942F210000FF097FC0DF10D0142F211000FF091FC0DF108
:204680000E0142F212000FF08BFCBDF808009DF80B209DF80C709DF80D609DF80E509DF827
:2046A0000A1004F8010B02F00102001204F8010B07F0010042EA400206F0010042EA8002BE
:2046C00005F0070042EA4012042004F8011B22701BB0F0BD2DE9FE43A44C80460F46B8F10F
:2046E000450F08D104F511753422284653F0AEF8C4F8345437E112F0C5FBFF2808BFF42041
:2047000000F0328194F8AF14022907D1B8F1E80F00F02981B8F1E70F00F02581944D05EB64
:204720008005A87810B9E978002937D0E978814208BFFB2000F01881B8F1580F24D0B8F13E
:20474000600F1AD0B8F1E00F0ED0B8F1E80F05D03A7890421FDC91421DDB1FE0387894F890
:204760007F1488421AD1FEE097F900000DF0E2F84FF6FF7181420ED010E038880A280ADB8F
:20478000B0F5804F07DA09E038888F2803DB47F60251814202DCE820BDE8FE83774E70688A
:2047A0008047814628786A783946201800F22C4053F04CF8B168484688474046503800F0D9
:2047C000C680801E00F0AD80401E00F0BD808D3800F0B580401E00F09B80401E00F0AC8080
:2047E000801F1ED00D3840F0BE800E2094F8AD748DF8020017B11B208DF8020094F96E147E
:204800009DF90200884204D0E0200DF10201FFF761FF12F07DFC94F8AD04002800F0A38018
:2048200073E0012103208DF8051030278DF8030000258DF808704FF4FA568DF8065094F84B
:204840007F14ADF80060052080298DF8040009DD842907DA8DF8030014278DF8087008200D
:204860008DF804009DF8030094F85114884204D04F200DF10301FFF72DFF9DF8040094F8D0
:204880005D14884203D0572001A9FFF723FF94F87F04842808DB862806DAC0208DF8080038
:2048A0004FF4FA47ADF800709DF8080094F86114884203D05A2002A9FFF70CFFBDF8000049
:2048C000B4F85E14884203D058206946FFF702FF94F87F0478B902208DF805000B278DF85C
:2048E000075024498DF806707D260E80E7200DF10701FFF7EFFEF7200DF10501FFF7EAFEDF
:20490000E1200DF10601FFF7E5FE0EF065FA2AE094F86F040FF00AFE012824D01A20BDE84F
:20492000FE8394F8550418B9022010F053FC1AE0022013F001F816E010F03AFE09E094F913
:204940006E0412F0D3FE0EE011F006FE01E011F0EFFD94F8AF04022805D107480078012822
:2049600001D00CF0ABFA0020BDE8FE831001002020A101006C1E00207C1E0020D818002018
:204980002DE9FE4F0746A148001D00688047DFF8208200248346002F88F803405ED011F0AB
:2049A0009BFB08F596602146AC22064652F06AFF804DA988C80000EB011080B252F0B4FF59
:2049C00008F5A86A0227A946C8F85005B9F8040000EB400080B252F0A7FF7F1E4AF8040BB3
:2049E000F4D1F01DFF21082252F04CFFFF2106F11000082288F8BF1452F044FF0227032396
:204A00004FF6FF7C012288F8D03406F19400A8F8D2C4042100F8042F417083707F1EC170AC
:204A2000F8D106F1A0000525022700F8042F417085707F1EC270F8D1B9F8047086F8A830DF
:204A40004FB12146D8F850057F1E084401F11801A0F802C0F6D1022088F8B40498F8400388
:204A6000554D18B1D8F8440300B180470EF0F6FA98F96E0412F03AFE0FF07CFD11F058FD43
:204A800011F06AFD10F094FD4C4F072657F8040B00B18047761EF9D112F0D4FC464606F1CC
:204AA0005400016809B110F00DFC4548006886F85E40C0B112E0384652F0DCFD029002A82D
:204AC00010F000FC21E0384652F0D4FD019001A810F0F8FB14E0684610F0F4FB52F0C8FC84
:204AE00000280090F7D137480078012802D02046FEF714FC344896F8AF8406F180070470AA
:204B0000D6F880000028DED13F1DD6F884000028D1D1C6F88040C6F8844086F88A4086F832
:204B20008B40B8F1020F86F88C4004BF2748C6F898002748C6F89001264FC6F89471264BB7
:204B4000C6F89831B470254AC6F89C212449C6F8A011244FC6F8A471234BC6F8A831264B28
:204B6000224AC6F8C8302249C6F8AC21234A214FC6F8CC20244BC6F8B0112149C6F8B4715B
:204B8000204FC6F8D0105846C6F8D470A968C6F8D830884706F255415220FFF79BFD96F8A6
:204BA0006F040FF0C3FC0EF059FA2046BDE8FE8F10010020641E0020D818002020020020B6
:204BC000AC3500203D1F0020B8350020157D010043180100837C01006964010015810000F8
:204BE0003DD20000096D0100AD59010045B000000599000079550100D3E60000F99C000078
:204C000039210100A1FF0000E9280100D81800202DE9FE4F0546287D012808D195F917007D
:204C20000CF088FE4FF6FF71814200F016819548EF7B017894481FB990F88B208A4208DB9D
:204C4000012F03D190F88A208A4202DBF120BDE8FE8F80462E6A95F83500B5F8289095F820
:204C60003470AC8B4FF0000A5FEA060B029017D098F84033002B2FD0D8F8581300292BD0B1
:204C800006F0FF008847D8F8581306B20BF47F008847361830B2001D00B2C83086B200E001
:204CA000C8260CB1241DA4B298F86404012809D147B1764802993F1897F804A0405C8019A7
:204CC000401D86B209EB040080195044801C80B252F04EFD071C02D11A20BDE8FE8F09EB69
:204CE0000A0033193881002C03EB070078600EBF0020B819801C00217822C7F8A40007F13C
:204D00000C0052F0BFFD09EB0600FF2110220019A7F84C0007F13C0052F0B4FD07F12C00EE
:204D20000F21102252F0AEFD00243C707C707868696A2A8D52F08AFD07F1840005F12C0196
:204D40000B2252F083FD07F19000294612F094FA6889A7F89A00287B87F89C00687B05F11C
:204D60000E0687F89D00326869460A60706848609DF800102046012908BF01209DF801100D
:204D8000012908BF40F004009DF80210012908BF40F008009DF80310012908BF40F0100045
:204DA0009DF80410012908BF40F020009DF80510012908BF40F040009DF80610012908BF62
:204DC00040F080009DF80710012908BF40F48070A7F89E00A87D87F8A000E87D87F8A1005C
:204DE00095F8380087F86C00AA8BA7F8A82022B1D7F8A400A96952F029FDA87F87F8AA0057
:204E0000286AC7F8AC00B7F8A800C0B1D7F8A400A8B17868401E7860F82101707868401E23
:204E200078600470B7F8A810B7F8A8607868401A786038898019801C38817868B865B7F89B
:204E40009E00410A16D395F83710042905DD00F0040100F00100084302D0E820BDE8FE8F60
:204E600008F1900630460CF0F9FA95F83710304612F0A2F998F80000394652F06FFB204636
:204E8000BDE8FE8F641E002010010020FC9D01002DE9F04F0546954C6F780026ADF1540DE6
:204EA0003846312810DC312800F0D680002800F01681401E00F00C81401E00F00581B0F191
:204EC0002E0700F0E180FDE0323800F0AE80401E4ED0401E012816D9801E40F0F380A88884
:204EE00002280DD12068002808BF182109D0A86852F0B3FE2168884712F0CDFC014600E0D4
:204F000027213620DBE010342068B84668B3A86802A911F0E4FFB8F1340F034618BF301C5C
:204F200002D152F09AFE9B1C13F8017BB8F1350F024603D1A988B81D884213D0B8F1340FDE
:204F40000ED1A98807F10800884209D1009364683B4602A803C8A04712F09DFC014605E09A
:204F6000272103E024683A46F3E718214046A6E0A88808284BD10C342068002845D0A8684A
:204F800004A911F0ACFF024652F067FE95788346F82DC8BFF825DFF858814FF0080A042005
:204FA000AF1CADF83A00D8F80010ADF838A05FFA87F90EA8CDF83C90884720BB109807462B
:204FC00008B3801C0090246804AB93E803005A462B46A047041C07D13C70494633203A4633
:204FE0007D7012F08BFD02E012F055FC04460520ADF81A004546ADF818A02968079706A812
:2050000088472CB96EE01A2402E0182400E0272411A8314602220CF0DBFB8DF84440332085
:2050200011AA022112F06AFD5CE0A888314605280BD11834206840B1A86808A911F04FFF68
:20504000226808A803C89047014612A852F0D7FD3220042112AAE5E7A888052811D10834E3
:205060002068002808BF18210CD0A8680AA911F036FF22680AA803C8904712F00CFC01467C
:2050800000E0272131201AE0A888092815D1241D2068002808BF182110D0A8680CA911F0BF
:2050A0001EFF52F0C9FD246802460CA803C83346A04712F0F0FB014600E02721302012F06A
:2050C00083FB0FE026260DE00A4A02200521A9E713A8432152F0BBFD13AA0120A1E701205E
:2050E00010F07AFB304615B0BDE8F08FC8060020D8180020F8AB01002DE9F04F8146D9F84D
:2051000000600C465FEA0208ADF11C0D14BF00214FF0FF3106F14805284612F0AAFBAA4617
:20512000002818BF0B2040F00B8188480025F460B8F1010F057007D06570022010F000FE46
:20514000062010F0FDFD01E0012060702078012840F2AB80801E012868D9801E012832D965
:20516000801E012800F2DD8012F0AEFD4FF080578346D7F8DC11A0784E6A0090217807F5DC
:20518000EE772846062908BF0120019001200290A068228A6368E168B0470646584612F036
:2051A00095FE002E40F0BF80B8F1000F02D012F0DDF802E0484610F0B1FE002800F0A48003
:2051C0003868806A2BE012F07FFD83464FF0805CDCF8DC0101270068009726786368A1688E
:2051E000A278AE46042E0CF5EE7408BFBE46064618467346B0470646584612F067FE002E68
:2052000040F09180B8F1000F02D012F0AFF802E0484610F083FE002876D0206840688047C4
:205220004949C1F8B0510D6006467CE012F04CFD07464FF08053D3F8DC01E18A80690091D6
:20524000E1680191218B0291A1780391217D04910122059221782E4603F5EE75022908BF40
:20526000161CE1786268A36884463046E0470646384612F02BFE002E55D1B8F1000F02D094
:2052800012F074F802E0484610F048FE00283BD02868006A8047061C45D12868A168E28AB9
:2052A0002369C569E078A847BEE712F00DFD83464FF08052D2F8DC01E18AC0680091E1684E
:2052C0000191218B0291A1780391217D04910121059127782E4602F5EE7507B90E46A368D9
:2052E000E178626807463046B8470646584612F0EDFDC6B9B8F1000F02D012F037F802E0D7
:20530000484610F00BFE08B9142019E0286840698047061C07D1286802692169E07890475A
:2053200082E74FF0FF36B8F1010F05D0022010F0A1FA062010F09EFA504612F0DBFC3046A2
:2053400007B0BDE8F08FC04650450240B73500208E492DE9F04F06460822ADF16C0D15A813
:2053600052F074FA8A4C94F8F30106F1280A06F12807002800F007817078002840F0038174
:20538000FF20844B8DF818001D78F06C012105AA02F05CFADFF80092DFF8008228B99DF840
:2053A000180008B99DF81C5070BBB08900F00700022814BF04200520B073B08900F007001F
:2053C000032807D173684046001D01681878042800F09C8096F83000022815D148468178C6
:2053E000012911D000F22C410D46022206F12800203111F0E1FA38B905F116010DF13E0046
:2054000052F09CFC0DF13E07706E002800F0BB80012102AA0BF041FC002840F0B4809DF817
:205420000800B073F06C40B1394612AA0DF14A03FCF7EAF8002840F0A6800DF14A00009043
:20544000706E394612AB07F0AFF9002840F09B804846801C0078012854D04FF4005013A9E2
:205460000EF09EFD13A815A9082211F0A5FA30B113A83946082211F09FFA002842D194F8AA
:20548000990100283ED0D4F88851B4F8846142F2010004A90EF084FD049A4FF00041002067
:2054A000E5FB0210051CD4F8900112F0BEF92D180498A84202D8761C2D1AB6B24746786870
:2054C00080475FFA80F8D4F88001A84205D1B4F87801B04208BF00260BD0C4F88051A4F81F
:2054E0007861002084F8750111F04EFB0126C4F88C01B968404688470EB10CF045FD012073
:2055000084F89801002084F899013CE0CDF85CA08847AB46224D0A274FF00008CDF864A0F3
:2055200096F83090189014F809A0287A484505D119995246284611F03FFA20B17F1E05F165
:205540000C05F2D100E0A8465FEA08070ED194F87001134A0C2110FB0127401C84F870016F
:20556000C0B20A2804BF002084F87001179938460A2252F06BF909491898896887F80AB08B
:2055800088470420B0731BB0BDE8F08F54A50100C00E00207B1E002010010020D818002024
:2055A000B80F0020F0B542F20400ADF12C0D0DF123010EF0F5FC42F205000DF122010EF0E7
:2055C000EFFC42F2010069460EF0EAFC814C82489DF82310C4F8A801642011FB00F1C4F817
:2055E000A0117E49C4F8C4119DF8221011FB00F0C4F8BC017A487B4EC4F8E001B07888B3DB
:2056000042F203000DF106010EF0CAFC11F030F805460DF1060029460DF030FE2D1A9DF89C
:20562000220084F89B5170B1009860B104F5DC700EF000FB04F5BA700AF008FF012084F817
:20564000940184F8980142F202000DF106010EF0A7FC0DF1060011F007FA04F5CE700EF089
:20566000E9FA11E042F202000DF106010EF098FC0DF1060011F0F8F904F5CE700EF0DAFA8A
:2056800004F5BA700DF078FB96F87F0410F088FBC07B022804BF012084F8F40194F8F801A4
:2056A000002840F0958004F128000021382252F0E9F80026A681E08900EB800080B2054624
:2056C00052F032F9206131462A4652F0DBF84648464FE06304F1300067630EF0ABFA42F2B4
:2056E0001B0001A90EF05CFCBDF8040001A9A4F84C0042F21C000EF053FCBDF8040001A944
:20570000A4F84E0042F21D000EF04AFCBDF8040009A920835D200FF025F89DF82400012782
:2057200000280CBF84F85C6084F85C70B4F84C0028B100EB401080B252F0F6F86065B4F817
:205740004E0030B1410001EB800188B252F0ECF8A065208B20B1C00080B252F0E5F86061B9
:2057600023490DF11A00082252F070F8354609E060690DF11A01082200EBC50052F066F811
:205780006D1CADB2208BA842F2DCB4F84C50668355B1606D4FF6FF720146A0F81F206D1E5B
:2057A0008E7701F12100F7D1B4F84E504DB1A06D4FF6FF71024681806D1ED67002F10600EC
:2057C000F8D1201D3146062252F05CF884F8F8710BB0F0BDC00E0020853C01000DC20000C2
:2057E0002F7C010010010020F5AD0000002A751554A501002DE9F04F7C4C02204FF0080AEC
:20580000ADF1540DADF81A002168ADF818A01020079006A8884700280CBF089F00270126B8
:20582000A14609A8ADF824A0D9F80010ADF8266088479DF828106E4C0B982170606067B1F9
:20584000D020387000257D70B970FD703D710220BD603946FD600FF073FB304611F0BAFEA3
:20586000A046E22008F10C0111F020FD182050F09FFF88F801005F48C8F808000EF052FACC
:205880005F4D5D480227382245625E4C47705B496280037801625C4D8670042764222370E5
:2058A0005B492F70594C2F7504F10C0052F0E0F94FF0000B574DA0606F68574C8DF840B063
:2058C0006FB110A8A11D009012AB0A6889881A6012AA998092E8030033465A46B8472A68EC
:2058E0004AB1A11D12A80B688988036012AF818097E80300904721680DF14100016027796A
:20590000077146480068400805D341208021062210AB03F009F8424C04F1140004F108018B
:205920000AF06CFC6060584652F05EF95E46A51E074605F802BF02206870304652F05AF997
:20594000014660683A46C9B20FF072FB761C022EEFDB344904F12000322252F089F9324C1D
:2059600004F10C00211D0AF049FC4FF0FF37072620600324ADF808A00A20ADF80A00D9F869
:205980000010039702A888470028F3D1ADF830A0D9F80010ADF832600CA888470E9D002815
:2059A0009DF836209DF834000F95E3D198F8001091420ED198F80110814207D0D8F8081066
:2059C0004B6C33B159462A46984702E02846FDF789F90F980028CDD0ADF810A0ADF81240C0
:2059E000D9F80010059504A88847C3E7D8180020181E002088190020580B00209D36010089
:205A0000517701001C1D0020D43300205C1C0020792A0100D0060020F8AB0100801E0020A9
:205A2000681A0020917A0500D01D002001282DE9FE4F40F0F480DFF820A2DAF8DC00012807
:205A400040F0EA800220CAF8DC0010F0BDFC01200EF098FF5FEA000805D00120CAF8DC0098
:205A600010F0C6FCDDE012F049F9704D6E49029000200860A86A00680146012088470128FB
:205A800018BF002003D100200CF0EAFA0120684F00903868112011F0E9FF00280CBF002402
:205AA0000124102011F0E2FF08B144F002040F2011F0DCFF08B144F004040B2011F0D6FFBB
:205AC00028B128685B49006B0246088890470A2011F0CCFF28B128685749006B024608885D
:205AE000904756480126066028688069014644F0200088475248066011F0B2FF00F001011D
:205B0000DFF844B10191400816D2286A806801464C4888478146B9F1040FF6D0B9F1010FCF
:205B200005D1286A406802464648032190475946086820F0030008604448006842F2107250
:205B400040F2AA23B0FBF2F15143401A83422CBF40484FF040403E49086028683968806BC8
:205B60008047019801280ED0B9F1010F05D1286A40680246334831469047DBF8000040F0E0
:205B80000300CBF80000286840690146204688470B2011F06BFF28B128682649C06A0246AA
:205BA000088890470A2011F061FF28B128682249C06A0246088890472048032206602049EA
:205BC000CAF8DC2000230B602868406B0146204688470128F8D1386804200EF0D3FE0446F3
:205BE0001148009D06603868012D02D130460CF037FA11F029FF08200EF0C4FE074602980D
:205C0000CAF8DC6012F04AF910F0F2FB57EA040018BF4FF0FF3804E06FF0040801E06FF033
:205C200001084046BDE8FE8F0C400940B80100102C2009404EAA01004AAA01002820086012
:205C40008001044300400340242208401C1400501C00094008E7A480041600207B4A2DE95E
:205C6000F84F8146854C5068800806D2106804F15001000C40F0F0000870D2F808B0DFF872
:205C8000D081754F641E5E46B00E11D2700E0FD3802084F820004FF6D801A4F861103D46DE
:205CA0002074A5F170000068C0F304600BF048F9684D55F8180CBA46C0F3400018B96749F5
:205CC0000020086001E046F040666549F00EB70E80F001004FF0805300F00100086087F0BB
:205CE000010000F001008860D3F8F06103F5F87072680090594648469047DFF86891DAF83E
:205D00000070594B39F83B2C07F0FF06101280F0C000B04211D002F0FF021968B04234BF5D
:205D200001214FF0FF3140180102864281F4404142EA010129F83B1CEFD13809C7F3033124
:205D4000C7F384466FF4017200F0F000014304F80810F90CA65401F0F00040F47040A4F851
:205D60006300DAF8046028681F4620F0100828F4F070286057F8080C5FEA9B6002D25FEAA5
:205D80005B6017D255F8180C800834BF300AF00800F0F80040F47840A4F86100207800F0E8
:205DA0007F002070207840F080002070C6F304400BF0C6F846F3050321783A6841F3050091
:205DC000984211D09842B4BF01224FF0FF3201F04001801800F03F020A43227021788342F0
:205DE00041F080012170E7D138683868C5F800801E4957F8080CDAF814004026C0F305302D
:205E000089F8A30F43F61803E675009A0B8010688168584688471649164A0AE0105C93788D
:205E2000141D834299BF204410F8010C20444078086008684B689842FCD10228EED1012043
:205E400048620D4F3860BDE8F88FC046AC4F0050FEFDFFFF28000940F813005094042A435D
:205E6000000220436BA00C40342009406AB00C4000600C4028AC01009404604206620840F8
:205E80002DE9F0477B4A854D7B4C117895F8AFC4012891464FF00101A0706F68117040F2F3
:205EA0009780DFF8D881DFF8DCA1801E47D0401E35D0401E00F09F80401E1FD0401E40F0E7
:205EC000A78097F86D00608197F86E60002E06BFE1700E1CE6706A495046007809784546D0
:205EE00005F1440311FB00F04643B1002964187820F00F0040F00300187089E0BCF1010F12
:205F000040F086800020F98A6071C90934BF95F8511495F87A14617011F046FD56E0BCF10D
:205F2000010F09D195F87F040FF03AFFC07B022802D1002009F0CEFD0FF0BAFD46E052489D
:205F40000668BCF1010F1DD09AF800008700F06B8047DAF804103C23401AB0FBF7F1B1FB10
:205F6000F3F25A43891A227812FB03F0401A3C301FFA80FAF06B804707FB0A0140460164EF
:205F800044301DE09AF800008700F06B8047DAF804103C23401AB0FBF7F1B1FBF3F25A43F5
:205FA000891A227812FB03F0401A3C301FFA80FAF06B804707FB0A014046C0F8C810CC300A
:205FC000017821F00F0141F0020101706F681FE00021FE8A6171F10934BF95F8511495F8C5
:205FE0007A14617078B995F82F0460B10229C4BF0220607007E097F86900607197F86A00F7
:2060000060700026A67100F077FC6F68002F2FD01E4806785EB97968087800F0200020710E
:206020008878E0710878800901D211F049FDA078032803D0022818BF062819D1144D68688C
:206040008047A17802290CD012490F7817B912490F7837B1022189F80010A9688847BDE8A4
:20606000F087832189F80010A96888470BF030FBBDE8F087BD350020481D00207C1300200C
:20608000791E0020701D002040180020B5350020D8180020B9350020BB35002010010020BB
:2060A0002DE9F043002B08BF002A10D10029BCBF00204FF0004106DB50EA01071CBF6FF0F9
:2060C00000006FF000410CF0D6FCBDE8F0835FEA530898EA610803D50026404266EB0101D8
:2060E0005FF0000913F0004E03D00026524266EB03031C461546002C08BF8D429CBF2C1CF1
:206100000025070C47EA01470E0CB44208BFBD429EBF240444EA15442D04070A47EA016711
:206120000E0AB44208BFBD429EBF240244EA15642D02470847EAC1774E08B44208BFBD4268
:2061400000F29280870847EA81778E08B44208BFBD427BD8C70847EA4177CE08B44208BF93
:20616000BD4265D8070947EA01770E09B44208BFBD424FD8470947EAC1674E09B44208BF73
:20618000BD4239D8870947EA81678E09B44208BFBD4223D8C70947EA4167CE09B44208BFBB
:2061A000BD420DD8E60146EA5566EF01B14208BFB84201D3C01BB14159EB09094EEB0E0E39
:2061C000A60146EA9566AF01B14208BFB84201D3C01BB14159EB09094EEB0E0E660146EAA6
:2061E000D5666F01B14208BFB84201D3C01BB14159EB09094EEB0E0E260146EA15762F01E2
:20620000B14208BFB84201D3C01BB14159EB09094EEB0E0EE60046EA5576EF00B14208BFF4
:20622000B84201D3C01BB14159EB09094EEB0E0EA60046EA9576AF00B14208BFB84201D300
:20624000C01BB14159EB09094EEB0E0E660046EAD5766F00B14208BFB84201D3C01BB14121
:2062600059EB09094EEB0E0EA14208BFA84201D3401BA14159EB09094EEB0E0EA34208BF77
:20628000AA423EBF2D0A45EA0465240A8AD373464A465FEA080803D50026404266EB010146
:2062A0005FEA480803D50026524266EB03031E4617460B46024631463846BDE8F08370473E
:2062C0002DE9FE4F0CAF9946934604467D680291294604F0D9FF061C00F0EE803888F08239
:2062E000774F347597F8400318B1012C04BF1520307506F1840029460B2251F0A7FA012CA4
:2063000004D00D2C1CBF7068401C00D170683062002597F8400335650028B5654ED0052C04
:2063200018BF012C45D14FF0040A86F86BA0F08A86F86950C00934BF97F8510497F87A040F
:2063400059460A2286F86A0006F1700051F07EFA9BF8080003282CD1032097F855340290DA
:206360003BB3DFF8608108EB8408D8F8000010F47F0F0ED086F82CA0D8F8000006F12C017A
:20638000012200F47F003063304602F021FDD8F8000010F0FF0F0CD02A2086F83C00D8F8C0
:2063A000000006F13C0100F0FF003064304607F059FB97F8400308B10D2C13D0009502998E
:2063C0004B4630465A46FBF753FF071C75D1E41F012C03D8707E40F020007076304606F0CE
:2063E00099FF6AE00520374C86F86B0004F13400016811F0F70F18D02A2186F83C10BA7862
:20640000006806F13C01012A00F0FF0030641CBF20F00800306497F8550418B9306C20F046
:2064200002003064304607F01DFB009502994B4630465A46FBF71CFF5FEA00083AD1224897
:2064400006603489756801A964200EF08BF91F4EA01C0DF1050187B206F1D0000780E920CF
:206460000EF080F99DF80500012806D13C46C4F30220022140F0180006E0241D0421A4B2A3
:20648000C4F3022040F0080005F8010D671A05F8014DB9B2C6F8DC50AD1C28460AF086FC0C
:2064A0009DF8040000280CBF09480A48C6F81801C6F8D800474600E01A27F8B2BDE8FE8FB6
:2064C00010010020D89E0100D01B00207C1300204E9055550E7A55552DE9F047044694F87D
:2064E00030900F46984615468B20ADF1300D0DF10A0102F0EBFD8A20694602F0E7FD94F82A
:20650000250000283ED1B9F1000F19D1BDF80A104FF6FE70884205DCBDF80A1088422FD1B6
:20652000694615E0B4F844009DF80A608DF80C0000128DF80D00BDF80A008DF80E601BE0E6
:20654000B9F1020F09D0B9F1030F19D104F1280103A851F0F3FB092612E0207CC00934BF90
:20656000B4F84200B4F844008DF80C0000128DF80D00208D8DF80E00001205268DF80F00F7
:20658000002013E002280CBF05260926012818BF04F11C0104D1892006A902F097FD06A925
:2065A000324603A851F052F994F826000DEB0601C8723A4603A831460BF034FA002840F01E
:2065C0008F80B9F1000F19D1BDF80A104FF6FE70884205DCBDF80A1088422FD1694615E09F
:2065E000B4F844009DF80A608DF8200000128DF82100BDF80A008DF822601BE0B9F1020FD3
:2066000009D0B9F1030F19D104F1280108A851F095FB082012E0207CC00934BFB4F84200FC
:20662000B4F844008DF8200000128DF82100208D8DF8220000128DF8230004203E6881466E
:206640000BA9822002F042FD9DF82C10307B8142D8BF9DF82C00002842D0074600244FF032
:20666000180A722029460FF05FFEB0689DF82C100019C8F80000007881422DDD296810FBF8
:206680000A1028600146D8F800004278012A1FD083782BBBB9F1040F06D0091D08A851F0E2
:2066A00035FB012816D017E008884B888DF82800042208A98DF82A3000128DF829001812F4
:2066C0008DF82B000AA851F085F8012802D003E0807828B9002004E07F1E04F10304C0D1B5
:2066E000F3200CB0BDE8F08784462DE9F84F7848DFF8FCB1DFF8DC91784EDFF8E481794D38
:20670000DFF8E4E1DFF8E4A104787348012C57D04F4601243C7000244FF0E04704701F4033
:2067200004EA0200347008BF00283DD10820274610401F4008BF00282DD0424692F9000085
:20674000B5F8A230401E107042F201429A4202D0121D9A4209D170460068826C6046904749
:20676000008842F6014181420CD1688FB0F5105F16D158460068514600F5C07008600FF05C
:206780007DF918E0E12009F017FE98F90000002800F08F8091E0454695F90000401E287044
:2067A0001D2009F009FE06E0454695F90000401E287010F053FE98F90000002879D07CE0F8
:2067C0004F4601243C700024047005F186003470068814EA03074FF0020000EA020008BF11
:2067E000002813D120464FF0E04710401F4008BF002803D11D2009F0DFFD4BE0454695F9F9
:206800000000401E287010F029FE43E0424692F900305B1E137043F20842B24208D0B5F801
:206820006A70931CB34203D0BA4218BFBB4212D170460068826C60469047008843F6030106
:20684000814206D008F0DAFD98F90000002830D033E0B5F86A70B5F8C21043F604008842F7
:206860001CD0B8421AD0B5F88620904216D0B1F5505F05D0080B0BD31D2009F09DFD07E06B
:2068800058460068514600F5C07008600FF0F6F810F0A8FD98F9000058B10EE015480078DF
:2068A00002280DD003280BD008F0A8FD98F9000018B92046FCF732FD05E098F9000002E0EC
:2068C000204609F079FD89F80040BDE8F88FC046BF0500203D1F0020301E00202F1E0020B5
:2068E000361E00207C13002040180020381800200C0100214A1D00202DE9FE4FDFF8E0813D
:206900000025804C98F8AF048DF800506678019011F04BF94FF0010B0BFA06F2DFF8C89142
:20692000744E4FF6FF718918014098F84003618138B3D8F8782322B342F21A00694690474A
:20694000684867790378B3B1AFB99DF8003093B1D8F89C0378B1804707464946701C09780F
:2069600000783FB16389083010FB01F0B7FBF0F15818608167799DF80010608907FB01003A
:206980006081A078002840F09280607898F8AF14574C012966D155480068C06B80478246A6
:2069A0000CF02AF9074604F1900299F8000011780223800063F3030107FB00AC11707178B3
:2069C000C4F88CC0083189B200FB01C204F17401087863F30300087004F1CC0322671878E5
:2069E00065F30300187098F8AF04012836D110F05FFE98B34946226F486890422ED204F102
:206A00009002107865F30300107004F17403C4F88C50187820F00F0040F003001870097892
:206A2000707804F1780608308B0082B203FB02F02067307804F178026BF3C300307010782D
:206A40006BF3041010704FF4FA53A4F8865007FB01F0C4F880300FF0E3FD2AE01C2009F0C5
:206A6000ABFC26E0A4F8AE5098F85D1484F8B01098F8507484F8B17094F8B21004F1B202AA
:206A800041F0200184F8B210117804F1B20621F01F0141F002011170317865F38711317010
:206AA00084F8B35084F8B40084F8B55001E003F07BF80198022810D10F481149007848B991
:206AC0000E48007830B98322084602700AF000FEBDE8FE8F022208460270BDE8FE8FC04654
:206AE00010010020B5350020701D0020401800207C130020781E0020B9350020BB350020B3
:206B0000BD350020481D00202DE9F04F794C6068ADF12C0D002840F0E38004F18006306857
:206B2000002800F0DD80DFF8C49109F123000078022800F0D580704D281D006880470A90E5
:206B4000D4F88000074678B3674E4FF0000A4FF01D083B7D0820711E11F8012F9A421ED09D
:206B6000401EF9D162483946524650F065FD787E30F07F0005D194F88B00401E84F88B00A3
:206B800004E094F88A00401E84F88A0087F8018057F80CBC384609F06BF95F4602E0BA461E
:206BA00057F80C7C002FD4D1352009F07DF8A9684E46002862D1452009F076F8A968002862
:206BC00056D1684601A90AF069FF4948006838B1017D252904D050F80C0C0028F8D113E00E
:206BE00090B196F89801002838D010F0CBFB00280CBF04210D21009F96F82B02401AB84243
:206C00001FD8012086F89501152009F04DF8A968A8B10A98884760680DF10601703001F09C
:206C2000EBFC10BB96F82B020099884203D91C2002F0BCFD54E0002086F896010AE00A98CC
:206C40004DE0252009F030F8A9680A988847002086F895010420FFF713F941E0252009F066
:206C600023F8A9680A988847192001F0F7FB37E00A98884708200CF069FD31E00A988847C7
:206C800096F8F401B8B10FF05FFFB18901B9F1893269491E89B201EB81018918D1F8011017
:206CA00011F00EF842F21071814292BF00206431081AC0B200E000206968002808BF0620D5
:206CC000D9D0C6F8D80188470446D6F8E011D6F8D80106F5F4720EF065FDA96820468847EE
:206CE0000BB0BDE8F08FC0464CA50100C00E00209001002010010020D81800202DE9F04196
:206D00001C4615468C4208BF854282BF00230022E5E0002C08BF002D0AD100290EBF0028F6
:206D20006FF000006FF0000100F0E1F8BDE8F0815FF000085FF0000E002C08BF8D429CBFE4
:206D40002C1C0025070C47EA01470E0CB44208BFBD429EBF5FEA044444EA15445FEA05455C
:206D6000070A47EA01670E0AB44208BFBD429EBF5FEA042444EA15645FEA0525470847EA2D
:206D8000C1774E08B44208BFBD4200F29380870847EA81778E08B44208BFBD427CD8C70877
:206DA00047EA4177CE08B44208BFBD4266D8070947EA01770E09B44208BFBD4250D8470916
:206DC00047EAC1674E09B44208BFBD423AD8870947EA81678E09B44208BFBD4224D8C7096D
:206DE00047EA4167CE09B44208BFBD420DD8E60146EA5566EF01B14208BFB84201D3C01B1D
:206E0000B14158EB08085EEB0E0EA60146EA95664FEA8517B14208BFB84201D3C01BB141CC
:206E200058EB08084EEB0E0E660146EAD5666F01B14208BFB84201D3C01BB14158EB0808C0
:206E40004EEB0E0E260146EA15762F01B14208BFB84201D3C01BB14158EB08085EEB0E0EBE
:206E6000E60046EA5576EF00B14208BFB84201D3C01BB14158EB08084EEB0E0EA60046EA6F
:206E80009576AF00B14208BFB84201D3C01BB14158EB08084EEB0E0E660046EAD5766F00EB
:206EA000B14208BFB84201D3C01BB14158EB08085EEB0E0EA14208BFA84201D3401BA14120
:206EC00058EB08085EEB0E0EA34208BFAA423EBF2D0A45EA0465240A89D3734642461E4667
:206EE00017460B46024631463846BDE8F08170472DE9F843784C714A7248734DDFF8CC816C
:206F0000744E94F8E430591E0B2900F2C980DFE801F0954F6629466629466629C80610680E
:206F200042F2107240F2AB27B0FBF2F15143401A874204D98020383D286000272F60674873
:206F40005F4900260125001D06600E200D6006F0EDFF02200EF08EFC84F8E45084F8E36024
:206F6000BDE8F883042B07D001220A2B40F8252C14BF0221032104E02023012140F8253C0E
:206F80000A4684F8E210002140F83D1C0827C0F8FB7FC0F8FF7F40F83D2CBDE8F883052BF9
:206FA00014BF09200620002684F8E4002E607EE094F8E17001213C38002FC0F81B1004BFF5
:206FC0000621002202D00022EA62032184F8E410032140F8011C2A602868800867D294F8B4
:206FE000E400012603281CD04FF08059D9F8A40140680027702204233946844600974046F3
:20700000E047D9F8A401C06870223946134684464046E04794F8E400062814BF0A20072008
:20702000C2E72B48006840680221702204230746009140460021B8470420B5E7116842F257
:20704000107340F2AB27B1FBF3F25A43891A8F4202D90821403D296001270F2130383760A6
:2070600042F62A2240F8011C4FF08059C0F80320D9F8A40140680225072300214FF4C0723F
:20708000844640460095E047D9F8A401C06800214FF4C072072384464046E047376004E094
:2070A000FEE70020306070600C2584F8E45004F1780010F0FFFDBDE8F883C0461C1400507B
:2070C00004800C403D400C4058600C4000A00C40A401001054600C400416002038500C4064
:2070E0002DE9F04107460C467148DFF8DCC1DFF8CC81DFF8D0E1724902883846D12810DC29
:20710000D12879D0713800F0B180401E00F0AB80401E00F0A480113810D04C3800F08680D5
:2071200007E0D23854D0401E41D0401E33D0401E28D0384610F0A6FBFF2802D1F420BDE842
:20714000F0815C4D05EB8005A97809B9E87850B1E878884208BFFB2000F0A78022789142CC
:2071600069DC904267DB544E70688047074628786A7841464018214650F068FBB168384626
:20718000884791E02278022A55DA0846641C00EB8200042285E021888A424CDDC8007746D1
:2071A000182200EB011039684018241D79E02678304602283FDA2C2505FB0680611C102229
:2071C000393050F043FB616905FB0680C1646BE022786178022A2EDA02292CDA2C2001EBF8
:2071E000420600FB02C34F1C0CEB460C022283F8E8740CF5A96030E02178608802291ADA1E
:20720000824218DD2C2303FB01C595F8E0340CF596629842A4BF431C85F8E03402EB81026B
:20722000D2F8901000EB40000322BDE720786778022800DA17B1E820BDE8F08161462C229A
:207240003D187E1C02FB001368000A2283F8D86400EBC500401800F22C50A41C21E01CB3DE
:20726000084608221DE0FCB1704692E7B4B90CF596600CF59561022700F17C020CF5A86CB5
:20728000983041F82C2F5CF8043B08617F1E02F10A0200F104008B60F3D105E04046582271
:2072A0002430214650F0D2FA0020BDE8F081C046681E00207C9E0100D8180020C005002015
:2072C0006406002060060020100100202DE9F04FDFF8CC8198F83904ADF1240D059098F833
:2072E0005804069098F82F04079098F864044FF0000B01280AD198F8E0713FB1664898F8ED
:20730000E1113F18445C3D79641D01E05D465C4698F88A60082EA8BF072698F83874F000B7
:20732000C1B278180019A13084B26019801C80B250F01EFADFF864A1DAF80490071C08BF5F
:207340005C4600F0A4805946902250F09BFA3819786098F838243D81D8F834147868841AE8
:20736000801A50F073FA3C62C8473546D946641ED8F88060049016E0707EC00911D371684F
:207380004878C0F3810003280BD1E41F491D204650F0D4FC6D1EEDB2641E09F110005FFA04
:2073A00080F956F80C6C002D18BF002EE4D1DAF8081004988847DAF804008047D8F8806005
:2073C0000EB37168491C0A78C2F38102022A16D1727ED20906D2317E890910D34FF0010BCF
:2073E0006DB910E0497904F80119716849796D1E09F10103EDB25FFA83F904F8011956F8A3
:207400000C6C002EDDD1DAF80810884704F801990020079E059D04F80109069B98F82D24DA
:2074200098F8021041EA420146EA8101090141F00F0104F8011945EA0311217079683E89AD
:20744000091BCAB2B11839817C6004463C65F882BC650B22387508F5EC718DF80C0007F1EA
:20746000840050F0F3F9BBF1000F03D0F88A40F00800F8820FF092FF01AA2346014600941B
:207480003846FAF7F5FE18B1384650F0EBF92746384609B0BDE8F08FFC9D0100D8180020AD
:2074A000100100202DE9FF470546DFF8C8A168789AF8AF14002840F0D18095F89A20022A63
:2074C0001CBF032AE82095F88F20802AC8BFE820012911D195F89010092901DB0A2900DDD0
:2074E000E82095F891700FB1042F05DB802FC0F2B480882F80F2B180002840F0AF809AF81B
:207500007F0495F89110884204D005F19101E820FDF7E0F805F19001E720FDF7DBF805F175
:207520008F01E120FDF7D6F805F19C015020FDF7D1F895F89A0002280CD04FF6FE70AAF8B6
:207540004C0405F192010AF2424050F0F7FB05F1920604E005F192063088AAF84C040AF5F9
:20756000017005F184010B2250F070F94FF001080220A5F816803146287501A80FF07CFE76
:207580006B68B5F89C905B1E6B60581E686005F19E000EF0B5F8187069682F7D0024481CF1
:2075A0002862781E087028892C659AF84033AC65801C002B288141D0042785F86940E88A97
:2075C00085F86B70C00934BF9AF851049AF87A0431460A2285F86A0005F1700050F036F941
:2075E00095F89A00032829D105F1700005F1920150F0A4FB9AF8550400B31D4E306810F4CC
:207600007F0F0CD085F82C70306805F12C01424600F47F002863284601F0DAFB306810F0DA
:20762000FF0F0BD02A2085F83C00306805F13C0100F0FF002864284606F014FA00942846A4
:20764000832101AA4B46FAF713FE071C02D1284605F060FE381C01D106E0E820687018206D
:20766000287028460BF038FA0090BDE8FF87C046E09E0100100100202DE9FE43DFF8C081F7
:20768000704D0E46B00958D3444604F184074DE00178D0290EDBD02909D181783970C178B5
:2076A00079700179B97085687D60C168B96050F0D9F848E004F1580528600BF00DFA2846AF
:2076C0000DF000FE3FE0884794F88C10491E84F88C10A9688847009801788DF80410A0658B
:2076E0004378CBB1DC2B0DD0DD2B0BD0E42B09D0F32B07D0DE2B05D0DF2B03D0E82B18BF0A
:20770000DB2B0BD105F09AFD9DF80400162805D168460DF0D7FD01E00BF0DEF99DF8040083
:20772000162803D004F158000DF0CCFD38464FF0A1FF002869680090C5D1F00BA946444635
:20774000C00305D0404F4FF093FE002800909FD1700905D32E208DF8040001A80BF0BCF989
:20776000700805D325208DF8040001A80BF0B4F9B00805D326208DF8040001A80BF0ACF9F2
:20778000F00805D327208DF8040001A80BF0A4F9300905D329208DF8040001A80BF09CF9EC
:2077A000F00908D300208DF805002D278DF8047001A80BF091F9300A08D300208DF8050011
:2077C00030278DF8047001A80BF086F9700A08D300208DF8050035278DF8047001A80BF03E
:2077E0007BF9F00A08D300208DF8050023278DF8047001A80BF070F9B00A08D300208DF80C
:20780000050036278DF8047001A80BF065F9606DD9F8041080B18847616D00270091D9F802
:20782000081067658847009804F1580630600BF053F930460DF046FD0020BDE8FE83C046D1
:2078400010010020D81800204C1E00202DE9F043894614460546ADF12C0D69460DF06BFFB3
:207860005FEA000800F0C580AD1C0226284602A90CF0B7F9071C00F0BC809DF80900814519
:2078800009D0ED19BF1908F10200BF1CAD1CBEB2B042EBDCADE0401E05F1020500F08D8084
:2078A000401E50D0801E33D0401E26D0401E20D0401E18BF622040F0AC80202F40F099805C
:2078C0002046294608224FF0C1FF083504F10800082229464FF0BAFF05F1080704F11000D5
:2078E000082239464FF0B2FF07F10805183408220BE0022F7DD1022207E0202F79DC2046F5
:20790000002120224FF0BEFF3A46204629467DE0042F6ED12046294602224FF097FFAD1C4D
:2079200015F8010BA070287800F00100E0702878C0F3400020712878C0F3800060712878D5
:207940004011A07164E00B2F53DB0DF11200002116224FF097FF2046294604224FF076FF2C
:207960002D1D201D022229464FF070FF42F20B0004A90CF015FBBDF81000A188884238DC7B
:20798000A81C10F8011BA17110F8011BE17110F8011B217210F8011BC1F3C202A2720DF112
:2079A000120200F0E1FA20B39DF82700A0819DF81670E78104F1100025E0052F19DB0DF185
:2079C0001200002116224FF05DFF15F8010B207015F8010B607015F8010BA07015F8011BBD
:2079E0000DF11202C1F3C2002071284600F0BCFA08B967200DE09DF82700E0809DF81670EE
:207A0000278104F10A0011220DF116014FF01EFF00200BB0BDE8F0832DE9FC41DFF8AC81D1
:207A20000025044688F8ED5298F8AF24607D062803DBE82088F8ED02607DA17D0E2905DD41
:207A4000032803D0E82088F8ED02607D032806D1B8F85C0040083CBFE82088F8ED0294F880
:207A6000287017B1E82088F8ED02012A12D1E07D092801DB0A2802DDE82088F8ED02207E91
:207A800008B1042806DB802801DB882802DBE82088F8ED0208F53B76214630460EF0BDF85A
:207AA000211D112206F12C004FF0D0FE94F8280008F53B77002804BF88F83453A07D04D0DF
:207AC00094F8290088F83403608DA8F82A03607E88F82C03A07E88F82D03E07E822688F89F
:207AE0002E03207F98F86F5488F82F0398F87E3488F83063364E88F8315398F87F24C8F8E1
:207B00001063042588F8145304F11D0188F8323307F1490088F833230B224FF097FE98F842
:207B2000ED0200284AD16078002847D1207E98F8EE728DF8000017B1EA2088F8ED0204F1B2
:207B40001701E720FCF7C6FD98F8340328B1207E022808BF01208DF8000098F87F049DF8D3
:207B60000010884203D0E8206946FCF7B3FDB8F85204184998F8AF74174E088098F8EE0277
:207B8000A0B103280ED00220307005F0A1F94FF6FF701249A8F85204022F088004BF104960
:207BA000088005E005F094F9032000E0012030702720207028460FF0E7F801E02A20207034
:207BC00020460AF089FFBDE8FC81C0461001002059790100361C0020FC3300208A1800200E
:207BE000E61400202DE9F04F8246ADF11C0D02F0DFFC5D4800780CF045FA5C4D002401286C
:207C000008D90A380FD0801E04D0401E0ED0401E09D006E00FF062FB022804BF01210C1C04
:207C200006D0296806E005211F2401E003210724284601604E4AD068C0F38150012804D13D
:207C400012680120120E904004430FF04DFEDFF828B1DFF82081FF2240185B46401E471C05
:207C6000C8F800007F1E03F8012BFBD1DAF80020002702F0FF03FE2B1CD0D4463B460126D0
:207C800002F0FF05FF2D0ED0A84205D3A94203D806FA05F52C4201D0022062E002F0FF02CC
:207CA0002F430BF802305CF8042F5B1C02F0FF05FE2DE7D1092006F0C9FA3048C0F800A094
:207CC000374801210EF09AF9364D00264FF00109B04609FA06F0044214D1074207BF06F061
:207CE000FF0141F4C0411BF806005AF82010244805F07EF8F0B24FF0FF310FF08BF9C5F88B
:207D0000008001E0042028601A480068761C2D1D8642DED904A80FF0CFFD1A4C20781B4A57
:207D200005901948102104AB0DF090F868460FF0E3FD6068174902901548CDF80C806A4643
:207D40000DF094F9144951F80D0C20F4F85040F4005041F80D0C114AC1F8FF9F4046C2F8B6
:207D6000009007B0BDE8F08FB6350020A41E0020A84F0050A01E0020483400201C3000207E
:207D8000007FC76748AC0100FC3400203170010038330020ED4701000D3009402C00094094
:207DA00018350020303200202DE9F84F6B4C074694F86901002800F0C480B4F85204B7F870
:207DC0004210884240F0BD8007F128000EF088FB002800F0B680002594F8550484F86951EB
:207DE00010B102200EF0D0FF94F80F0210B101200EF0CAFF387C400905D310200EF0C4FFC7
:207E000080200FF0A9FD20200DF0E4F904F5087009F024FB7A685178107804F5047B00EBE4
:207E20000120C0F30321C0F3003684F86511C0F3031384F8583400F00F0184F8666194F8CF
:207E40007B0484F86A110F2804D0884202DDD67806B9014684F8391494F8396484F84052A4
:207E60000F2E09D194F8670102286AD10DF084FD07F0CCF9BDE8F88F39480078012802D038
:207E80000120FBF74BFA3748001D0068804782460EF06EFD2C4B2D4894F8AFC499465A6802
:207EA0001978856C2A4BBCF1010F18BF856DA81A94F8392403F58A78890090FBF1F003EBBD
:207EC0008203D3F814110CF0A1FFC9F8045058F8260020630D4660630CF078FFA16A284681
:207EE0000EF08AFB0BF0AEFB1A4881685046884794F86701022810D1584609F0AFFA94F8E0
:207F0000390404EB4001B1F82C214FF4707606FA00F15846891A0EF03DFD3989022009F08E
:207F20008BFF04F5A675284609F098FA0A48C4F85401D4F8601128460EF02CFD10200FF046
:207F40000BFDBDE8F88FC046701D002020180020FC9D0100D8180020B9300100100100201D
:207F60003D1F0020D81800202DE9F04F154601F00708C1F3C2074FEAA119044683460C2214
:207F8000ADF11C0D002168464FF07CFC5FEA080034D0012879D101A8594603224FF056FCCE
:207FA000E41C14F8010B022200F00F0021468DF808000DF10A004FF049FCBDF80A60A41C27
:207FC0000721DDF804C052486E754268624507D1027A9DF808309A4202D14289B24206D0AD
:207FE000491E00F10C00F0D10020014601E0017840788DF800108DF801001FE014F8013B81
:2080000007218DF8003014F8016B40488DF8016010F80C2F9A4202D14278B24205D0491EC1
:20802000F6D100200246114603E04268017A4089687501928DF80810ADF80A0003A807F08B
:208040007FFA9DF800009DF80110B8F1000F10D0B8F1010F19D10198049A9DF814109DF8AC
:208060000860424071408918BDF81600BDF80A2004E09DF80D309DF80C205940504008185A
:2080800003D1EF701FB1022F07D000203BE0281D214602224FF0DAFBA41CB9F1010F27D045
:2080A000B9F1020F2CD1BDF80A10281DC91DCA1021464FF0CBFBBDF80A00C11D04EBE10457
:2080C000F0B1401E811000EB5171C910C9B249190E798210012700EB527222F00702801A08
:2080E000C0B2401C07FA00F0FF303040087107E0291D20460BF04CFD207804EB8004641C47
:20810000A4EB0B04A0B207B0BDE8F08F580F0020640F0020F8B507466748B0F85C2000218C
:20812000930804D2B7F89E30DB0828BFE82112F0600F04D1B7F89E20920828BFE8215F4E94
:208140003B8906F1080212889A42B8BFE82197F89C5035B997F89850002D08BFF52100F08A
:20816000A780002940F0A480D7F8AC5090F8401315B9012903D026E0002900F0988097F824
:208180009840002C18BF032C05D1D7F8AC5045F00A05C7F8AC5015F0FF0F07D02A21D7F831
:2081A000AC5087F83C1005F0FF01396415F47F0F07D00421D7F8AC5087F82C1005F47F01D4
:2081C000396390F84013002441B397F898504268042165B925233B75D28AD20934BF90F802
:2081E000510490F87A0487F86A00801C08E015233B75D28AD20934BF90F8510490F87A04C2
:2082000087F86A0087F86B100A2207F1700087F8694007F190014FF019FB01E00120387534
:2082200097F8A050B7F89E00FD7697F8A130F8827A683B7797F82C103A622546BD650F2965
:208240003D650AD0B7F8A80007F12C01224600B90122384600F0BCFD04462CBB97F83C00BF
:20826000FF2801D1B86D28B107F13C01384605F0F9FB0446C4B9009597F89C10B7F89A305B
:2082800007F190023846F9F7F3FF041C0CD130893989884203DB384605F03CF804E0E52044
:2082A0007870384607F0E4FD211C01D1F8BD1821384607F0EDFFF8BD10010020641E00209A
:2082C0002DE9F84F0F4680460EF026FE4FF6FF71814208BF682000F0B8805D4E440004EB37
:2082E000C004A419D4F8026016B9D4F8065025B3D4F80610B14208BF692000F0A6806078F3
:20830000401E13D0401E09D0801E16D13868864200F295808142C0F092800EE038888642F6
:2083200000F28D808142C0F08A8006E03878864200F285808142C0F08280464E70688047C4
:2083400042F2020BDFF8109100904046A0EB0B0001282FD90A3801281CD9C01F49D1207896
:2083600062784D460021281800F5FE704FF08AFA637838464FF088FA05F5FE798342D8BF22
:20838000181C02DD38464FF07FFA2178024601EB090034E00EF06CF9B668398888424CDD75
:2083A000207862784D463946281800F5FE704FF04DFA28E00EF05CF90546384629460AF083
:2083C0005DFFB6682D1A5FFA85FABAF1000F34D0207862784D463946281800F5FE704FF0E0
:2083E00035FA5846404514BF85F89BA185F89AA109E0207862784D46281800F5FE703946D7
:208400004FF024FAB6680BF11900404504BF0020A5F884020BF11A00404513D1B5F884721F
:20842000B5F88202C119322901DC07430AD10220A5F882023027A5F884720098B0476A208E
:20844000BDE8F88F0098B0470020BDE8F88FC046E0A50100D8180020C00E00202DE9FC4138
:20846000644C064694F8400394F8AF84002798B1D4F8782382B1D4F8980368B142F21A009A
:2084800069469047D4F89803804728B19DF8000010B1E12E08BF0127B8F1010F04D194F8E1
:2084A0007F040DF07DFC01E00FF0FEFAC07B02280CBF052501256068002800F09280002E4B
:2084C00077D01B2E06D1017D052903D094F8AE34002B6ED0E92E29D047BBE12E16D10FF0D8
:2084E00097F890B16068C18AC9080FD294F86014817694F84E144A1C84F84E244068817015
:208500002846FDF7BDFCBDE8FC8160681C2E51D1616A002952D08847334900200978606028
:2085200001295ED0FAF7FAFEBDE8FC81F1200EF0B0FE61688F7E4FB90FF06AF820B1606843
:20854000C18AC90836D2D1E7606833E0B8F1010F04D14868098908F029FC61684868008876
:20856000000905D394F8407317B10DF06DFA6168C88AC00811D3087E00F07F000876087DF0
:20858000032803D1487E40F004004876F0200EF080FEE168606888470FE0887E401E887667
:2085A00012490127F0200F700EF073FE10480078A7E70026467007F05BFC6068C08A000A96
:2085C0000AD394F8400318B994F86F040BF0AEFF94F96E040FF08AF80020606010200FF0E8
:2085E000BBF9BDE8FC81C0463D1F0020B53500204A1D0020100100202DE9F04F80460D46F3
:208600005E4898F808108778ADF1140D0229CDF80C8014D1012F12D000F22C410C46022206
:20862000404620310EF0C8F938B903208DF8080004F1160168464FF081FBCDF80CD02FB30B
:20864000DFF848B198F808904D4CDBF8040014F809A080470A266427F8340490207A484594
:2086600005D15246204641460EF0A6F920B1761E04F10C04F2D103E00027EF72A07A2873B5
:20868000DBF8081004988847002F73D03C49DDF80CA04FF0000864278B468E6DB1F84E0077
:2086A00085F81E804446D9460AE0BAF80010761C2134B6B233E0B9F84E00641CB61DA4B240
:2086C000A04218DDF0780028F5D0B0880BF002FB514608220EF070F90028ECD1F078A877AA
:2086E000308800046860B08885F80B80A5F81F00B07847462873DBF85440002F3AD085F88D
:208700001E8042F219000DF10A010BF049FC0EF05BFA81461B480188642746468246B1424D
:2087200028DDA07F0028C0D0B4F81F000BF0D2FA039908220EF040F90028B6D1E07A02289B
:2087400003D0E07A80B161270FE0BDF80A000E4A6168424348460FF05FF828B9A07F6C2768
:2087600040F00800A07700E047462846214621224FF06CF8384605B0BDE8F08F10010020FA
:20878000C00E00200C0F0020808D5B00D81800202DE9F04141780025ADF1280D891F6CD05C
:2087A0000A392DD0891E00F09F80DC3940F09A8081688088012814BFFF2008788DF80C0047
:2087C00098B1401E09D0401E05D003A8FF21092208F0FEFF10E04D4900E04D490A680DF18F
:2087E0000D0002604968416006E04A490DF10D031820E2224DF0F8FCEE20092103AA7EE081
:2088000086888768052E34D3434C38782070606878BB387868B30820424AADF8000004230C
:2088200001961168ADF802306846884700BB02986060F0B1781C4FF0FFF95FEA000806D12B
:20884000781C4FF47A714FF0DAF94FF47A78668060683946324607F08BF9A068642101FB66
:2088600008F10FF017FB04F10C004FF035FA00E06560102031463A4641E08188052925D165
:2088800080680378401C4FF0D7F901468DF818501846401E09D0401E16D1204B08461968C2
:2088A00002080BD2C0F3100006E01D4B08461968020803D200F00100014303E06FF0004259
:2088C00042401140196005E0252001E0272029468DF818000DF119004FF091F906200521C2
:2088E00006AA0CE026250CE00EF07EFE8DF820000EF07AFE022108AA8DF8210012200FF064
:2089000003F928460AB0BDE8F081C046C87F0500F0120050654701005C1C0020141F0020E1
:20892000801E0020D81800202DE9F04F81460E469046ADF13C0D5D4C8DF810909B468DF808
:208940001160B8F1FA0FADF814802168CDF818B074DD584C04F114000078042802D007200A
:208960000AF048FF4646F620B6FBF0F0401CC0B202460746B1180C92491E800091FBF2F163
:20898000C9B20B910DF094FC00210D9000280E9134D089466FB30A908A460B988642D4BF51
:2089A000F5B2051CB9F1000F18BF0E9802D1281D0DF07EFC03460A9840F8043B002B0A9003
:2089C00008BF4FF0030910D010201870414683F801A0981C4FF03BF92A461B1D594618467E
:2089E00007F0C6F8761BB6B2AB447F1E0AF1010AD3D14F4627750C98607500E0277D04A9B8
:208A000091E8061004F11C0080E806100E99A1770D9A6262227F102342F080022277E37793
:208A20003FB90B9AA275A4F8188007F0EFF80E9002E005200AF0DEFE0E9834E002204FF0DA
:208A4000080AADF81E005FFA88F8ADF81CA008F10300089007A8884700280CBF099F002733
:208A600013480578002F408824680A9008BF062019D087F8008087F80190F81C59464246E1
:208A8000BE7007F075F8ADF800A0ADF802A08DF80450039700268DF808600A98ADF80600E5
:208AA0006846A047C0B20FB0BDE8F08FD81800201C1D0020D4330020F8B5074661485F4CEE
:208AC000001DC26A0168B7F5C067C2F30722C4F8B870C1F38441C4F8BC20C069C4F8C01089
:208AE000C0F38120C4F8D00000F0A38094F8D8606EB9C4F8D470D4F8C000C4F8C800D4F8BC
:208B0000BC60C4F8C460D4F8D050C4F8CC50D4F8D400D4F8BC50002854BF02236FF001035A
:208B200004F1C802116800EB4000C018431000EB937001EBA0011160D4F8C810C4F8C45047
:208B400000291CDD1E293DDDD4F8CC0030B93429B4BF15391E21C4F8C81025E02A29BABF4F
:208B6000D4F8C8000B381E20C4F8C800D4F8C4003E28D4BF401C3F20C4F8C4001FE0D4F8CD
:208B8000CC00032812D011F10A0FA6BFD4F8C8000B300120C4F8C800D4F8C4000028CCBFC5
:208BA000401E0020C4F8C400032009E011F1140FA6BFD4F8C80015300120C4F8C800002083
:208BC000C4F8CC004FF08057D7F8A401B4F8C4101B4D40684FF47F42082306460091284679
:208BE0003021B047D7F8A40101214FF40032112340680091064604212846B047D7F8A4016B
:208C0000B4F8C81040684FF4F80212230646009104212846B047D7F8A401B4F8CC104068AB
:208C20004FF440620A230446009120212846A047F8BD002084F8D800F8BDC0460416002093
:208C400000A00C4000A00C402DE9FE4F9A469146884604460FF038F8DFF86CB10CAFABF190
:208C6000350529680290A14208BF69680DF1050042464B460090204600F0DAFA061C11D142
:208C800095F8340040F0040085F834000298AC620FF01CF99DF80500022873D16FF0020009
:208CA000BDE8FE8F04F178000FF006F8C6F80880464899F80430F460B18D86F82E301430CD
:208CC00001803E48C6F804A097E80C00202100271940B846104086F82F7006F1100383E8FF
:208CE000030006F1180282E8800199F80500012805D196F82F0040F0100086F82F0002989C
:208D00000FF0E4F895F83500042806D1E86AB5F9301095F832200EF06AFF0EF0D5FF804695
:208D200095F8350002280BD196F82F0040F0800086F82F0084F8C27040460FF0C7F839E046
:208D40001F4D012812D11F480EF0B6FF96F82F0040F0800086F82F00686884F8C2700028C1
:208D6000EAD140460FF0B2F85846007830F004001ED12846314601AA0BF0AAF930B9404643
:208D80000FF0A4F86FF00100BDE8FE8FB08DA4F8C0009DF8045096F82F0040F0800086F839
:208DA0002F00012D84F8C270C6D140460FF08EF80EF0CCFBB6F92C00BDE8FE8FFDEFFF9FAA
:208DC000343500202434002035330020343500202DE9FE4F07461046002F00910CBFE821E7
:208DE000002101910099002900F0AC800199002940F0AA8060B17868401E7860F821017014
:208E00007868401E7860002606703889801C3881DFF83C81009C4FF000094FF0020BCDF801
:208E20000890C246083C14F8080F00F00F010F2900F08580012821D004287AD19AF8400398
:208E4000002876D0DAF8581360688847061C26D03889B7F84C108019801C81421FDB78681A
:208E6000DAF85CC36168029B3A46801BE047B0B178683989801B8919786059E0009A0298D4
:208E800004254A44D21C12F8011FFF2941D021293DD13989B7F84C300B318B4202DA1A2066
:208EA000BDE8FE8F7968B8F86834491E79601B120B707968491E796098F868340B707968C2
:208EC000491E7960029E0E7098F86A147B68197098F8663479681B01491E796043F00F030E
:208EE0000B7098F858C498F839347968491E796043EA0C130B707968491E796021260E7080
:208F00007968C01D80B2491E796005260E706D1EB9D17968C0F30122491E796042F08802B0
:208F20000A707968491E7960087039890918891C3981BBF1010B09F108097FF474AF7868A3
:208F4000B86501E0E82001900198BDE8FE8FC046100100202DE9F0470446880FC0F0A38077
:208F600000200AF057FF51480EF062FD504A002140F60A00108002F10C0551802B7802F195
:208F80000D0661F303032B704A4B516035784FF0010A6AF3030535701F78A6688C460D46B8
:208FA000718007B95546637C1D4318BFD446338891466546A3F602076FB141F21E02BF1A0A
:208FC00009D006F119031A7861F382021A707DB106F1180208E006F111031A7861F3820215
:208FE0001A702DB106F11002138861F309131380C21F6174354602F1010800E03D466F68FB
:2090000037B13B88984203D09A4218BF9845F5D1C5F8049005F10D03187861F303001870DC
:2090200025480EF063FE8068008882421CD04246824219D0278DCFB104F12800E16204F186
:20904000340341801A78353461F303021A7022786AF30302227009F10D07C9F80400387829
:2090600061F30300387001E0144801601448007880B9144800680068014650468847012845
:209080000ED00D3528786AF3030028700E480EF0CFFC05E00BF0BAFD0028FBD00BF0D6FDA1
:2090A00030460EF069FCBDE8F087C0468529000074350020B13500203435002070340020EB
:2090C00081340020E00100109D3801002DE9F041074651480C46018838467138022840F269
:2090E0009880133828D0514A4C387CD0401E65D0401E4FD0DFF82C81401E3BD0DFF828C1ED
:20910000401E2BD0401E1AD038460EF0BBFB0646FF2E11D0414D68688047414A0746B00075
:20912000115C801842784346C91820464EF08EFBA968384688470EE0F420BDE8F0812178CA
:20914000022966DA6046641C0422001D00EB810120464EF07BFB0020BDE8F0812088814213
:2091600057DDC100674601EB001138681822241D0918EDE72678022E4BDA2C25601C05FB80
:209180000681102239314EF061FB05FB0680C06C6061E0E72378022B3BDA607802F5966135
:2091A0002C2505FB032292F8E824824231DD00EB430001EB40010222983128E02378022BB9
:2091C00027DA618802F596602C2505FB032292F8E0248A421DDD00EB8300D0F8900001EB3C
:2091E00041010322C3E72178022912DA607802F596632C2505FB012292F8D824824208DD43
:20920000401841000A2201EBC001C9187C31A41C9EE7E820BDE8F081681E0020D818002035
:209220007C9E0100C005002060060020100100202DE9FE4F554E04468A469046002006F16A
:20924000350108700C9A0192834682F800B00DF0EDFA0093071C08BF012000F08A804C4D1F
:20926000B16AB5F914008C4200F101006FF31F30B88507D196F83400410824BF00F0FE00AF
:2092800086F834001846006800B95846B86298F80C0000F00F00022814BF5846D8F80800D7
:2092A000BAF1000F78626DD00AF19C000EF0FCFA00285DD1204629460CF002FE041C0DD12D
:2092C0002B685BB169682A68384605F04BFF28B1012386F83530286838602F6096F83590E5
:2092E000B9F1000F4ED10CB92C6894B122683846214605F037FF18B92468002CF6D108E026
:209300000221206886F835103346386093F835902760B9F1000F35D100980179504603F09D
:20932000B5FE014601292AD096F83500002829D1012927D0296809B10868F0B998F80C0009
:2093400000F00F0002281DD198F80C00C011400818D241B96868A8B1696838465A4605F050
:2093600001FF28B10EE038465A4605F0FBFE48B9022001995F46087004E00968DCE7042004
:2093800086F835003846BDE8FE8FC04600330020343500202DE9F843554C67684FF0FF3059
:2093A0000EF05EF9002F00F09980DFF83C81010925D2810801D3E6680EB307F1100191E89D
:2093C0006000002105EA00020E4008BF002A00F085803A6A284007F11806104396E80C00E8
:2093E00007F118053862386AA7601943104385E8030040464FF480410EF084FC6EE03969FE
:209400003E6A07F1180595E80C0041F00A0108403043364D3862386A00211943002610435A
:209420003A69666007F1180383E80300286807F110039043286093E80300083D2868324681
:20944000091C88433946286004F1100081460AF03FFE404602210EF055FCE06800283DD09D
:20946000E068F968C068884238D1E06890F82F1097F82F00084310F0070015D0410806D223
:20948000810804D2E16891F82F20104304E0E16891F82F0040F0010081F82F00E16832467A
:2094A00048460AF015FE18E0E0686060E0680069C0436860E0680069A9680843A860E06838
:2094C000103003C8081CC04345F8040CE068103003C82F68081C38432860E6600AF0B6FE08
:2094E00005F092FCBDE8F8836C33002014100440343500202DE9FF4104466668A7680D4649
:209500000EF0E2FB3178012903D10EF0DFFC00208DE0012131700EF0D9FC2878707068786D
:20952000B07068687060A868B060E868F06028693061287D3075687D7075A87DB075A8691A
:20954000B061287F3077687F4FF000087077A87FC6F82080C6F83080B07745467562756343
:20956000B562B56386F82C5086F82D50786804F06DFE204605F082FA204604F02BFF78B9FC
:209580002C480068C068014638688847786804F0CDFC0EF099FB35700EF098FC2C4645E014
:2095A00068460EF089F93A7B06F17C00B9680192214A00946B460BF049FC68460EF09CF970
:2095C000396902911D49009406F198006A460BF04DFDB07830B906F1CC0029460CF00EFD8E
:2095E00017483061707830B906F1E80029460CF005FD1448F06068460EF00DFB01958DF8E3
:20960000005006F58270104902940A226B460AF0B5FEB969FA6906F13C000EF021F90B4A6F
:2096200006F16800042123460CF0F6FE20460090BDE8FF81D001001049A30000A95001006B
:209640000F7C0100077C0100850B0100B97901002DE9F04F06464FF00108ADF1640D092213
:20966000B07D8DF84C8006F117018DF84D000DF14E004EF0EBF84B4D68688047179016A989
:209680008120FFF723FD707D002840D09DF85800022817DA042000238DF80300347D8DF8E1
:2096A00002809DF858708DF8013069468DF80040781C8DF85800D220FDF712FD812016A9DB
:2096C000FDF70EFDDFF8E0A000274FF0FF0B3C46B94618E0307D69460DEB8000C0F810901F
:2096E000D420FDF7FDFC01E08DF824B08DF82670307D8DF8257008A98DF82000D120FDF732
:20970000EFFC641CE4B2BAF80000A0422ADC307D00279DF84D208DF840000DF14E018DF841
:2097200041700DF142004EF091F88DF84B80D02010A9FDF7D5FC071C0FD1307D314610225A
:209740008DF828000DF129004EF080F830690AA90F90D320FDF7C4FC0746A9681798884711
:20976000F8B21CE0307DADF8224008A980F001008DF82000D120FFF7A9FC0028B4D19DF8FA
:209780002400FF28B0D0ADF800006946D420FFF79DFC00289ED0A96817988847192019B000
:2097A000BDE8F08FD8180020681E00202DE9F843504C80466068002800F09980DFF8389183
:2097C000B8F1000F18BFB8F1E90F17D14D46AE892F690DF0E9F906EB8606F619C6F80100E5
:2097E000A88995F8F521014601EB81017A54E989401C80B28142D8BF0020A8813F4D686813
:20980000B8F11C0F37D0B8F1000F0BD099F82300032807D1B8F1E10F04D0002089F8F20122
:20982000072000E0052009F091FF676899F8230003280FD077B10020FE8A87F86900F00935
:2098400034BF94F8510494F87A0487F86A004046FEF704FE99F89701012848D168688047C2
:20986000044608F041FDA96820468847002089F89701BDE8F8838047064661682048C98A32
:209880000078C90804D294F88B10814204DB28E094F88A10814224DA616804F180004DF076
:2098A000A9FF6068C08AC00805D294F88B00401C84F88B0004E094F88A00401C84F88A0079
:2098C000A968304688476068007D252819BF012089F89601012089F8950100206060BDE8D2
:2098E000F883A96830468847F120FEF7B7FDBDE8F883C04610010020C00E0020D818002088
:20990000641E00202DE9FE4FDFF82091484C494FDFF824A1DFF8248199F8400399F8AF144E
:2099200088B9606880473F7847B95246A16817782FB9832342461370884760E0A16802239A
:209940004246137067E001290BD199F87F040CF027FAC07B022804D13E48C01C007806F074
:20996000B9F80CF0A5F8364D286A364E016CF06888478346606880473F780290002F41D18E
:209980005046007800283DD1D9F88C1300208847F42001A90AF0E6FE2B4F9DF904005845D7
:2099A00014DCBB7993B9A1680298884704214046BE790170D9F88C13701CB87109B1032070
:2099C00088470320788100F0EFF825E0832140462A6A0170536CF0686A4600219847B5F91C
:2099E0000600BDF90010884214BF002001200AF027F8A16802988847387A1449087007F0B4
:209A000067FE09E0022140460170A16802988847D9F88C13042088470D480078012802D041
:209A20000020F9F77BFCBDE8FE8FC04610010020D8180020B9350020BB350020BD350020F6
:209A4000201800202C1C0020481D00207B1E00203D1F00204A1D00202DE9F04FFF25ADF1EE
:209A6000140D8DF800504FF6FF79ADF80290ADF804900BF049FDDFF82CB104900BF102003C
:209A800000880027001F84B2082C64DBC8464646C246201F02A9082280B24DF0BFFFBDF8B7
:209AA0000800814508D1BDF80A10894506D1BDF80C20924502D107E0BDF80A1051EA00030C
:209AC00014D1BDF80C308BB9BDF80E00C10BCB030AD100F108018C4238DA4DF0D1FF0498B1
:209AE0000DF0D0FA002058E0241F31E0C20BD3032AD1C20B28D3BDF80C3000F0FF029542D4
:209B000003D1884508BF9E421ED0C5B28DF800508846ADF802801E46ADF804609DE80600D6
:209B2000384608F0D3FA78B9BDF80E20A01A07F18851001F083280B292B24DF06FFFBDF814
:209B40000E00C019083087B2BDF80E00241A083CA4B2082C9DDA0AF08DFE3FB110484FF05B
:209B600088513A464DF07AFF0DF038FE04980DF089FA59464E78002E1CBF0020021C0BD1FF
:209B800004204FF40052C0EA0740C2EA0742A2FA40F01FFAA0F280B24A8005B0BDE8F08FDA
:209BA00004400500901E0020F8B5504C4C4E4D4A203C7089717894F8AF34012B6AD102F10D
:209BC00074031978002565F30301197002F1CC031567197802F1780765F3030119703B789A
:209BE000012161F3C3033B7002F178073B7861F304133B704FF4FA57C2F8807008B9718152
:209C000008463B493B4F491C94F840330978083148433978002B01FB00F0009036D0D4F815
:209C20008023002A32D0D4F8840300282ED006F10801684690477179737862682A4E6528B3
:209C40001AD0A8B9107D052820D194F85504E8B9606890F82C00211D042817D10968D4F87D
:209C60005C43906D096B2B46A04778B91A2000E03570FEF7F3FBF8BD82F8691082F86A30ED
:209C8000D4F8841335701C208847F8BD00980CF0C7FCF8BD002394F85D04A2F8AE3094F8DC
:209CA000507482F8B00002F1B20682F8B170307802F1B20563F345103070287802F1B20787
:209CC00020F01F0040F001002870387863F38710387082F8B41082F8B33082F8B530F8BD98
:209CE000481D00207C130020BD35002030010020781E0020701D00202DE9F04705466C78EE
:209D0000ADF1180D002C40F08B804A48B5F89A100088884218BFE82405F1900101A88846FD
:209D20000DF0AAFA444E01A80CF0DAFB30B995F89D0030B1707820B9E82471E0002085F8C7
:209D40009D00002C6CD195F89D0000280CBF0120052004272F754146E8820DF10E000DF0D1
:209D60008BFA686895F89C40401E6860411E6960B5F89A9004702B7D69680024481C286201
:209D8000581E087028892C6596F84023AC65801C002A288136D085F86B7005F170004146D7
:209DA0000A224DF053FD95F8980005F1700A032828D105F1900150464DF0C0FF96F8550431
:209DC00000B31E4E306810F47F0F0CD085F82C70306805F12C01012200F47F0028632846FB
:209DE000FEF7F6FF306810F0FF0F0BD02A2085F83C00306805F13C0100F0FF002864284641
:209E000003F030FE0094284603210DF10E024B46F8F72EFA041C02D1284603F07BFA2CB19F
:209E20006C701A202870284608F056FE06B0BDE8F087C0466205002010010020E89E0100A3
:209E40002DE9F04705464B4890F8009028798028D4BF0020E820494C0027B9F1010F0DD167
:209E60006979092901DB0A2900DDE820A97909B1042903DB80297ADB882978DA002876D183
:209E800094F839040F2872D0B4F852144FF6FF7088426CD0B4F84C14884268D0E87901281C
:209EA0000BD040B1FF2862D194F8670100285ED10126374602E0012600E0022604F508700B
:209EC000824607F0CBFA04F5047007F0C7FA04F5A67007F0C3FADFF8A88008F104000068B2
:209EE000804784F8676166680246FF210020C4F86001002E84F864110CBF0121011C84F83F
:209F00006911012F84F8687108BF032084F840024046816810468847A91DE820FAF7DAFB72
:209F2000691DE720FAF7D6FB291DE120FAF7D2FB94F86901012802D120200DF0FDFC0E484F
:209F4000B9F1010FC4F8280207D094F839144FF47070884000F2564106E094F839144FF43B
:209F60007070884000F2636150460DF025F9BDE8F087C046BF050020112201001001002067
:209F8000D8180020F8B54B4C4D4D002859D194F8391460680F2957D067680F20398984F845
:209FA0006501012007F048FF94F82F0478B194F8550460B14048D4F85C2194F83014C4F8A1
:209FC000D80204F53470891820310CF0E3FC94F85804D4F860110F2807D03848C4F8540179
:209FE00004F5A6700CF0D6FC01E00CF0DDFA606840680078000958D3686880470646D4F805
:20A000008000074670B10022387E800905D23A4657F80C7C002FF7D104E004F180003946F4
:20A020004DF00AFBA96830468847002F3DD0787E394640F01000787604F180004DF0DAFB22
:20A0400033E0606894F839140F292ED104F53A71076D0A784FB1082094F87F7484F8EA026C
:20A06000974202D0E820FAF735FB94F8550410B102200DF061FC1348001D00688047D4F877
:20A0800080706FB1397E01F0FD013976890903D3797E41F01001797657F80C7C002FF1D103
:20A0A000A968884708200DF057FC201D0BF00AF9F8BDC04610010020897C0100DD3301000A
:20A0C000D8180020D81800202DE9F043054605200327E88268682F75401E6860411E696051
:20A0E00095F89A10017095F89A00ADF1140D18B14FF6FF70A5F89800B5F898606868411E4C
:20A100006960311201706868411E696095F8984004702B7D6968481C2862581E08702889EB
:20A1200005F18F01001D288101A84DF007FE05F18F0600248DF80C70DFF8C4802C6598F8FC
:20A140004003AC65002839D04FF0040985F86940E88A85F86B90C00934BF98F8510498F8ED
:20A160007A0485F87870314685F86A0005F170004DF0E4FD98F8550400B3224E306810F472
:20A180007F0F0CD085F82C90306805F12C01012200F47F0028632846FEF71AFE306810F02D
:20A1A000FF0F0BD02A2085F83C00306805F13C0100F0FF002864284603F054FC0094B8F878
:20A1C00052342846394601AAF8F752F8071C02D1284603F09FF83946DC290BD0DD2909D0FC
:20A1E000E42907D0F32905D0DE2903D0DF2918BFDB2902D1284606F04BF805B0BDE8F08386
:20A2000010010020E49E01002DE9F8434B4D4C4C686894F8AF8480478146A96860680028EB
:20A2200040F08780E0698047D4F8807040F01000002F7DD00022797E0140884205D03A46E6
:20A2400057F80C7C002FF6D172E004F1800039464DF0F2F9B8F1020F02D1384604F0F6FAD4
:20A26000002F65D06760787E30F07F0005D194F88B00401E84F88B0004E094F88A00401E74
:20A2800084F88A00A9684846884761680889C98A06F0ECFBB8F1010FA4F8880004D194F882
:20A2A0007F040BF07DFD01E00DF0FEFB05466068C18A090A08D3C07E0AF038F9606890F9C9
:20A2C0001C000DF013FA6068B8F1020F04D1C18AB4F88870490A10D2E97B012906D002294E
:20A2E00029D10520FBF7CCFDBDE8F883007E401080F0010000F00100F4E797B190F86C60BD
:20A300007EB196FBF7F10F4F068980F86D10791C0A78122ED4BF0C21282191FBF2F1C9B269
:20A3200002E0012180F86D1080F86E100620D9E7A96848468847BDE8F883C046D8180020A4
:20A3400010010020781E00202DE9F0478046D8F808603068076CD8F8045047646A6CA96B07
:20A36000286C17F4F06FA0EB020935D1F8091ED278096AD3B1B196F821003E4A145C601E0D
:20A38000814294BF0C1C641E404621460BF064F9A86B001BA863A86B002856D105F198008F
:20A3A0000DF0B2FC404649460BF09CFB4DE00029F8D040460BF050F9014695F82D00A96356
:20A3C00018B9A86B002840D101E00020A86305F198000DF099FC38E0F80A1AD24FF00009E6
:20A3E0004C4603E0A86B401EA863A96B49B3404601210BF031F93068446814F00F04C0F87C
:20A400000490EFD0296B686B491E2963401E686317E0306844680022202904F00F04426017
:20A42000CCBF4FF0200A8A46404651460BF014F9CAF120008145C8BF8146494640460BF034
:20A4400051FBEC77404608F053F8B80910D3AF6A77B1404639460BF037F9A862AD6A3DB958
:20A4600096F820000449095C4046C91909F03AFFBDE8F08758AC010064AC0100F0B5494D75
:20A48000014695F80F020027ADF1140D002855D195F82E04002851D0087ACF68C0F3021617
:20A4A00000F0070100E0BF1C0846411EC9B248B17A783878B5F8564400EB0220A042F2D12D
:20A4C00002270FE005F22C44443400E008373046411ECEB2A0B3204639464DF017FC002861
:20A4E000F4D0032795F80F0240F0040085F80F0202A80CF009F801200CF046FC05F501719C
:20A500008720FEF7E3FD05F503718520FEF7DEFD05F20D218620FEF7D9FD05F20E21882078
:20A52000FEF7D4FD0120009005F501760196B5F85234394602AA0520FBF7C2FE002F2FD138
:20A5400095F839040F282BD095F85814814227D095F8550420BB95F85E0008BB124800780B
:20A56000012802D00120F8F7D9FE104C6068804795F86711022911D195F86411FF290DD0F5
:20A58000696859B9D5F8801041B9A168884705F5A67006F063FF08F08FFD01E0A168884704
:20A5A00005B0F0BD100100203D1F0020D81800202DE9FF47494C94F8E700002879D1012580
:20A5C0003E4E84F8E750307B84F8E6007768C4F8107101A80DF01FFB002704F10C00029792
:20A5E00001AB8DF80470364903973A4609F0C6FE344904F1300001AB3A4609F0BFFE324961
:20A6000004F1540801AB3A46404609F0B7FEB0680146284688472D48DFF8B4900078767BF4
:20A62000D9F80400C0F3815A26B1BAF1030F04D184F8E150BAF1030F20D0BAF1020F1DD04B
:20A64000BAF1010F2ED14FF08058D8F8A401214C406803214FF040521C230646009139460F
:20A660002046B047D8F8A401406839464FF400720923064600952046B04713E002200BF0B2
:20A680005FFBBAF1030F0CBF4FF47A7142F2107111480068B1FBF0F140460DF009FB40469A
:20A6A0000DF008FBD9F80000C00802D238460BF047FB00200090BDE8FF87C046C8AB01001D
:20A6C0002BDF0000350E01008D060100B6350020B04F005000A00C40A03500200416002023
:20A6E000F0B5477EADF1140D37F07F0700F08A80017D012918BF032940F08480424909888F
:20A7000001F0020201F0080111437BD041684878C0F38102022A8DF8082006D0032A10D14F
:20A72000491D68464DF00AFB09E08A79487940EA0220ADF80000C8780A7940EA02209DF881
:20A7400008200446022A18BF032A19D16846214606F040FDFF284ED19DF8080002460CF0FE
:20A76000D9FF0026012505FA06F1084202D0761C052EF8DB052E09D1022A18BF032A05D1F8
:20A780000CF050FFFF283DD1012039E01F48022A06D004466946082204EBC600903012E00C
:20A7A000BDF800108DF80C40271204468DF80A1004228DF80D7004EB8600091274308DF800
:20A7C0000B100DF10A014DF041F89DF808102046022914BFD0F88C30036F05FA06F20229B6
:20A7E00043EA020314BFC0F88C3003670A46304629460AF0CBFA0CF015FFFE2802D1002059
:20A800000CF002FA05B0F0BD6C0100202018002030B5ADF1140DFFF7CBFE3049314A086832
:20A8200040F0020008602E48026068460DF064F82D4DA8782E4902902C486A460AF016FCCC
:20A8400068460DF039F828782B4A002419216B46019028488DF808400AF0F8FA68460DF093
:20A860004BF8E8780290264924486A460AF0FEFB68460DF021F801206B788DF808001A2195
:20A88000214A204801936B460AF0E0FA1F4820492246134609F072FD1E481F4A0421234676
:20A8A0000BF0BAFD234804701C4A1470072554701B4B94701B491D701D480C700525056062
:20A8C0001A4A1460184D1C492C704FF4FA728A601A48CA600DF0ACF805B030BD0020094069
:20A8E000CC210840110000E070AC01006C330020E96D0100C4340020F5260100A0330020D8
:20A9000009E90000E03400204910010024340020516801004C350020753D0100B03500202C
:20A92000F83200208134002082340020703400207C34002068340020003300201DBA0000A8
:20A940002DE9FF4707463878012866D0002840F08B8097F8281097F8304097F838004E0001
:20A96000E500804673197119414426311FFA81FA1918263188B20BF0AFFC5FEA000973D0A9
:20A98000002100F8011B797800F8011BB9694DF036F9391D0AF0BCFFF9894DF058F9398A11
:20A9A0004DF055F90446B87C04F8010BF87C04F8010B387D04F8010B787D04F8010B387F99
:20A9C00007F11D0104F8010B20460CF0CBFB97F828000B3404F8010B97F8300004F8010B6C
:20A9E00097F8380004F8010BF96A3246204605F0BFF8796BA4192A46204605F0B9F8F96B1A
:20AA00004246601905F0B4F8832051464A4605F085FE48460CF058F826E07E7801208DF8D6
:20AA2000016097F82C108DF8000097F828508DF8061097F829408DF8025097F82A308DF886
:20AA4000034097F82B208DF8043097F82D608DF8052002A8F98D8DF807604DF0F8F86A4661
:20AA600083200A2105F05AFE0090BDE8FF8770472DE9F8430446080B7CD3474804273E490B
:20AA8000077001250D7038460BF05AF93B4E3068016AC90804D3C16900220B4639469847A1
:20AAA0003748384900220DF015F937480CF0C0FF30684168886808B9C86810B133480CF0D5
:20AAC0005BFF284609F0A6F9D4F808900021A9F80210A0680288A2F602072FB141F21E0278
:20AAE000BF1A18BF183000D11030038840F60A06F21F61F3091302F1010803804B46657412
:20AB000000E03B465F6837B13888864203D0824218BF8045F5D103F10D065960307865F3E4
:20AB2000030030701A480DF0E1F88068008882421BD04246824218D0208DC0B104F12800AC
:20AB4000E16204F1340641803278353461F303023270227865F30302227003F10D0758606B
:20AB6000387861F30300387001E00A48016048460CF002FFBDE8F883823400206C34002051
:20AB8000C4340020A96C010085290000510007063435002074340020B03500202DE9F84FC8
:20ABA0004549474C6FF00100A66B0870301C03D194F839140F297DD14249404F01220028A7
:20ABC0008A460A7069D00AF00FFD7168884262D394F83904A56B0F284ED0002D5DD004F197
:20ABE000280B4FF0000895F80C90AE680AF0FCFC696888420DD2A06B30B1216B406881424D
:20AC000002DD0AF00DFD48E00BF0B2FE4046A06343E04846B04778688047814659462846D2
:20AC20000CF04EF920B904F12C0128460CF048F9A06BA84219D1A06A4646C4F8388086427A
:20AC40000BD0216B4068814207DD0AF0CDFCA66A71688842C8BF7060A663E56A2DB11EB16C
:20AC600070686968884200DDA563B96848468847A56B002DB7D110E07DB10AF0B5FC69689F
:20AC800088420AD3A06B054606F0E8FBA968287B8847A56BF0E708F0D5FC786880470446BA
:20ACA00002F0DEFCB968204688470CF077FA00208AF80000BDE8F88F2D1E0020D8180020BC
:20ACC000100100203D1F00202DE9F04F474C80466068ADF12C0D80470A9000258DF80080EF
:20ACE00069468DF80150D020FEF7F0F9A346D0B99DF80B00012802D19DF80A1019B990B929
:20AD00009DF8061079B1002814BF08270427FF210DF102007F1E00F8011BFBD10570694648
:20AD2000D020FCF7DDF9304EDFF8C4A0B0884FF6FF792F4631E03C4601E0641CA4B2B088B5
:20AD4000A04213DD9DF82000ADF8224008A980F001008DF82000D120FEF7B8F90028ECD122
:20AD6000BDF800009DF824108842E6D1B088A0420FD1ADF80490ADF8069002A8FF21082272
:20AD80004CF080FD0DEB880069460761D420FCF7A7F9504600886D1CEDB2A84205DCDBF8F8
:20ADA00008100A98884738461AE08DF82080ADF8225008A9D120FEF789F90028E9D19DF8C6
:20ADC0002400FF28E5D0ADF800006946D420FEF77DF90028AFD0DBF808100A988847192084
:20ADE0000BB0BDE8F08FC046641E0020D8180020681E00202DE9FE4F0BF0E6FE434C04F150
:20AE0000280202901168E0624FF40050491C1160694609F0C5F8DFF8FCA0DFF8FC90B4F86B
:20AE2000520000285FD0A66DB4F84E0000254FF6FF7BA0462F4654E0B07F800822D3B6F88F
:20AE40001F0008F047FF0146082268460BF0B4FDC0B1716802982E4A0CF0DEFC90B9B6F8A1
:20AE60001F00B77709F012FEA6F81FB0DAF800008047B4F8503013B15B1EA4F85030D9F820
:20AE800008108847B8F84C006D1C2136ADB235E0F078800821D3B08808F01CFF01460822DB
:20AEA00068460BF089FDC0B130880104184A02980CF0B2FC88B9B088F77009F0E7FDA6F834
:20AEC00004B0DAF800008047B4F8523013B15B1EA4F85230D9F808108847B8F84E006D1C5D
:20AEE000ADB2A842D4DCB4F8500048B1A046666DB8F84C0000254FF6FF7B2F46A8429BDCF5
:20AF000004F1300008F096FEBDE8FE8FC00E002000A493D6DC180020D81800202DE9F041E8
:20AF20003A4A39483A4916780778ADF1180D002E60D04048067836F07F065BD1C88A354DAA
:20AF4000012F00F10100C88209D000248DF80C4002948DF80D4005F144002C6404E000247D
:20AF600005F1CC00C5F8C84001782B4E2B4B64F303010170012030701978012901D0F8F7DA
:20AF8000CDF9012F01D10BF0EFFE2B48001D006880478046294B2A48DFF884C0066818688D
:20AFA000012F05D005F13801082302AA4C8008E0049402238DF8154005F1C0018DF81430BB
:20AFC00004AA8DE81800346D6346A04715490880154900280AD4154A92F90000401C1070F5
:20AFE0001348012F14BF3835C035C56089684046884706E0088B401C0883002010700CF02A
:20B0000095F806B0BDE8F081BF050020BB350020481D00207C1300202F1E00203D1F0020C6
:20B02000F90A0100C81B0020D8180020361E002020180020BD350020D8180020381C002097
:20B0400040180020B0B5044645480078002800F0828094F88F00002871D13520207504F146
:20B060009101112204F170004CF0F0FB04F13C00FF2110224CF006FC04F12C000F2110223B
:20B080004CF000FC94F8900004F13C0500283ED0401E29D0401E14D0401E5AD12A202870EC
:20B0A00002272764042305F8103C4FF410222263032184F86B10204607F0ACFC071C3BD123
:20B0C00037E02A200A272870042327644FF44C1205F8103C02212263204684F86B1007F0AE
:20B0E00099FC071C28D124E02A2002272870042327644FF4102205F8103C01212263204613
:20B1000084F86B1007F086FC071C15D111E02A2002272870042327644FF4502205F8103C0A
:20B1200000212263204684F86B1007F073FC071C02D1204602F0EEF8381C0DD1B0BD0128AA
:20B140000CD10848D0F850038047002808BF002002D0192000E018200CF0F0FAB0BDC04655
:20B1600050040020100100202DE9FC4706467568D6F80880A86B002818BF4FF0FF307ED183
:20B1800029630024EC77171C6C631BD005F13C090CF09AFD82466946484609F077FD002847
:20B1A00020D450460CF092FE9DF80000296B0870686B296B7F1E00F10100686301F1010123
:20B1C0002963E5D169786A6B286B0129A0EB0200286305D1E868296B0346304698476A6B75
:20B1E00014464BE0AF6350460CF070FE0CF06CFD244E0746307820B902200AF0A1FD012038
:20B20000307038460CF062FED8F80010086B40F400700863D8F80010886B40F4FA60886306
:20B22000687808BB696805F1E80738460CF021FBB8B1AC63384621460CF01BFB88B10CF07B
:20B2400043FD0746307818B102200AF013FB347038460CF03BFE1022696B286BEA77401A1B
:20B260002863686BBDE8FC8795F82D0030B1686B20B1AC6305F198000CF046FD2046BDE822
:20B28000FC87C046B33500202DE9F84F05464248DFF80C81814646192D3698F8400334787F
:20B2A0000F46C0B1D8F85813A9B109EB850ADAF8DC0000F0FF0088478346D8F85813DAF86E
:20B2C000DC0000F47F008847584480B218B131780818001DC4B298F8640401280AD1387AAF
:20B2E00040B148447B7A067919F803002418641DE4B200E000260D2D06D104EB060ABAF135
:20B30000F80F07DC254F18E0A0198246801C4CF02FFA07468FB902204CF02AFA011C09D048
:20B320004D4495F8490008701A274F7098F800004CF014F90020BDE8F88F0AF1020238468C
:20B3400000214CF09FFA07F10C00002178224CF099FA07F13C00FF2110224CF093FA07F122
:20B360002C000F2110224CF08DFA38197860022D3E810BDB0B2D09DA7868401E78606D1EC3
:20B3800005703889641E401C3881E4B2A7F84C403846BDE8F88FC046FC9D0100202F002066
:20B3A000100100202DE9F041424C04F1100528460CF09CFC071C7AD00AF090FA7B683A6A03
:20B3C00000263E6243B397F82F0000F00700401E0BD0401E06D0801E18BF002308D14FF0DF
:20B3E000805304E04FF0804301E04FF00053324697F82F00000908D397F82F0010F0070F33
:20B4000003D04FF08070324303437968B7F92CE0F8688C467146E0470CF056FC8046B4F901
:20B420001600401C6FF31F30E082206980F82F6028460BF06BFF40460CF048FDB4F914009C
:20B44000B4F91610884232D1F86890F8C20000280CBF0520072005F0F1F91748F968056857
:20B460008D4208BF456891F8C240002C0CBF0C68341C81F8C2604DB195F8C23023B92868BF
:20B48000A04228BF041C01E085F8C26064B1B4F1FF3F0CD00949F86809687830B4FBF1F113
:20B4A0000CF077F8BDE8F08108200AF035FBBDE8F081C0463435002000330020A0350020CC
:20B4C000F8B53A4D0646287800286DD03F4CB4F91600B4F91410884214D0304621460AF043
:20B4E000EFFC021C06D1616830460CF00DFA00B162683AB1B2F92C1030464FF0E0430022E3
:20B5000000F0FEFE0CF0E0FB074629480168B14219BF00244460002404602878401EC0B2B6
:20B520002870244D58BB244800782E6002280ED108200AF0F1FA38460CF0C8FC06F14000F2
:20B540004FF0FF310CF095F90CF0BEFB074620480CF0D2FB19480CF0B5FB1E480CF0CCFB89
:20B5600017480CF0AFFB17480CF09CFB16480BF08BFB307C012802D10E2002F0D7FC2846EC
:20B58000016806F140058E4208BF046038460CF09DFC28460CF0ACFB06F178000CF082FBFF
:20B5A00006F19C000CF07EFBF8BDC04680340020003300206C340020B0350020C4340020C4
:20B5C000E0340020243400204C350020343500206C330020A03300202DE9F84303200AF075
:20B5E000AFFB364D0024032005F11C0141F80C4F401E8C60FAD105F14C00264608270146F7
:20B600007F1E21F80C6BFBD14FF008082D4F2C492D4AA0F800803F1D816005F1200996462A
:20B6200027F00301531A6B628C46E9610846296201E040F8046B8242FBD8B80823F00303C8
:20B64000AEEB8000E827801001EB800040F8046CEC3BCCF800702046C1F8E830E8316961A9
:20B660004AF00CFEA861D9F8000019496861174D0A682846026049684160164942460BF0A7
:20B680009BF920B914480168296040686860134813498165046644660467124F4467124DF8
:20B6A000C765124B8566816DC36609B1204688474AF022FEFAF79EF8BDE8F883D8180020FF
:20B6C00045690500BE350020003B0120241E0020C87F050038AC0100F01200506C060020D1
:20B6E000CD4B0100F54F010099540100CDD80000B0B50546AC682078ADF1400D641C8DF80D
:20B700000800214668460BF04FFB083420464CF0A4FAA41CADF80A0014F8010B8DF80C0033
:20B7200014F8010B8DF80D002778082200210DF10E0006F04DF8780824BF01208DF80E0017
:20B74000F80824BF01208DF80F00380924BF01208DF81000780924BF01208DF81100B8099B
:20B7600024BF01208DF81200F80924BF01208DF8130037F07F001CBF01208DF81400641CD6
:20B7800014F8010B8DF8160014F8010B21468DF817000BA80BF0D8FC0B3400208DF81E0057
:20B7A00020464CF049FA271D089038464CF055FABB1C02461846ADF828204CF04EFA9F1C16
:20B7C0000A23ADF81C00BDF82810099712188DF8373090B27C182330FF270694AA888DF838
:20B7E0003870904218BF272105D1054918206A464AF0FAFCC1B205200BF0DCFF10B0B0BDD9
:20B80000114C00002DE9F04F404CADF1340D0A90606880470027FF254FF6FF783E46A3466E
:20B820000B90DFF8EC908DF800608DF80170D0206946FDF74BFC00285DD19DF80B00012846
:20B8400010D19DF80A0068B90DF101020820394612F8013FFF2B03D1401E01F10101F7D13D
:20B86000082948D03C460BE050460BF003FE28B18DF8245008A9D120FBF732FC641CE4B2D6
:20B88000B9F80000A04236DD8DF82060ADF8224008A9D120FDF71AFC0028EFD19DF82400A9
:20B8A000FF28EBD0ADF800006946D420FDF70EFC28B1DBF808100B988847192023E00A994B
:20B8C0000DF1080A082250464BF084FF0028CBD0ADF80480ADF8068002A8294608224BF045
:20B8E000D1FFD4206946FBF7FBFB8DF8245008A9D120FBF7F5FB761C022E94DBDBF8081054
:20B900000B98884738460DB0BDE8F08FD8180020681E00202DE9F0410746394C787894F80B
:20B920003984002865D16078374E20B1301D0068B8F10F0F55D1D4F8C801417A0F2911D1B2
:20B9400003F0B8FAD4F8C80190F83000002850D094F8400300284CD0D4F84803002848D043
:20B96000804746E003F0A6FA0AF0A6FDD4F8E052B8F10F0F23D1D4F8C81122484A7A00EB33
:20B980008202D2F814212263497A00EB8100D0F8140160637068804780461D491B48097821
:20B9A000203D89004D4301686D1A456001F058FEB1684046884709F009FAD4F8E052154870
:20B9C0002946C4F8C80204F530700AF0E3FFD4F8C80190F824000F281CBF012084F8EA0221
:20B9E00007E080470C49C4F8C812B1688847BDE8F0812D203870384607F06EF8BDE8F081CA
:20BA000010010020FC9D0100D818002004300440701D0020B53E0100E159010070B50C4680
:20BA2000A00852D2E0085ED32F480125057004200AF086F92E480068006B80472B49086086
:20BA400036480CF053F92B4C216870B1C068064649B18E4207D0316AC90804D3C16900225B
:20BA60000B460421984731462160486822490078086002200AF064F9112002F0E7FB226876
:20BA80001E49107C0D7008B1487818B90E2002F0DDFB22685168886808B9C86810B11848AF
:20BAA0000BF06AFF174A07201749106000260E60164D4E600A6845EA0200086014480BF0C3
:20BAC000B7FF19200CF002F970BDFFF76BFC11480CF00CF910B907F037FA70BD0E4844F0F4
:20BAE00002010CF00FF970BD82340020703400208C0100106C340020D0210840B0350020DD
:20BB00005100070600000460141004400A000040558F0000443500206C33002034350020EC
:20BB20002DE9F04F844609AF0020002A9A46ADF1440D3C89D7F804803D888DF83C0067D040
:20BB40003548875C0026042AA4EB0704A4B2B8BF01265FEA06090EBF2D1BA04400243048B6
:20BB600007AB0826ED1B2530ADB210F801E9761E03F801EBF9D1080E284E03F8010B080C4B
:20BB800003F8010B080A03F8010B306C03F8011B9DF83C101A704369F06B62469847834610
:20BBA000BBF1FF3F24D00BA9049101208DF801009DF83C308DF8023007AA01928DF80090A6
:20BBC0008DF80370CDF80880CDF80CA0ADF81640316CADF818500223F06B0A6A8DF814304D
:20BBE000694690478346306C8269F06B0FA99047BBF1000F18BFE4200BD14FB108EB04011B
:20BC000038460BAA12F8013B401E01F8013BF9D1002011B0BDE8F08F009E01001001002079
:20BC2000620500202DE9F04F3C48354E90F800A03078ADF12C0D01285FD101200BF05AFAB1
:20BC40003748A0F13408D8F820002E4F436CF868022108AA98479DF82000002846D1DFF89D
:20BC6000B8B00BF10400006880470025022409902548039502A90290F8688DF8104003F0DF
:20BC80006BF82249224B34702846BAF1010F01F11009D8F82060A9F802000AD006958DF8A4
:20BCA0001C4001218DF81D1049468DE830004D460BE006958DF81C408DF81D0001F110057D
:20BCC000024621468DE806002946346DF86806AAA0475F4629460F4AC8F80C1092F900005F
:20BCE000B968401C10700998884706E03078012803D1002030700BF099FB0BB0BDE8F08F1E
:20BD00003E1F00202C1C002000093D007C1300204D4D0100361E0020D8180020BF05002046
:20BD2000541800202DE9FF47394CA11D0888401C08803849082268464BF088FD0AF044FF0E
:20BD40004FF000084FF6FF7746464546824618E09DF80830616D2BB902EB4210401840684C
:20BD6000010403E002EB42104018416850460BF0A7FF804503D29DF80890804616466D1CF2
:20BD8000ADB2208BA84238DC244D281D006880478046B4F85200B9F1000F0DD1A26D7100DB
:20BDA000002301EB8601401E8918CB708A888F8080B2A4F852000EE0606D06EB4616002347
:20BDC0003618B377B6F81F20A6F81F70B4F85000401EA4F85000104867690088121A91B26C
:20BDE000082207EBC10069464BF030FD608BA968401E60834046884706E0284602A904F0CA
:20BE0000B3F902469742A3D10090BDE8FF87C046C00E002054A50100681E0020D818002082
:20BE20002DE9F84390460F460BF04EFF814641463648DFF8DC8002788324381C06D0401E96
:20BE40005AD0401E52D0401E0CD009E04246101D0768002F08BF802451D05068808D4DE044
:20BE600003244CE00D6850220021284605F0B0FC2848022729462B46844610305CF8042B52
:20BE80001A60027A1A7345685D6050F80C2B1E467F1E06F110032A44B260EFD142465768A4
:20BEA000002F08BF02200ED05068C36857680B6297F82E30566881F82C30736A55684B62B6
:20BEC000AB6A03208B621768CFB1052817DAFB6801EB0012136097F82E3013737B6A536041
:20BEE000BB6A93603F68401C40B2EDE70020022A08BF0120087002E00748007808804846F6
:20BF00000BF0E4FF2046BDE8F883C046B03500203435002000330020F83200202DE9F04343
:20BF200004463B48083000680E1C1F461546ADF12C0D16D0ADB131784FF0010808FA01F1AA
:20BF400008420ED0104600210BF0CCFE6660A5600BF0BAFE2A4D2E788146022E03DB0BF012
:20BF6000B5FF002048E016B9FEF752FC2E782948711C40F82640C9B2297048460BF0A6FF2F
:20BF80001FB903AF38460BF075FB386820607868E060387C46462074B96966742162788A99
:20BFA0006082184DA561E5616561F86800B1A061786900B1E061B86800B16061A0220021CE
:20BFC00004F1280005F004FC04F1400000210AF015F868460BF01FFE04F178000A490294D6
:20BFE00000226B4608F0CAF9084904F19C0000226B4608F0C3F920460BB0BDE8F083C0460B
:20C0000080340020FFD70000697001007D7C0100CC210840003300202DE9F04707467D689B
:20C02000D7F8088091460C460BF04EFEAE6A8246002E65D105F582700BF03EFE2C62002420
:20C04000EC7750466C620BF041FF0BF03DFE304E3378824623B9022009F072FE012030708F
:20C0600050460BF033FFD8F80020106B494640F480701063384609F027FBA862C0B93846D2
:20C08000494608F02FF9A878D0B9A96805F1CC000BF0EFFBE8B1AC621020E8774146284665
:20C0A00004F084FB0BF010FE8246307840B323E0D8F80010886B40F020008863A87810B1AF
:20C0C0002046BDE8F087A96805F1CC000BF0D1FB10B9686ABDE8F0873846494608F002F98D
:20C0E0001020AC624146E877284604F05FFB0BF0EBFD8246307818B1022009F0BBFB3470CF
:20C1000050460BF0E3FE4FF0FF30BDE8F087C046B43500202DE9F04106AF3D793E689846DE
:20C1200004460B1CADF1180D074611D0012B15D130797379641C3870B17904F8013B337ABF
:20C1400004F8011BB17A04F8013B7389181201E03178707804F8011B04F8010B8AB9002D3C
:20C160000CBF42F20C0042F20D00694607F018FF9DF80000BDF8003004F8010B181204F80E
:20C18000010BB8F1010F34D0B8F1020F39D1002D0CBF42F2020042F203000DF1020107F0B5
:20C1A000FFFE7589CDB1681E01468B100DF1020201EB5371C910CBB2811000EB517121F047
:20C1C0000701401AC0B20121401C01FA00F0D15CFF3080F0FF000843D054E81DC2100DF113
:20C1E000020120464BF032FB7089C01D04EBE00407E0002D14BF02210121204602F05CFFE6
:20C200002418E41B06B0A0B2BDE8F0813EB542F2050002A907F0C4FE9DF80800002865D03B
:20C2200042F20100694607F0BBFE314D95F89401002836D020200AF089FB9DF8080000241D
:20C2400064229DF80810C5F88001009B85F89441581A02FB00F105F5DC70C5F8BC1107F059
:20C26000E9FC2648007868B995F8960130B92148007800283AD105F0B1F83EBD10200BF0ED
:20C280006BFB3EBD01A808F021FC95F82A020199451EB1FBF0F24243891A01918D4225D9B4
:20C2A00018E09DF80810642011FB00F0C5F8BC0105F5DC7007F0BEFCB5F878010124401C41
:20C2C000A5F878010023C5F88031202085F894410AF05AFD084991F85514204621B94FF40E
:20C2E00000700BF031FB3EBD07F030FA3EBDC046C00E00203E1F0020100100206505002064
:20C300002DE9F8439946904604460E1C44BF0020011C68D40BF0F2FC054631468022204674
:20C3200008F0FEFE071C04D097F82F0030F07F0003D128460BF0B2FD53E097F82F0010F0D8
:20C340000F0F46D100200A2107F1180640EA090941EA080896E8030008EA000019EA010653
:20C3600008BF002820D028460BF098FD07F1180003C804F1700604F1700508EA000809EA43
:20C38000010986E8000395E80C0007F1180696E8030007F118059943904385E8030070342A
:20C3A00094E80300BDE8F88310487968884202D07968A166786004F1600080E8000328461B
:20C3C0000BF06CFD04F140004FF0FF310BF051FAE5E728460BF062FD97F82F0010F00F0F9F
:20C3E000FAD102200021BDE8F883C046292601002DE9F04F09AF3C897D6816464FF0000A5D
:20C400000246002EADF1440DA04610933C888DF83CA05CD0304810F80690042E03DAA8EB25
:20C420000900C8464519F868A4EB080407AB0827A4B2C01D10F801C97F1E03F801CBF9D178
:20C44000080E264F03F8010B080C03F8010B080A03F8010B386C03F8011B9DF83C101E70EC
:20C460004369F86B98478346BBF1FF3F2AD0042E04DA03208DF80000022002E002208DF8BE
:20C4800000008DF8140002959DF83C608DF8026001218DF80110386C8DF8039007ABADF889
:20C4A00016800BADADF81840026A0193109E04956946F86B039690478346386C8269F86BAD
:20C4C0000FA99047BBF1000F18BFE42000D1504611B0BDE8F08FC046009E01001001002015
:20C4E0002DE9F04F06460020ADF1140D0090364F0291786801968047344D0390303D286AC3
:20C500002B4CC36CE06804216A469847DFF8A490DFF8A4B0DFF8A4A0DFF8A48026F0010610
:20C5200029F00109B14515D0584620F00100B04223D19AF900102F6AE06811F1020F06D0FB
:20C540005146BA6B91F9001090472F6AE0681D4908310EE098F900102F6AE06811F1020FAB
:20C5600006D04146BA6B91F9001090472F6AE0681449FF6A029A019BB847B14507D059467E
:20C5800021F00101B14204BF5146087001E04146087001202F6A0090E068FB6C04216A4615
:20C5A0009847094903988968884705B0BDE8F08F2C1C002059F300009DAB00002D1E0020AF
:20C5C0002C1E00207C130020D81800205018002039482549C0F878122449C0F87C12244959
:20C5E000C0F880122349C0F884122349C0F88812304AC0F8EC21C0F8FC212049C0F88C12A6
:20C600001F49C0F890121F49C0F894121E49C0F898121E49C0F89C121D49C0F8A0121D49C6
:20C62000C0F8A4121C49C0F8A8121C49C0F8AC121B49C0F8A0101B49C0F8A4101A49C0F823
:20C64000A8101A49C0F8AC101949C0F8B010002180F80C1280F80F12022180F8F011012163
:20C6600080F800127047C046A5740000F1380100B9480100653E0100BD270100415501000E
:20C68000996801004149010001300100CD4C0100CD7301005111010089520100FD730100D0
:20C6A00019790100D97001003900010085280100197D0100597901001001002070B5394D6F
:20C6C000064695F8EE02ADF1180D80B995F8300382280CD031480068314C016C206888472D
:20C6E0000AF025F895F83013D5F80423505495F83003822814BF401C002005F53B7485F8DC
:20C70000300395F8300304EBE00292F82C00411082F82C10400807D295F83003401C85F8DE
:20C720003003C0B28128ECDB95F8300381282EDA04F14401E120F7F7CDFF02204FF6FF73A5
:20C740008DF8100095F8EE12ADF8083031F0020019D0012919BF0720832108208021002216
:20C760004934009202AA0194F9F7AAFDDB2807D0E52805D0F32803D0DF2818BFE8280BD15E
:20C7800085F8ED0203E0304604F064FF04E02A203070304606F0A0F906B070BD401800204F
:20C7A000381C0020100100202DE9F04FDFF8D89000240646ADF13C0D4FF0010B2546A0464D
:20C7C0000D9318980C91DFF8C4A00E9047E016F8020FA41CA4B2401E1CD0401E09D0401E58
:20C7E00004D0401E35D1022F33D135E0032F30D132E0072F2DD1B1787078042240EA0120BC
:20C80000AAF88401F11C0AF5C4704BF01FF88AF899B121E0052F1CD1CDF80880B11C02A8AD
:20C8200003224BF013F80C9803A9FBF7E5FE9DF82A0088B1029BD9F80020039340F002001A
:20C84000049200F0F7008DF82A0003A805F0D2FB02E07819801C85B2E419F619A4B2304621
:20C86000694609F0C1F9071CB1D1022C03DC44466720254600E040460D990C800E990FB02A
:20C880000D80BDE8F08FC04650100020C00E002010B50446A068ADF1380D03464BF0CCF930
:20C8A0001B1D009018464BF0D8F99B1CADF8040013F8010B8DF8060013F8010B8DF80700A1
:20C8C00013F8010B8DF8080013F8010B8DF8090013F8010B8DF80A0013F8010B002100B180
:20C8E00001218DF80B1013F8010B002100B101218DF80C1013F8010B002100B101210DF1C1
:20C900000E008DF80D1019460AF01EFC0B3319460DF119000AF018FC0B3313F8010B0021BC
:20C9200000B101218DF8301013F8010B8DF8240013F8010B8DF8250018464BF08EF99A1C08
:20C94000ADF8260012F8010BA1888DF82C009DF82C000A922A30884218BF272105D1054958
:20C9600018206A4649F040FCC1B203200AF022FF0EB010BDCF7B01002DE9F04F364C606834
:20C98000ADF12C0D804700264FF6FF79FF273546A0468346DFF8C4A08DF800508DF80160D0
:20C9A000D0206946FCF792FB002849D19DF80B00012810D19DF80A0068B90DF10102082083
:20C9C000314612F8013FFF2B03D1401E01F10101F7D1082934D034462EE08DF82050ADF827
:20C9E000224008A9D120FCF771FB18BB9DF82400FF281FD0ADF800006946D420FCF766FB96
:20CA000028B1D8F8081058468847192020E0ADF80490ADF8069002A8394608224AF032FF7D
:20CA2000D4206946FAF75CFB8DF8247008A9D120FAF756FB641CE4B2BAF80000A042CCDCBC
:20CA40006D1C022DA8DBD8F808105846884730460BB0BDE8F08FC046D8180020681E002035
:20CA60002DE9F84F0746344800788B4620B93846F7F7AEF8BDE8F88F304DE989002405E038
:20CA80003868E989641CA4B280193860A142D8BF61204FDD38465946F7F79AF895F8F41127
:20CAA000002847D19BF80080D7F800A0002940D023480168C88AC2083BD280094FF00006B0
:20CAC00002D3087D152834D00AF03EF8AB898646002B06BFB5F80EC06346B5F80EC05B1E83
:20CAE000BCF1000F9BB224D0D5F810906146184600EB800048440278904506D003B9634646
:20CB00005B1E491E9BB2F2D113E0D0F8011070460BF0D6F842F21073642101FB0A018B42CA
:20CB200005D942F242706423401AB0FBF3F6002EA6D10020BDE8F88FB4100020C00E0020F9
:20CB40001401002035492DE9F04F0822ADF1140D039001A84AF07AFE314C60688047804624
:20CB60006946722009F0E0FB2E4C241FA0884FF6FF7690B10746002500990398091D4BF0B9
:20CB8000C5F8012808D000987F1E05F1010500F118000090F0D100E02E4621498968404617
:20CBA0008847A0884FF6FF71B14218BF301C30D18346194800F118010F88002F08BF0024CD
:20CBC00025D081461649D9F81450D1F8048000263446AA46504601A9082209F0EDFE40B1E9
:20CBE0007F1E06F108060AF1080A04F10104F1D10DE00399701908224AF028FEC047B9F876
:20CC00001A10074F491CA9F81A10B96888475C44A0B205B0BDE8F08FC00E002054A50100C1
:20CC2000D8180020681E00202DE9F0410AF006FF4FF08058D8F8E801406880470AF010FFB0
:20CC4000044604F00C000C284FD0E0081ED209F0B1FA294E37680546012001460AF003F9FC
:20CC600031686943884211D2244CF020B0FBF7F0291A20460BF00EF920460BF007F9012083
:20CC8000F8F7D4FE20460BF0FDF830E020092CD208F5EC75286880680146194888470428CD
:20CCA000F8D01849620905D220B10846016821F0010103E00846016841F001010160D0F878
:20CCC000981041F00301C0F89810D8F8B80180690146202088470C4CD8F8B8012168806BFA
:20CCE000804701202060206801E00AF0D9FF0AF0ABFEBDE8F081C0468CAC01001016002053
:20CD0000004003408C2108402C2009402DE9FF413448002407782C48334D0470203D2C7030
:20CD20006C702A48047028696C6110B128690AF0EFFF2E48801D008805F11008012F14BFED
:20CD400010300E3080B209F0CFFF06462E618DF804401F4B00969DF8050064F301008DF841
:20CD600005009DF8050064F383008DF805001889012F12BF1030174908809DF8051064F3E5
:20CD800007118DF80510ADF80600D8F80000082269464AF05BFD2E626C6200F099F80E4DC1
:20CDA0002878012802D02046F6F7B8FA0B4804700B4F3C702878012802D02046F6F7AEFA70
:20CDC0000090BDE8FF81C046B9350020BB350020641E00209C1400203D1F0020BD3500207A
:20CDE000B5350020BF0500201C340020661E00202DE9F0470D4606465FFA85FA280824BF5A
:20CE00002F4845402F494FEA8A032F4AC85806EA0504224085EA000706F4E0243740B4F550
:20CE2000E02F20EA0600C7F3006742EA000201D1500E14D306F4E020074310D002F4E0274C
:20CE4000B7F5A02707D0B7F5803704BF22F4003242F4A02203E022F4803242F4C022DFF888
:20CE60006C80CA5008F1D00739680122002002FA0AF40C4218BF101C5FEA000906D1F00D87
:20CE800004D34146C5F3805001F80A00300E0BD30AF01AFF290E34BF0021211C3A68A2436B
:20CEA000114339600BF012F8B9F1000F06D0F00D04D34046C5F3805100F80A10BDE8F087E0
:20CEC000006000A000100840007F077F002002407CB53148314E324D344C0078012813D1E6
:20CEE0006420694607F03EFC4034C6F830519DF80000C6F8344100280CBF2A482A48C6F8BE
:20CF0000D800C6F818017CBD2246C6F8485106F2471302F14C00C6F84C011978012506F21F
:20CF2000471465F3000119702378002006F2471160F3410323700B7865F382030B7006F2AC
:20CF400047110B7860F3C3030B7006F247110B7865F304130B7006F247110B7806F247147F
:20CF600060F345130B70217806F2471065F386112170017865F3C7110170052386F85631DC
:20CF800086F8573102F18804C6F8584102F16C05C6F85C517CBDC046BF0500207C13002014
:20CFA0001C3400204E9055550E7A5555201800202DE9FC47334DD5F8800095F8AF840028E1
:20CFC0005DD00020304E0090301D00688047D5F88040009F8146A74229D0607E30F07F0028
:20CFE00020D0608A401E80B2608210B1607EC00818D354F80CAC05F1800021463A464AF0F8
:20D000001BFBB8F1020F02D1204601F01FFC684621464AF065FB95F88A005446401E85F8C0
:20D020008A0002E0274654F80C4C002CD5D1B1684846884795F88A0078B195F839040F28EA
:20D0400001D0687848B905F5DC75284604F006FA4FF4707128460AF0AFF8F026E92509E031
:20D0600002F052FF607EC00834BF66706570204602F0FEFE68464AF0FDFA041CF0D1BDE870
:20D08000FC87C04610010020D8180020334B2DE9F0418846596804460AF036FC002750B1D4
:20D0A000586890F82E0041460AF0D1FB3E46051C18BF5F6801E03D460126186800B31A682A
:20D0C0001CE0204611460AF01FFC28B192F82F0040F0080082F82F0012682BE020461146CD
:20D0E0000AF012FC48B192F82E0041460AF0AFFB002608B10DB9174605461268002AEDD19D
:20D10000002E18BF022027D1002D14BF002F002022D058683A4690420CD1596820460AF09F
:20D12000F3FB38B1596891F82F0040F0080081F82F001A68002AC4D1094905F001058C6243
:20D14000BB8DCC6291F8340081F8325040F001020B86012081F83420BDE8F0813435002050
:20D16000003300207CB5344C054694F839040F285DD0697E6078890959D2297E002841F0B7
:20D180000201297639D069684A1C1078801010F0030F32D000F0030002280ED1B4F84C3459
:20D1A0004FF6FE70984208DD56791179002001EB0621994208BF012004E004F24240491DEC
:20D1C0004AF0A4FDC8B9687E696840F0010068764A78C2F38102022A2DD1491D4A78097860
:20D1E0004FF6FF7601EB02218E4224D1297E00F0EF0041F0200129761CE0687E40F0030015
:20D20000687694F86701B0B994F86F048DF80000FF238DF8033094F87E648DF8016094F895
:20D220007F548DF8025068460AF0D5FC7CBD687E40F0010068767CBD1001002070B50646C2
:20D2400000210B22ADF1280D0DF119004AF01AFB2E4D3078C01E15D0801E04D0143811D0C2
:20D26000801F01282FD801208DF8180006F18F0103A84AF063FD032495F840038DF8144085
:20D2800070B113E000208DF8180006F18F0103A84AF054FD032495F840038DF8144028B94F
:20D2A000B5F856040224ADF8020005E00DF1020005F58E614AF042FD8DF80A40B5F8520481
:20D2C000ADF8160017E002208DF8180006F1320103A84AF029FD0DF1020006F128014AF04E
:20D2E00023FD0B48008806F11C01ADF816000DF119000AF0CFFC0B208DF8000075788DF866
:20D300000150684600F0DCF80AB070BD10010020620500202DE9F843324C94F8AF940546C2
:20D320000AF0D0F9297E2E48090902D2297D012900D0401CDFF8B08007784646706880477A
:20D3400004F180010B68002B08BF0D600CD07F1E0026FFB202E07F1E1346FFB253F80C2C29
:20D3600022B92FB143F80C5C012601E0002FF2D1D8F8081088475EB3B9F1020F02D1284691
:20D38000FDF7AEF9A16928468847E88AA168C0081AD2D8F80400804794F88B10491C84F8D9
:20D3A0008B10D8F80810884794F8400310B1D4F8540330B9E88A400A0FD2FCF725FFBDE826
:20D3C000F8838047BDE8F88328468847BDE8F883F1206870284602F04BFDBDE8F883C046D7
:20D3E000641E002010010020D81800202DE9F043DFF8BC808946054617464FF0FF31ADF16A
:20D40000140D40460AF035FA2A4C04EBC504666825680AF059FC84462068006849460028F3
:20D4200007D42868002803DC41B14FF0FF3107E021B160460AF04AFD002431E02968491C4E
:20D44000296060460AF042FD2868022828DA1FB903A80AF0B4FB03AF38686860B768684695
:20D460000AF02AFA317B009405F12C006B46124A0191394607F0EAFC05F16400002108F0BE
:20D48000BDFD05F14800012108F0B8FD706800F0DDFE0A4A05F118002346042108F0BCFF7F
:20D4A00040460AF027FC204605B0BDE8F083C046A834002040AC010055670100F77B010077
:20D4C00070B50646304930780D5C401F1CD0083851D0401F4FD028464AF04AF9041C0DD13E
:20D4E00030780C2808D1706830B1301D07F0EAFE28464AF03DF90446002C43D02A46204655
:20D5000031464AF0A3F937E0B07810BB307C317A2D184C10480000F00E002D1804F0380005
:20D520002D182435E8B24AF023F9041C2AD0314618224AF08BF904F11800606071682422E8
:20D540004AF084F96068243060617169327C0E46D6E7012816D12435E8B24AF009F9041C3F
:20D5600010D0314618224AF071F904F11800606071682422EBE7344624B10448007821463E
:20D5800049F0ECFF70BDC046A0AB01004C1E00202DE9FE4F8046314DDFF8BC9095F84003C4
:20D5A000174609EB4806683634880191C0B1D5F85813A9B109EB880BDBF8DC0000F0FF00B8
:20D5C00088478246D5F85813DBF8DC0000F47F008847504483B21BB13088C018001D84B213
:20D5E00095F8640401280AD1387A40B148447B7A067919F803000019401D84B200E00026C9
:20D60000A01980B24AF0B4F895F800A0071C19D0002122464AF036F9002587F8008008EBF7
:20D62000090138197D704A7D786007F1840001993E814AF00BF95046394649F08FFF2846A6
:20D64000BDE8FE8F8DF8008068461A2102F020FE1A20BDE8FE8FC046FC9D0100100100205D
:20D660002DE9FF412E482D4F00683E78C06B80477968401AB100B0FBF1F4B868FF6800252A
:20D68000A8464146BC4271EB080101DAB84206D82946424684428A413CDA074600E02946C5
:20D6A00038463246F317001BA94109F01FFF272704464FF47A7200230D46ADF802700820D2
:20D6C000ADF800002046F8F7EBFC01901548016868468847029843464FF0000100F6FC023E
:20D6E000A41A9D416042A94111DA0F48026829462046F8F7D5FC0D4604464FF00001604242
:20D70000A94104DA204607F001FA002000E00120064908700090BDE8FF81C046701D002099
:20D7200040180020D8180020181C0020BC3500202DE9F04106467078032806D0777D3D4609
:20D7400010B105EB4515ADB201E000273D461635ADB2284608F0C0FD5FEA00084DD004464F
:20D76000307804F8010B707804F8010BB07804F8010BF078311D112204F8010B204602F090
:20D78000F7F9717D04F1110000F8011B747844B3B46957B3214608F0BBF861894AF057FA00
:20D7A000A1894AF054FAA17B00F8011BE17B00F8011B217C00F8011B617C00F8011B6169AB
:20D7C0004AF01DFA0346207E04F1190103F8010B184609F0C7FC243403F10B007F1ED9D143
:20D7E00003E0B1693A4602F0C3F929468C20424602F094FF404609F067F9BDE8F08170472A
:20D800002DE9F041804608F033FFC01DC51098F8230000284DD198F87E4008F029FFA042D6
:20D8200047DD284A5368E1100846C91891F8701004F007042141CFB2082409E0411C04EB2B
:20D84000C000C9B2CE1896F8707088F87E00084647B9691E8142F1DC5068002188F87E10EF
:20D86000417029E098F97E10C0000830884226DD401A79080BD298F87E10401E4FEA67072F
:20D8800001F1010188F87E10F3D1BDE8F08198F87E000D49087098F87E0088F8810098F831
:20D8A0007E00401C88F87E000320F8F7E9FABDE8F081002088F87E00072005F047FFBDE860
:20D8C000F081C046100100207B1E002003B42DE9F047304C4FF0000908AF84F801903968BA
:20D8E000ADF1100D02A80160B988818002A803C89A46164608F0A4FDA046051C14D04C4659
:20D9000086B12846694601224AF088F81AF804009DF80010884205D1641C6D1CE4B2ADB27D
:20D92000A642EEDCA6422ED0B8F80200F61C4FF6FC7441F6F8753440001985420ADA0AF000
:20D9400023F8FCF789F8B8F8020000198542B8BF012019DB396802A8BE88016002AD868073
:20D9600095E803002246534601F07AFF98F80100B8F80210002818BF814604D16418083416
:20D98000A0B2A8F80200484604B0BDE8F04702B07047C046901E00202DE9B04314460F4680
:20D9A00080460AF091F981462D48027883254146381C45D0401E3DD0401E38D0401E32D09E
:20D9C000401E22D02249401E0FD0401E29D1D2B908460AF08BF9B0B921681E480AF096F9BF
:20D9E00021681D480AF092F92CE062B908460AF07DF940B9216819200AF06EF921681A20F0
:20DA00000AF06AF91EE000251CE0206828B1012807D1802008F080F814E0802009F0DAFBB6
:20DA200010E003250EE020680C4908600AE02088488207E00122C8684A746030C86001E0AE
:20DA40002068086048460AF041FA2846BDE8B083343500206C330020A03300207C340020C2
:20DA6000B03500202DE9FC4707460E1C14BF4FF000084FF0E808002F50D0B8F1000F4FD161
:20DA80007868401E78603F210170BD6D002D0CBF802000207968DFF894900224083E491E0E
:20DAA0007960DFF884A008703889A7F85440801C388116F8080FFF282DD02A2829D1706864
:20DAC00038B3D9F858138847054678689AF80020401B78607168CC4631B9DCF85CC33A46F8
:20DAE0000023E04750B10CE0DCF85CC3786871688DF800206B463A46E04710B9EB20BDE8CD
:20DB0000FC873889B7F85430401938815819A7F85400641ECDD17868386501E04FF0E8086B
:20DB20004046BDE8FC87C0467A1E002010010020F0B506460F4600251446ADF1240D8B2009
:20DB40000DF10E010095FBF7C1FA8A2001A9FBF7BDFA707A00282ED1387AA0B9BDF80E108A
:20DB60004FF6FE70884205DCBDF80E10884220D101A90DE020489DF80E700488BDF80E0058
:20DB80008DF812700CE0022807D0032811D1394604A84AF0D3F809240BE038888DF81200E5
:20DBA0008DF81040211200128DF8111005248DF81300284611E002280CBF05240924012811
:20DBC00018BF311C04D1892007A9FBF77FFA07A9224604A849F03AFEB07A0DEB0401C873F1
:20DBE0006A4604A8214603F01DFF002814BF281C009809B0F0BDC04662050020F0B5314E65
:20DC0000044696F8EE02ADF13C0D022807D0012805D005281CBFE82086F8ED024AD196F830
:20DC2000340300284BD1002109A8182286F8ED1249F028FECDF828D009A8214600F02AFC96
:20DC400096F8020396F82C13814220DDD6F8045370B10746BDF80A006989884204D1284653
:20DC600069464AF03DF890B97F1E05F12405F1D196F80203D6F80413242210FB0210694635
:20DC800049F0E4FD96F80203401C86F8020396F82E0428B19DF8340010B996F82C0328B92F
:20DCA00009A8FFF70DFC96F82C0340B196F80213884204D12A202070204604F00DFF0FB0C5
:20DCC000F0BDC046100100202DE9F04F044628480078ADF1140D012843D10125DFF89490BC
:20DCE000DFF8948089F8005098F80000012802D02846F5F713FB204605F020FC1F4F7868B0
:20DD0000804700248DF80C50834602941C498DF80D401D4D4C80286A1A4A066D02238DE868
:20DD200018001A4B10688A4602AAB047B968E88000280CD54846047058468847404600787C
:20DD4000012802D02046F5F7E9FA20460DE0104A92F90000C5F80CA0401C107058468847A9
:20DD600002E0204605F0EAFB012005B0BDE8F08FBF050020301E00203D1F0020D8180020A9
:20DD8000CC130020381C002020180020E5440100361E0020F0B5304C284B0021382004F118
:20DDA000B402ADF13C0D11FB00250F46EB62791C17FB002595F82670C9B2002FF3D04FF058
:20DDC00080561F48D6F8D87101211E4D3B6810630A4628469847D6F8D801426801212846CE
:20DDE00090471E4818495C3802681948914218BF2C3008D115490C224A71032781F82470C9
:20DE0000022681F82560F9F7EDFE684600213C2208230AF033F84FF448770126204600F500
:20DE2000E6716A460897002307910A4906960AF021F80AF01BF80FB0F0BDC04663F10000AC
:20DE4000816001000040034000808220941B0020E8A80100D9B500006C060020F012005069
:20DE60002DE9F04180460C46B8F1850F0CBF33253425B4F84010608C4018401985B228464C
:20DE800008F02AFA071C4ED0214607F041FD04F10A0107F03DFD616949F0B1FE218B49F0C1
:20DEA000D6FE618B49F0D3FEA18B49F0D0FE0346A07F03F8010BE07F03F8010B94F82000E4
:20DEC00003F8010B94F8210004F1300103F8010B184609F047F9E16A03F10B0049F08FFEBA
:20DEE000B8F1930F04BF94F8281000F8011BB4F8401049F0ACFE618C49F0A9FEE16BB4F898
:20DF00004020064601F034FEB4F84000616A628C301801F02DFE404629463A4602F0FEFBC9
:20DF2000384608F0D1FDBDE8F08170472DE9B043044609F0C9FE81462A48221892F8EF10C1
:20DF4000491ECFB2002F82F8EF7044D1284901EB84010D78498835F07F0788461AD1E9092E
:20DF600011D24FF08054D4F8B801806901464046884704F5DC742068406B01464046884789
:20DF80000228F8D121E000EB8800D0F80411002088471AE04FF08054D4F8B801006A01460B
:20DFA00040468847D4F8B801806A014640468847D4F8B801006B01464046884701210A4AFF
:20DFC0000A48116001688908FCD305F03F00152801DAFFF7ABFF484609F078FF0020BDE806
:20DFE000B083C04604160020282008602820084020AA01002DE9F84314460D46804609F0E6
:20E0000063FE04F00107C4F34006274C294681460325B1F1FF3F08D16168404609F074FC64
:20E0200000280CBF2168616804E04046002207F077F80146002930D091F82F0030F07F00E2
:20E040002AD0201D006888420FD04046324601F031F908B31548007801281BD0042819D0A6
:20E060001348022109F04EFE14E091F82F200120002F00FA07F040EA020081F82F0014BF29
:20E080000C480D4808F0AEFB26B121684046324601F010F9832500E00425484609F016FF91
:20E0A0002846BDE8F883C04634350020B03500206C3300200100020401000104B0B5304D90
:20E0C000044695F8AF04002701280DD1E07A09281CBF0A28E827207B08B1042804DB8028DA
:20E0E00001DB882800DBE82794F8340010B195F8400348BBA07A8028C8BFE827607B1028EB
:20E10000A8BFE8270F2804D0B5F85C10090938BFE827A17B884202DA0F2918BFE827E07B12
:20E1200050B194F828000F2818BFE827608D43F6FF71814218BFE827B5F856044FF6FF7112
:20E14000814208BFEC2719D0C7B904F10C01E820F6F7C0FA04F10B01E720F6F7BBFA34200A
:20E1600049F0E2FBC5F8C801002808BF1A2705D0D5F8C801211D342249F068FB3846B0BD4D
:20E180001001002070B52A4D95F8AF04012802D0A878012801D003F021F902F097FF95F83B
:20E1A000400318B12348016801208847234895F8AF64007808B922480078224C606880476C
:20E1C000214AA1681378022B27D101231A4C1370A378022B03D0032B18BF062B01D1832345
:20E1E00013708847A17831F001000AD0042908D0052909D1012E07D10020607109F0D4FBEB
:20E2000001E0F8F779FBA178022903D0032918BF062903D103F05CFA00E0884795F84003D5
:20E2200028B1D5F8540310B1102009F095FB70BD1001002030180020481D0020B93500200E
:20E24000BB350020D8180020BD3500202DE9F041064609F039FD2A4D8046711991F8EF008B
:20E26000421C002881F8EF2043D1264C04EB8604277807F03F00152801DAFFF7E7FF6688DA
:20E2800037F07F001AD1F80911D24FF08054D4F8B801406901463046884704F5DC7420686B
:20E2A000406B0146304688470128F8D121E005EB8605D5F80411012088471AE04FF08054DA
:20E2C000D4F8B801C069014630468847D4F8B801406A014630468847D4F8B801C06A014653
:20E2E000304688470121084A0848116001688908FCD3404609F0EAFD0020BDE8F081C04639
:20E300000416002020AA010028200860282008402DE9F8432E4D0120002428702648DFF8CA
:20E320009C80DFF8A0900470254800F1C2010F8814EA03064FF0020101EA020108BF002967
:20E340000FD120464FF0E04710401F4008BF002823D0424692F90000401E107009F07EF820
:20E360001BE0424692F90010491E117047B901F045F84846047098F90000A0B1424616E007
:20E38000B7F5505F07D111480F49006800F5C070086007F073FB09F025F84846424604709F
:20E3A00092F9000018B92046F4F7B8FF01E092F900002C70BDE8F883301E0020361E0020EF
:20E3C0007C1300202F1E0020381800200C0100213D1F0020F0B585686A7D2C49ADF1140D5A
:20E3E00042F000462B7DAC7D009646680027FF2C41EA03024FF00203019202D0E87DFF28D9
:20E4000000D13FB1EA7DA87D11430423039140F000400290FE2106F154004DF8231069460D
:20E4200001F0ECFE3066306E002808BF381C2AD0174C29688C4214BF13220F22697D07F0B8
:20E44000C7FD2868844214BF14221022297D306E07F0BEFDA97DFF2902D0E87DFF2800D1F4
:20E4600087B12868844214BF15221122306E07F0AFFD2868844214BF16221222E97D306EF7
:20E4800007F0A6FD012005B0F0BDC0460000C0A000100040F8B505460E460520287096F812
:20E4A00049006968E870F06B4861686806F1280149F03AFCB6F842006968488196F8460029
:20E4C00069684874686800240476214869680078C873686806F11C01193009F0DBFB307CAC
:20E4E000696888737268696812F8010B8881696812F8013B888940EA0320888117786968A8
:20E50000F81117F0070708744FF0030017FB00F1204618BF01204018C1B28918491C11F8E4
:20E52000010B287200F00702E960401000F0380000EB420040187268318968615318834269
:20E5400039BF2C72211C801A091A2974F8BDC0468E05002000B581882829ADF12C0D50D119
:20E56000836818788DF811005B1C13F8010B8DF8120013F8010B8DF8130013F8010B8DF81A
:20E58000140013F8010B04288DF8150007DD9DF81100032803D010B104208DF8150013F878
:20E5A000010B002100B101218DF8161013F8010B8DF8170013F8010B8DF8180013F8010B32
:20E5C000002100B101218DF8241013F8010B8DF82500184649F041FB9B1CADF82600194619
:20E5E0000DF1190008F0B0FD112203F10B01684601F0BEFA064918206A4647F0F5FDC1B202
:20E6000000E027210C2009F0D5F80BB000BDC04691E7000010F47C1F7CB524D110F00F0F07
:20E6200024D006460024012505EA0600AE436D00401E13D0401E0FD0801E0BD0001F0FD107
:20E6400042F20500694605F0ABFC9DF8000038B1093404E0241D02E0E41D00E0641DA4B2BC
:20E66000002EE1D133E010F00F0F01D000207CBD064602244FF4803505EA0600AE436D00A2
:20E68000B0F5803018D0B0F5803013D0B0F500300ED0B0F5802009D0B0F5002004D0B0F5F6
:20E6A00080100FD1072008E0062006E0052004E0042002E0022000E0012000F083F9001918
:20E6C000801C84B2002ED7D1022CD8BF002420467CBD70472DE9FF472A4C89468246211DAC
:20E6E0000888401C088028490822684649F0AEF8208B4FF6FF7880B1656907460026284637
:20E700005146082208F058F930B17F1E05F1080506F10106F3D100E0B0464FF6FF75454593
:20E7200004D1207A401C20722E4627E0404602A901F01AFD0646B542F6D09DF808000128F9
:20E7400007D0A16D700000EB86004018A0F8049005E0616D06EB46104018A0F81F9060690D
:20E760006946082200EBC80049F070F8074D68688047618B491E6183A96888473046009064
:20E78000BDE8FF87C00E002054A50100D818002030B50546ADF12C0D08F0C6FF002818BF93
:20E7A000FC2051D168462946112249F04FF8AC7C697D8DF81240687C8DF81510EB7C8DF8EC
:20E7C00011002A7D8DF81330AC7D8DF81420002104B101212C7E8DF8161095F825208DF833
:20E7E0001840E87D8DF8252095F824308DF81700EC8C8DF8243005F119010B220DF1190070
:20E80000ADF8264049F022F8687C002448B9812049F08AF80A9080B1FF21812249F032F844
:20E820000DE09DF815000A9448B1242110FB01F080B249F079F80A9008B91A2403E00720EA
:20E84000694603F0AFFC20460BB030BDFEB50446607E30F07F0053D0207D0027012818BFFC
:20E8600003284DD1274DB5F85C0000F0020100F00800084344D061684878C0F381000228A1
:20E880008DF8080006D003280ED1491D684649F055FA09E08A79487940EA0220ADF80000D1
:20E8A000CE78087946EA0026D5F880000146A8B1487E30F07F000AD0087D012818BF03285F
:20E8C00005D14A686846314606F018F828B954F80C0C00280146EBD100E0274687B99DF8F3
:20E8E00008003146022818BF032809D1684602F071FCFF2804D09DF80820002106F046FA77
:20E90000FEBDC046100100202DE9F843DFF8AC9099F84900002848D0002501212C4699F83D
:20E92000492001FA04F0104203D1641C032CF6D33BE099F849201020A040104218BF0D1C6A
:20E9400009F0C2F999F849201121A14081F0FF01114089F8491009F0B9FAE0B208F0AEFD79
:20E96000071C22D0B87A00B397F90960304608F0FBFF38687C68012D804606D0387A022812
:20E9800004D1F868400B01D303E08469384602F063FC012D19BF311C4FF000636FF0FE0131
:20E9A0004FF0007340460022A04799F8490018B10348002109F0A6F9BDE8F883B03200204D
:20E9C000A033002010B5401EADF1380D28D0401E09D0801E4FD0401E43D0401E3FD0401E16
:20E9E0003BD0002048E001A800F0AAFD04460CA942F2090005F0D4FA9DF83000002808BFD1
:20EA0000002203D0022007F0A0FA024601209DF83010009001AB204605F03BFE0A3028E0FE
:20EA200001A800F08DFD04460CA942F2080005F0B7FA9DF83000002808BF002203D0012008
:20EA400007F083FA024600209DF83010009001AB204605F01EFE001D0BE020200CE00220FC
:20EA60000AE042F2130004A905F09AFA04A848F00BFF80B200E004200EB010BDFEB54FF08E
:20EA8000805684684568D6F8D0112068C9688847216822488A6B1040886340F2F271206890
:20EAA000204B41641E4994F8210094F82020085C9A5C216810434863684609F0F5F81C4F86
:20EAC000DFF868E0D6F8D0112B7FDFF85CC06A7FA87F496857F823705EF82260AA695CF8E9
:20EAE00020300D46206801993E433343A8472168C86A40F01000C8622168086B40F0010019
:20EB00000863A07D0027FF2802D0E07DFF2800D11FB1086B40F440400863FEBD0DF8FFFFD8
:20EB20005EAC01006AAC01008CAB010050AC0100E8AB010038B520481E4CE0641F482065FB
:20EB40001F48C4F8F4001F48C4F8F8001E48C4F8FC001E48C4F800011D48C4F804011D48B7
:20EB6000C4F808011C4820671C4860671C48A0671C480025E067D4F8C801C4F80C5108B118
:20EB800048F0E6FEC4F8C85117486570082384F8CC512946C4F8C0010B2284F8C43104F20C
:20EBA000CD1048F06FFE04F5EC7029460B2248F069FE38BD10010020D91501004D5201008E
:20EBC000C9A00000BD450100496D01005D130100D1650100B1CF00005927010039FA000036
:20EBE000D15D010001770100597901002348F8B500248460224904602848224609F06AF878
:20EC000020480068006B80472049254B1E4D0A685F782968801A01EB1030286037B19F7887
:20EC200027B91B490968B0EBC12F21D908F0CCF8D0B1184840F60901018000F10D02448078
:20EC4000117800F10C0621F00F0141F001011170317864F3030131702146416008F08CFE24
:20EC6000418811F4406FFBD02C609C700120587005F0CCFB08480460F8BDC0460C10044040
:20EC8000F52601008C01001078340020703400207C3400207435002000000460C434002016
:20ECA000B0350020BFB50446FFF708FA071C48D1607B0F2828D0DFF89CC09CF867110229E9
:20ECC00022D1E77BEFB90CEB4000B0F82C019CF85874400083B260684FF4707202FA07F571
:20ECE000E91881420BD89CF8391402FA01F1CB1A834204D3A37B491B9A40914202D2FD27F6
:20ED00001FE00020CCF83C04607C0027C8B194F83400B0B90E48007898B904F112010920DB
:20ED2000FCF7B2FA68B102218DF80C104FF6FF72ADF80420A77A0097238901A901F04CF895
:20ED400003E067702046FCF7E5FD0090BFBDC04650040020100100202DE9F0470F462749F5
:20ED60003A6805464FEA9209494502D3387A022802D00320BDE8F08708F0A6FF204C8246B1
:20ED8000201D0068A84214BF00260126B00080F004002158284607F0AAF88046194802688F
:20EDA000B8F1000F0CD194F83400A56240F0020084F83400504609F089F80020BDE8F087C9
:20EDC0003968B00000EBC600001901613B7A9C35B9FBF2F10376284608F0DBFB504609F055
:20EDE00075F8B8F1010F06D1E06AB4F9301094F8322008F0FCFE8320BDE8F08740420F00BF
:20EE000000330020A035002098B5294C204608F06DFF0746012004F0C3FC606800283FD1FD
:20EE2000002F39D01F48F9680068884231D1684604F00AFD38B1009828B1E06818B908205A
:20EE400006F06AFE98BD082008F0C4F938691649C043486038698A681043886007F11000A1
:20EE600090E80C00181CC04341F8040C07F1100090E80C000A68181C10430860B86807F08A
:20EE8000B1FC204608F042FA6060002004F088FC98BD4FF4806100E00221044808F032FFE2
:20EEA00098BDC0466C3400200C1004406C3300203435002038B5294C0546D4F8C80190F8C5
:20EEC000300010B194F84003B8B9687A84F83904A87A84F85804287B05F1240184F82F04FF
:20EEE0005F20F5F7F7FB05F126016020F5F7F2FB05F125016120F5F7EDFBE87AA07005F067
:20EF000039FB05F10801E820F5F7E4FBE91DE720F5F7E0FBA07838B1291D5020F5F7DAFB9F
:20EF2000A91DE120F5F7D6FB94F839240121002061700F2A18BF081C84F8CC0105F10E01CF
:20EF40000B2204F2CD1048F081FC04F5EC7005F119010B2248F07AFC38BDC0461001002090
:20EF6000F8B5284C6068804706462148A1680278832A3AD11F4D2F797FB38621017008206B
:20EF800007F002FF688B1D49401C68831A481E4FC1621B493A7891F8AF34012B13D191F8CC
:20EFA0007F14802908DD842906DA40F6485191FBF2F101F6B8310BE040F6485191FBF2F15C
:20EFC00001F2A32104E040F6485191FBF2F19631243008F0F1F8A16807E0852202703046DD
:20EFE0008847002001F0E8F9F8BD30468847F8BDBD350020481D0020C81B0020694101005C
:20F0000010010020D8180020701D002090B5044600214022ADF1440D684602F0D9FBA07875
:20F020008DF80000E0788DF801009DF8000000BB616811B101A805F0E8FC217A01F007027B
:20F040008DF82820E0689DF82870C1F302118DF8301027B19DF828100B9000EB41009DF8E1
:20F06000307007B10D90207C8DF8380067690F9719E0616811B101A805F0C7FC677A8DF881
:20F080002970A37A8DF82A30207A8DF82800E27A8DF82B20217B8DF82C10677B8DF82D7007
:20F0A000E389ADF82E300348006801696846884711B090BD201E0020F0B501290446054677
:20F0C000ADF1140D04D0022941D142F2030001E042F20200694604F063FF04B16D1C07F0D8
:20F0E000C7FAC01DC010C0B2002830D000230646ADF1010C1F4618461CF801EF00224EFABD
:20F1000002F101F00101884211D028B97F1CBFB25CB102EBC30103E03CB102EBC301491ECB
:20F1200005F8011B091205F8011B80F00100521C082AE4DB761E03F10103DDD130B12CB1BA
:20F14000D800401E05F8010B001228700FB9002005E004B12770012000EB870080B205B033
:20F16000F0BD7047F8B50B4601460024104603B90124002200B90122DFF88CC0DFF884E02F
:20F18000E3B19E6AD6B14F6AC7B1DC68CD68A54206D073461D68A54214BFDB689B6800E0C7
:20F1A0000023BC086546A4EB9604E41AA54222DBB4F1704F01DB002C1DDD0124F0B1476AD5
:20F1C000E7B18E6AD6B1C068C968884206D073461968814214BFD868986800E00020C0EB64
:20F1E00097006546A0EB9600854204DBB0F1704F03DB002801DC0020F8BD01221440E0B2E5
:20F20000F8BDC04600330020FEFFFF2F70B5274C0120002684F86401254D6670ADF1180DEA
:20F2200084F86761281D006884F8696180470246D4F8800068B1417E8B0806D341F00101C5
:20F240004176017E01F0FD01017650F80C0C0028F1D1A96810468847102008F07DFB0820CA
:20F2600008F07AFB94F86801D8B9E0258DF8015009208DF80000B4F852348DF80F6094F860
:20F280006F24ADF8023094F87F148DF8042094F87E548DF8061068468DF80550FEF710F9BD
:20F2A00001E084F8686106B070BDC04610010020D81800202DE9F843264C814620680F4697
:20F2C00090460025B8420AD0206800E0006820B1016811B101688F42F8D1074606E004F168
:20F2E00010064846394608F00FFBE0B977B310343968484608F008FB88B1396891F82F0026
:20F3000040F0040081F82F00086800223860204604F0DEFE6D1CB8F1010F01D016E03F6801
:20F32000002FE5D112E097F82F0040F0040087F82F00204607F0EAFF30463946002204F005
:20F34000C7FE27686D1CB8F1010FCAD02846BDE8F883C04634350020F8B50120204E2149BA
:20F3600030706FF00100087021480068C06B804720490A7894004A68821AB2FBF4F363434B
:20F38000D21A801A4860896804FB01011648FDF7A7F8164DEF6A2C6BA96A604207F02CF938
:20F3A00005E078688442DCBF001B78603F68002FF7D1686BA04202D0286305F007FD04F097
:20F3C00041F90D4C606880470546FEF749F9A1682846884707F0E2FE00203070F8BDC046F1
:20F3E0003D1F00202C1E002059F300001001002040180020701D0020D818002070B504212B
:20F400002548244C254D017094F8AF64687994F85014401CC0B28142687137DBA8780328F5
:20F4200034D0012E02D101F0D9FFA878042807D194F8400320B1D4F88C1309B10220884723
:20F44000687894F85D14421C9142C4BF401CC1B269706168012E04D14868098901F0A6FCD1
:20F460006168496894F840030988090902D308B106F0EAFAA878052805D1012E09D168792B
:20F4800008F092FA70BDF7F737FA70BDE12000F093FF70BD10010020BD350020481D0020F7
:20F4A0001CB5214C04F5DC7006F0DAFE04F5CE7006F0D6FE04F5EA7006F0D2FE0021882216
:20F4C00004F5BA7048F0DEF908F098F807F0D0F884F89A01154984F89B0115480860012040
:20F4E0000DF1010184F8F30142F2040004F058FD42F20500694604F053FD0E489DF80110F3
:20F50000C4F8A801642011FB00F1C4F8A0110A49C4F8C4119DF8001011FB00F0C4F8BC019A
:20F520000648C4F8E0011CBDC00E002030180020B15C0100853C01000DC200002F7C010066
:20F54000F0B50446E820ADF1240D08A905F00AF99DF82000694607F0C4F800280CBF00989A
:20F560001D480DF121016060E82005F0FBF89DF8210004A907F0B5F858B90599C820032293
:20F58000B1FBF0F0401EB0FBF2F15143401AC0B200E00020207207F06BF8002167686081D6
:20F5A000072321700D4A61705568BD420CD1157A267AB54208D15589854205D1107820703D
:20F5C00057786770084604E05B1E02F10C02EBD1012009B0F0BDC04638C40D00640F0020F4
:20F5E000F0B520480127F84201D004F055FE204D204F214EBD4206D203CD0478A4003459E5
:20F60000401CA047F6E71D48002800D08047164D164FBD4202D210CDA047FAE7F0BD032591
:20F620001BE0416808300A1C2A400BD11A1C2A40AB4305D0046804300C600431043BF9D1D5
:20F64000131C05D0047801300C700131013BF9D1021C2A4001D0A84304300368002BE0D186
:20F660007047C046FFFFFFFF000000000000000080B10100A8B1010050B10100D5BB0310A0
:20F6800003B426482DE9F041008806AF1646ADF1080D001F84B2082C39DB3D78201F694672
:20F6A000082280B2804648F0B9F9BDF80000C10B19D300F0FF00854215D17888BDF802106E
:20F6C000884210D1B888BDF8041088420BD1BDF80600002E18BF40461AD1C0F30E00241AA0
:20F6E000241FA0B214E0BDF8061008466FF30E0048B908460830844202DA48F0C1F906E0F7
:20F70000641A083C00E0241FA4B2082CC6DA002002B0BDE8F04102B07047C046921E0020F3
:20F7200080B58188ADF1200D1D2918BF27213FD18068034648F091FA9B1CADF8000018469D
:20F7400048F08BFA9B1CADF80200194601A808F09FF903F10807384648F06EFA3B1D0690E7
:20F7600013F8017B002007B101208DF80C0013F8017B002007B101208DF81C0013F8017BD0
:20F78000002007B101208DF81D0013F8010B19468DF80D000A680DF10E073A604B687B6019
:20F7A000087A387205496A46182046F01DFDC1B2332007F0FFFF08B080BDC046614100003F
:20F7C0002DE9F84F244C834660688A46804706462248A16800F180021768884627B930465F
:20F7E00088470020BDE8F88F002581462C46BC4220D0787E30F07F0018D07A68514658460E
:20F8000005F07CF890B144B1207D012812D16168087840F0100008700CE03C46607E40F023
:20F8200010006076207E40F08000207657F80C7C002FDED141463046884754B199F84003A4
:20F8400020B1D9F8540308B1804701E0FAF7DCFC01252846BDE8F88FD81800201001002084
:20F8600003B426482DE9F041058806AF1446ADF1080D98464FF6FF70ADF800000222ADF8CD
:20F8800002006946ADF8040044F40040ADF80600281986B2304602F03FFBBDF806000222F1
:20F8A00069466FF3DF30ADF80600304602F034FBA1102846CAB2414602F02EFB387840F4C5
:20F8C0004040ADF800007888ADF80200B88802226946ADF80400304602F01EFBBDF800006A
:20F8E000022269466FF3DF30ADF80000304602F013FB02B0BDE8F04102B07047921E0020E8
:20F900001B4838B50468B4F1FF3F08BF002407F057FB04282BD12048164B00251038056051
:20F920001868806C80471448006820B1134800682046F6F793F9124812490560124C0A6873
:20F940006FF35B4244EA0200086010490868C0F30130012806D10A680D48104040F40032E6
:20F960000A6008600B4908680028FCD138BDFEE71C130050F00100108001284380052043CE
:20F980008C210840482003400000390128000940EFFFFCFC0C00684294046042F0B5214838
:20F9A0001F4DE86000F5877028611F48ADF1240DA86004F03DFF684607F0C0FC4FF4E130FB
:20F9C000069003208DF81C0000248DF815408DF816408DF81D4001208DF800008DF80100E6
:20F9E0001248039012488DF8174069460490204605F078FB20212246686008F0C7F80D4E50
:20FA0000706880470746202205F1140168682C8008F0C1F8B1683846884709B0F0BDC046AE
:20FA2000601B002060110020B94F0100DD120100A1630100D81800202DE9F84FDFF88C903C
:20FA4000DFF88CA005464C469AF8AF84606880478346DAF88000E726074618B30022544676
:20FA6000787E30F07F0007D0387D012804D1287997F89D10884205D03A4657F80C7C002F65
:20FA8000EED10FE004F18000394647F0D5FDB8F1020F02D13846FEF7D9FE94F88A00401E70
:20FAA00084F88A00D9F80810584688473FB1384600F02AFA3846F02100F0EAFB0026284670
:20FAC000314600F0E5FBBDE8F88FC046D81800201001002010B5244C08BB04F1CC02117828
:20FAE000002004F1740360F303011170197860F303011970206794F8781004F1780241F0F6
:20FB0000080184F87810117860F30411F420117004F1790104F026FE44F6206019E004F123
:20FB20007801087840F00800087094F8780020F0100084F8780047F03DFF0A2280B24FF4F0
:20FB4000FA6390FBF2F1514344F62062401A10FB0320064AC4F8800092F8401319B1D2F805
:20FB6000A01301B1884710BD7C13002010010020002A4AD05FEA000C8B071CD1830722D10F
:20FB8000102A08D370B4103A78C978C0103AFBD270BC103238D0042A2CD3082A05D30C2A6F
:20FBA00024BF08C908C008C908C008C908C092072AD0920F22E00B780370491C401C521E3A
:20FBC00022D08B07F7D1C30714D18307D8D0121F12D308C903801B0C4380001D121FF8D28C
:20FBE0000AE008C903701B0A43701B0A83701B0AC370001D121FF4D2121D05D00B78037081
:20FC0000491C401C521EF9D1604670472DE9F041244C0B460146207D002704283ED08D783A
:20FC2000666A012819D1C3B1616A4FEA850851F8083033B151F8250006F036FF46F8087028
:20FC4000207D617D6D1CEDB2A942D8BF27831CDDA577A27D218B891A2183032812D0607DC4
:20FC600056F82530401EA842D4BF227EA27D0120617F2075207F121DD2B2F8F755FE071CFA
:20FC800003D1207D032802D008E003202075208B00280CBF0620052003F0ACFD3846BDE8AE
:20FCA000F081C046D4330020D0B5244C04F180010F68002F3FD0002215280AD13B7D01266D
:20FCC000022B08D0032B06D0052B04D0042B02D000E03B7D0026984200D016B17B7E5B098A
:20FCE00005D23A4657F80C7C002FE5D123E00846394647F0A1FCF88A6760000A03D397F994
:20FD00001C0007F0F3FC387D022818BF052802D1012007F039F86068407E30F07F0005D1E7
:20FD200094F88B00401E84F88B0004E094F88A00401E84F88A003846D0BDC04610010020A7
:20FD400070B50546204C1F48A1680068401A4FF47A7141431D48006800680E0C8047216943
:20FD6000401A48BF404240F6B831AD19A94211D306280FDAA268E1688A420BD8206848B152
:20FD8000891A134A51438A0C02EB1141884288BF011C08E00F49486840080ED208687D21A6
:20FDA00000F0FF004143C82905D3B1F57A6F88BF4FF47A6103E0C82101E04FF4FA6108467A
:20FDC00070BDC0463020094060350020EC01001040420F00AC4F0050BCB504460920207550
:20FDE00060680D461112401E00F8011906AF00F8012939781D4A00F80119B2F85614091225
:20FE000000F8011992F8561400F80119191200F8011900F80139411C2162217D491E017005
:20FE20006168091ACBB260602189287AC9180328218114BF0020012002F2CD110B22E0822A
:20FE400004F1840047F002FD0020032120654FF6FF73A0652A4600902046F2F709FA071CF9
:20FE600002D12046FDF756FA3846BCBD10010020B0B50446227D012A05D0152A03D0252A2E
:20FE800018BF352A17D1207E000914D21C484E30007858B160781B2806D1012006F074FFD8
:20FEA0004FF4806007F050FD002060706178204600F0EEF9B0BD1148237E4169DD0918D2F4
:20FEC000012A18BF152A01D119090BD267781B2F06D00C49002F0CBF1A312831895C02E057
:20FEE000232100E0312121700078214647F036FBB0BD09B160788847B0BDC0461001002042
:20FF0000700500201D9E01002DE9F843DFF88880054608F104000068804781461F4880300B
:20FF200004680027A7422CD0607E30F07F0024D062686B68501D591D52785B78C2F3810283
:20FF4000C3F38103934218D1022A05D0032A14D147F0DCFE064609E00A78037800269A4251
:20FF600004D149784078814208BF0126301C04D0607E274600F0BF00607654F80C4C002CC2
:20FF8000D2D11FB1787E40F0400078764046816848468847BDE8F883D8180020100100206D
:20FFA00030B5044660684078ADF1440DC0091FD31F4DB4F84200B5F85214884218D1A878A8
:20FFC000A0B995F85C0498B104F1280006F088FA70B9012000901C340194B5F8523405F214
:20FFE000424203210620F6F76BF91FE007F058F80BA80021182247F045FC02A821460C9069
:020000040001F9
:200000000BA8FEF747FA2C208DF82C000BA802F063FD08485038007810B19DF83C0028B13A
:2000200005208DF82C000BA8FDF74AFA11B030BD100100208E05002038B5054695F8300078
:20004000032839D195F83A00032835D105F128044A202146F4F73EFB8A202146F7F740F825
:200060006C686178207800EB0120ADF8000069465020F4F72FFBA41C6178207800EB012019
:20008000ADF8000069464B20F4F724FB8B206946F7F726F8A41CE1202146F4F71BFB641C88
:2000A0006178207800EB0120ADF8000069465320F4F710FB002000E0E82004492A240870EB
:2000C00028462C7002F008FD38BDC046FD0300202DE9F8432020EFF3118780F31188214C80
:2000E000A068012107F0BEFE4FF001094FF0000865692168A4F81C906A1A2168A4F81E80AD
:20010000461B401A904227D387F3118840462D18361A4846294607F0A1FEB042F7D9202194
:20012000EFF3118781F31188E18B012903D14046294607F093FEB0F1FF3F06D0A169801BF7
:20014000814238BF081C291801E0A069411907F081FEA4F820902560A4F81C8087F31188AA
:20016000BDE8F88318170020F8B50A46034621492148B1F84E70858891F809C08C6D86466C
:20018000ED18ADB25FB10020A41FA41DE67816B1A688B54208D07F1E00F10100F5D10CF1D3
:2001A0000100C0B2487206E04FF6FF7484421CBF002111701CD101201070B1F84C70BEF888
:2001C00004604C6D4A7AF01883B267B10020213C2134A67F1EB1B4F81F50AB4208D07F1EA6
:2001E00000F10100F4D1521CD0B248724FF6FF70F8BDC046C00E0020641E00202DE9F8434E
:20020000DFF87C900F4604464FF0FF31484607F030FBDFF870801D4800210AE0FF2A07D006
:200220000368934202D358F822600EB1002421E0491C1FB117F82120FE2AEFD100202060E6
:20024000012660600546A0600EE0FF290BD0636806FA01F048F8214018430B496060126835
:20026000204605F0EDFA6D1C27B107EB85021178FE29EAD1484607F03DFD2046BDE8F883B2
:200280001835002030320020007FC767A01E002090B50C46214A0178575CADF11C0D0B2FB5
:2002A0008DF8007034D0002F35D00C2F04D0112F28D147F0D7FA25E01A2C21D090F89D1050
:2002C0000190C7688DF80210038A0297C28AADF80C30510904D21249827E0978891A00E0E5
:2002E00000218DF80E10877F8DF8107090F91F308DF81130826A0592417F8DF80F1001E0C9
:20030000002001908DF801406846FDF7D9F802E04470FCF793FF07B090BDC0461D9E010012
:20032000700500202DE9F041224D044668680F46ADF1380D8047804609A98920F8F7C6FE85
:2003400081200CA98DF82C40F8F7C0FE0026344601E0641CE4B29DF83000A04204DCA9687A
:2003600040468847F32022E08DF800408DF80160D0206946F8F7AAFE0028EAD19DF80B00AF
:200380000128E6D10DF1020009A9092247F022FA0128DED18DF80C4003A9D320F8F796FE82
:2003A000A9680446404688470898386020460EB0BDE8F081D8180020F8B506460025204885
:2003C0001E4C0570204894F8AF24057094F8400318B1D4F88473616867B9012A02D0A078A9
:2003E000012801D000F0FAFF00F070FE3046F8F735F81AE0087D35280CD1012A04D14868C1
:20040000098900F0D3FC616848680088000901D305F01AFBD4F88413304688470948007832
:20042000012802D02846F2F779FF606810B1007D352801D006F0D6FFF8BDC0461001002007
:20044000B53500203D1F0020BD350020F8B5044642F209000DF1020103F0A2FD9DF80200A6
:2004600050B19DF8020002282FD1A08894F8271001F0AAFC064606E042F20D00694603F023
:200480008FFD9DF80060134D686880470F4B12490F4A1F780C390E701FB91778A9684FB9FC
:2004A00004E01778A96837F07F0703D1884702F0D3FB00E088470020A4F87C6094F8217044
:2004C000607017B1102007F047FAF8BD50040020BD350020D8180020381C00202DE9F04116
:2004E000804621483C3800680D46416927208847012404FA05F6194DC5F80064C5F87C47B9
:200500000327C5F8807716480460C5F88477D5F80404012818BFC5F80444C5F8FC63114834
:200520000460C5F800801023AB60204607F097FBD5F88C074008F8D3D5F88C17204611F0A3
:20054000404F09D1C5F884770021C5F8FC16D5F80024164218BF081CBDE8F08104400240AA
:2005600000E0484200004842EC0100102DE9F041804604200826ADF1180DADF80A001E4D4E
:20058000ADF808602968039602A8884700280CBF049F002747B398F80000C01CC0B20446CC
:2005A000801C05F071FE786050B9ADF800600520ADF802002968019768468847002713E0C9
:2005C0007868FE210170786822464146401CFFF7CFFA7D682146681C06F064FF6119487066
:2005E00000263E70A51C7D80404606F08DFA384606B0BDE8F081C046D81800202DE9F041BF
:200600001E4D804668680E468047A968074607F021FA70BBB6F5877FDCBF0021081C05DDB0
:20062000A6F5877008F587714FF48776144C616132464146E08004F59370FFF799FA0120CC
:200640001049A680A3680870581CA060686880470D4C8046324621696068668007F0A0FA2D
:20066000B0F1FF3F04BF00206080A96840468847A96838468847BDE8F081C046D8180020E8
:20068000481100203F1F0020601B00207CB5204C3C3CE06B0068014604208847022818D0B4
:2006A000032816D018480068C0F38150032814BF41F288324FF47A721648174C01684C3419
:2006C0002046B2FBF1F107F0F3FA204607F0F2FA7CBD20680D4E406803214FF040521C2300
:2006E0000546009100213046A8472068406801214FF4007209230446009100213046A0470C
:20070000022005F0B7F87CBDB44F005000A00C40E0010010A03500200C16002013460246D2
:2007200010B5803A132A3ED8DFE802F032302E2C2A2826243D3D211E1B19163D13100D0A5C
:200740004FF4803226E04FF4004223E04FF4806220E04FF400621DE04FF400521AE0082296
:2007600018E04FF4805215E04FF4007212E04FF480720FE040220DE080220BE0202209E0A5
:20078000102207E0042205E0012203E0022201E04FF48042044C2468224204D00A4601467A
:2007A0004220F8F7C1F810BD141F0020F8B50E463268916B054621F020019163286E317DC3
:2007C000012203F047FE286E317D012204F030FC286E317D002205F0FBFB286EB17D002200
:2007E00005F0F6FBA878012807D005F1CC004FF0FF3107F03EF8306803E030688169090986
:20080000FCD20D4C84420CBF10221422317D286E05F0DEFBB17D0027FF2902D0F07DFF28C3
:2008200000D13FB13068844214BF15221122286E05F0CEFBF8BDC04600100040F8B5054605
:2008400007F042FA1F4C064604F1340220681178A943117030B19C3007F026F8002700B16B
:20086000012700E00027606838B19C3007F01CF838434FF0000718BF012794F83400E0B9A8
:20088000012F1AD0A06AD8B1016A89080AD24569304607F01BFBA06A00214FF400030A46E1
:2008A000A84707E0C569304607F010FBA06A02210022A8470020A062F8BD304607F006FB39
:2008C000F8BDC0460033002070B506467468B568206E06F0B9FA29681C488A6B1040886344
:2008E000304600F037F8304601F002FE2968C86A20F01000C862296815480A6B10400863D1
:200900006868FDF713FB04F17C0007F0DBF904F1980007F0F1F9A07818B904F1CC0007F0BA
:20092000E7F9607818B904F1E80007F0E1F904F5827007F0B7F907F0C7F90021217007F08E
:20094000C5FA04F1680006F09FF970BD0DF8FFFFFEFCFFFF2DE9F04106467568B46807F042
:20096000B3F9A96A39B921688969090903D207F0ADFABDE8F0810027AF6207F0A7FAA17DC2
:200980003846FF2902D0E17DFF2900D118B128462146FFF70BFF2168886B20F02000886353
:2009A0002168086B20F48070086307F08DF90B4C8046207818B1022004F05CFF2770404643
:2009C00007F084FA696A286A2F696A6A401A2862296A3B4630469847BDE8F081B435002065
:2009E00038B50C4644220546002100F0F1FE04F12801284606F0AEFC04F1320105F10A00B3
:200A000006F0A8FCE06B6861B4F840002883B4F842006883B4F84400A88394F84600A877AC
:200A200094F84700E87794F9480085F8200094F8490085F82100B4F850006884E06C6862A1
:200A4000A07B85F8280094F8520085F82900606D0B2204F11C01E86205F13000FFF788F860
:200A60002089A5F840006068E86338BD38B504461F4800780D4601280FD004F10800690809
:200A800080B224BF04F12C0080B2122CCCBF14210621401880B2400028E0E920694603F04C
:200AA00061FE144890F87F04802801DD84280FDB04F10D00690880B224BF04F1260080B27F
:200AC000122CCCBF05210221401880B2C0000DE06001690800F5967080B224BF00F21E20BB
:200AE00080B2122CCCBF28210C21401880B238BDBF050020100100202DE978411C4C012099
:200B000020701C480078012814BF08200220DFF86880002103EA010502EA00068D4208BFC8
:200B200086420DD000214FF0E0401140184008BF002905D11249088C4546401C088404E0DB
:200B4000454695F90000401E287006F0EFFA06F049FC0A480026067095F9000018B93046A9
:200B6000F2F7DCFB01E095F900002670BDE878813D1F0020BF050020361E00202F1E0020D1
:200B8000481D00202DE9F04107461F49BE687C68306809688069C0F3C00018BB07F094F80F
:200BA0001A4D8046287820B1022004F063FE00202870404607F08AF93168886B20F02000AC
:200BC00088633168086B20F480700863206A616A2569626A401A2062216A2B4638469847CB
:200BE000BDE8F0814FF4FA70B0FBF1F1012998BF012104F58274204607F05AF8204607F007
:200C000059F8BDE8F081C046A0350020B4350020B0B504680D4617464FF0FF3104F148003C
:200C200006F027FE28464FF0FF35092808D0227A01218140114211D111430546217210E0D9
:200C4000227A0721012303FA01F0104202D0491EF9D503E0227A0D4610432072B5F1FF3FCA
:200C600015D0A7B1062005F06BF829463846FFF735FC0746062004F0FDFD47B1217A012090
:200C8000A8404FF0FF3580F0FF000840207204F1480007F02FF82846B0BD7CB515460E469A
:200CA000044600E024182046694604F09DFF00282DD014F8021F8E42F4D1491E04F10104E1
:200CC0001FD0491E12D0491E08D0491E18BF622027D102281BD12078287021E0032816D18C
:200CE00014F8010B28702078687019E007280ED161782078042240EA01202880A11C281D41
:200D00000CE0052803D120780628287001DD67207CBD281D002103220160611C46F096FDB8
:200D200000207CBDF8B51F4CA0F5C060D4F8B810C4F8D4000029B8BF49420028B8BF40421D
:200D400081422BDA4FF08057D7F8A401B4F8BC10154D40684FF47F42082306460091284645
:200D60003021B047D7F8A401B4F8C01040684FF4F80212230646009104212846B047D7F8EB
:200D8000A401B4F8D01040684FF440620A230646009120212846B047012000E0002084F848
:200DA000D800F8BD0416002000A00C40C8B50F46082F0BDA002F3CD001787F1E91FAA1F124
:200DC0004FEA216100F8011BF6D1C8BD414201F003017F1A4618BBB2864203F0030200EB71
:200DE000010709D9361A0178761E91FAA1F14FEA216100F8011BF6D123F003017F18874282
:200E00000AD9391AC91C8E100168761E91FAA1F109BA40F8041BF7D1BF18874209D93F1A42
:200E200001787F1E91FAA1F14FEA216100F8011BF6D1C8BD2DE9B84106F046FF1E4C1C4D47
:200E4000804604F1E000007848B9A8680146022088470746102003F095FD1FB31EE001F073
:200E600077FA78B9134800683221B1FBF0F101B9012104F1300006F01BFF04F1300006F001
:200E800019FF0FE0A8680022014684F8E020022088470746102003F075FD1FB1A86801465C
:200EA00003208847404607F011F8BDE8B881C046C8AB0100A0350020041600203EB51C4DD7
:200EC00005F5A8710878012464F30000087005F5A871087864F38200087005F5A871087814
:200EE00064F30410087005F5A871087864F3861008701048022205F5A871047042F20200DE
:200F0000ADF800000DF1020046F0A0FC01A8224605F5A97146F09AFCB5F83A01022806D180
:200F200006480068044D426A2868694690473EBD7C1300207C1E0020381C00204018002098
:200F40000146F8B501F01E0201F01F00162AA4BF01F01F002038184E317801F01F01162912
:200F6000A8BF2039814225D0144F3B68144A23F010031C0A14D323F08004A2F108053C608F
:200F80002C680DE014688142B4BF01244FF0FF340919347801F01F0504F0E00425433570BF
:200FA0008842EFD11068180A04D3106810683B6052F8080CF8BDC046066208402800094071
:200FC0003420094010B51E4C207840B91D481A494FF47A726538FEF7CBFD012020704FF073
:200FE0000451012481F82644022381F8DA33032281F8FE23042481F8B443052381F80034BD
:20100000062281F8E323002081F8EC03072481F8E143082381F80134092281F802240A2408
:2010200081F8DE430B2381F8DF330C2281F8DD23024CC1F8884410BDC87F0100ED4200217E
:201040001C1A0020894000212DE9F8431D4C1948676806F041FC1849054608680E6800F0B1
:201060002000284006F4602614D09FB107F1180191E80003A760044600201837210040EA9C
:20108000080041EA090187E803000F484FF4005106F038FE16EA05000AD0084A92F8491076
:2010A00041EA504082F849000548002106F02AFEBDE8F88320000E000C100440B032002076
:2010C000A0330020343500206C3300209EB5194C606880472146184C2289E388934225D0E3
:2010E000164B1F7817BB164B89681F7837F07F071DD1E28088471023124FE088ADF80030A0
:2011000001A9ADF804003A7809880DF1020739800D48012A18BFC838BDF804100B4F01807E
:201120003868426AE068694690479EBD896888479EBDC046D81800202C1C0020BB35002091
:20114000BD350020BF0500207614002040180020F8B50546012004F03DF81D4C04F5F27071
:2011600000F07CF904F5FA7000F078F969684A78087800EB0220ADF800008F7804F5F27619
:201180006FB953206946F3F7A5FA05F128014A20F3F7A0FA05F128018A20F5F7A1FF06F123
:2011A000200005F11C010B2246F050FBBDF80010384604F0C7FB94F80F02800803D368787A
:2011C000002106F0F7F8002084F80F02F8BDC046100100202DE9FE430646307A02281CBF1E
:2011E000B14608240DD130880F128DF80A100DF108098DF8080004248DF80B7000128DF81B
:20120000090000254FF00108124F307A024606F081FA08FA05F1084216D0A7F16C01022A3B
:2012200019BF01EBC501903101EB850174316846224646F00BFB48466946224646F0CAFA5B
:20124000012808BF281C03D06D1C052DDDDBFF20BDE8FE838C1800202DE9D841074606F099
:2012600033FD80468FB3B87A78B397F9091005F0ABFD0123064603FA01F05FFA80FC46B169
:20128000144C226811318B409A432260D94344F8041C00221146B97239723960796007F1C7
:2012A000100686E806000C49FA6001F1480291F84A7013781843107027B191F84A00401E07
:2012C00081F84A00604604F027FC404606F0FEFDBDE8D8810C100440B03200202DE9F84366
:2012E0001D4C606817468047A0461A4C81462FB904F108052A6800260C351BE02188E368B4
:20130000002604F114053046B1F5877F09DA2A5C5A542E544A1C401C91B2C0B287422180FD
:20132000F2D8A268B84205D042B161884FF487709047A26812B1B8B231469047268060682A
:201340002946202206F027FCD8F8081048468847BDE8F883601B0020D818002070B5044644
:20136000207C0125ADF1280DC00820D3B4F8421004F128000646FEF723FAC0B91648007855
:20138000012813D004F11C0106A80B2246F05EFA06F004F801463020009006AB0193B4F8BC
:2013A000423032462846F4F78BFF00E0002510208DF8080004F128010DF10A0046F0B4FC92
:2013C0008DF81650B4F84200ADF8140002A8FCF777F80AB070BDC0466A1E00202DE9B841CB
:2013E0001848194C05786068804780461748007818BB1749DFF85CC0012D0AD00F780120A9
:2014000037F07F0713D161460F7837F07F070ED10CE00F78012037F07F0708D10E490F7889
:201420002FB961460F7837F07F0700D1002080F00100C0B208B105F097FCA1684046884776
:20144000BDE8B881BF050020D8180020BA350020B9350020BD350020BB35002070B504460C
:201460001D480078012802D00120F1F757FF194D281D006880471349064620460B462831A3
:2014800005F01EFD20B903F12C01204605F018FD986BA04212D10C4C94F9000010F1020F13
:2014A0000AD00B48094B006894F90010826B186890476FF00100207002F0C4F8A96830463D
:2014C000884770BD100100202D1E0020381C002040180020D81800203D1F00202DE9F843AB
:2014E0008146EFF31188202080F311880124164E164DF461164F6C60F86A016A142088471C
:20150000D9F81000810C14BF000C0420A861386802682321002090470E480068C6F88042CE
:2015200000280CBF211C03210B4807680FB141F00401286820F4E02040EA01402860346074
:2015400088F31188BDE8F8830000244300200940840100107CAC010080AC01002DE9F04155
:20156000054606F0B1FB194C0126804605F19C00A67006F0A1FB164FB7F91400B7F91610F3
:2015800088420ED1207802280BD01248007840B1404606F09BFC0720FFF750F906F094FB44
:2015A0008046B7F91400B7F91610884218BF85F8C26006D105F1780006F07EFB082004F0BB
:2015C000ABFA404606F082FCBDE8F081B0350020343500203433002090B504466078ADF13C
:2015E000140DF3282FD0DF282DD0E8282BD0DB2829D02046FCF762FD071C23D1607C08B33F
:2016000094F83400F0B912480078D8B904F112010920F9F739FEA8B102218DF80C104FF644
:20162000FF72ADF80420A77A0097238901A9FEF7D3FB0746F32F05D0DF2F03D0E82F18BF8C
:20164000DB2F03D16770204603F000FE05B090BD500400201D4938B5283991F8303301EB7C
:20166000E30595F8F142012203F0070302FA03F383F0FF03234085F8F13291F8EE3201F599
:201680003B70032B18D091F83433012B10D0022B08D0B1F82A138A409102A1EB821101F530
:2016A00070710EE0B1F82A239101A1EB820108E0B1F82A138A4001E091F861249102A1EB1E
:2016C00082111C3005F078FD38BDC046380100201A4898B5007802282CD0062828D00528CD
:2016E00005D0012827D9C11E012926D823E0144C94F8AF04012820D105F0DAFF21460028CC
:2017000009DD114A0F4B12781B689200B3FBF2F2801A48BF00204F7847B191F839140F296F
:2017200004D018B91C20FEF747FE98BD052002E0062000E00220F0F7AFFB98BD4A1D00209D
:2017400010010020FC130020701D00201A4970B50A684BF2F5214843040AC2F381400128F7
:2017600013D14FF08056D6F8E011D6F8EC018D6800688047A847D6F8E011C96888472111F2
:20178000C01000B2484304EBE0340D4901F1E500007830B90948006820F07F40241864087B
:2017A00002E0002081F8E50006480460210C41600126866070BDC046B44F0050102009403D
:2017C000041600207C600C40002213460A46194671B510F0030F0BD0002A82BF00F8011BEB
:2017E000B2F1010210F0030FF6D1002A08BF71BD11F0FF0141EA0121042A18D341EA014177
:20180000082A0FD30E46102A08D30C460D46B2F10F0312F00F0272C0103BFCD812F0080F74
:2018200018BF42C012F0040F18BF40F8041B12F0020F18BF20F8021B12F0010F18BF017013
:2018400071BD704710B58188ADF1200D1A2918BF27212CD1846820788DF80B00641C14F80B
:20186000010B8DF80C0014F8010B8DF80D0014F8010B21468DF816000DF10E0005F094FA78
:201880000834204646F0E9F9E31CADF8180013F8010C0DF11A0103F0AAFD6846194605F005
:2018A00053FC05490246182044F09EFCC1B2062005F080FF08B010BD5B7B010070B51B4E46
:2018C00096F839040F2828D096F86411FF2924D096F8660170B102290CD103F085FE054610
:2018E0001348D6F85C4196F830340178083113FB01F00FE003F078FED6F86051B6F8884032
:2019000096F858342D1A06EB43062D1BB6F82C4101F072F92D1B2D1A01D5002070BD4FF676
:20192000FF70A842C8BFA8B270BDC04610010020791E0020F8B51C49194BDFF868C00C31A0
:201940000C6893F8AF1401290BD1614693F8AD740A78002F0CBF2169616902EB82025218C1
:2019600000E0226914790021032501E0491CC9B28C42D8BF4FF6FF7010DD136811FB05F6DD
:201980009B1993F90070B842F0D1B3F801106046C01D018010688019B0F80100F8BDC046A7
:2019A000100100202D1C00203018002038B51C4C002084F8690194F8395494F84002401C87
:2019C000C0B2042884F8400224D0202003F002FC94F87B240F2A0AD094F86A0194F8391478
:2019E000814204DD154684F8390404F009FA04EB4501B1F82C5194F8393494F840124FF4C3
:201A0000707204F504709A40491C01FB152104F0C1FF38BD03F0B0FFFDF7F8FB38BDC046D9
:201A2000100100202DE9F84F8346894617467120114604F079FC81206946F7F747FB4FF013
:201A4000F308002507E0B8F1000F23D038686D1CEDB22C3038609DF80000A8421ADD386802
:201A6000066890F804A0002402E0641C0A36E4B2A245E8DD737A002B0CBF052009208145CD
:201A8000F3D14A463046594645F0A4FE0128ECD14FF000084046BDE8F88F70472DE9F8431F
:201AA0001A4C05460E46201D01681648007820B9002028603080BDE8F8838847DFF84880E6
:201AC000D8F804725FFA80F908F5DC7005F094FFD8F880214FF47A73410001EBC001B1FBE2
:201AE000F3F129605018B8F8781128608742318003D8C01B2860491C3180A168484688471C
:201B0000BDE8F88358100020C00E0020D818002070B5054605F098F8194CC0F5877081B2E6
:201B20006088A94229DDAEB23118B1F5877F0EDD0319C0F587711A1D8EB2C0F5877399B252
:201B4000104604F0E5F8AD1BAEB20020608000193146001D04F0DCF86088084D4FF4877248
:201B6000801980B290FBF2F15143401A02216080E869698106F09EF970BDFEE7580B0020DE
:201B8000F014002038B51B4C184A0023164994F8E200136020B3012817D0022807D00328F9
:201BA0001ED151F8350CFFF7BDF80B2016E051F8355C2846F6F780FF40F2FE50A84202D2EE
:201BC000C01CA842F1D2082008E051F8350CFFF7BDFD074800780028E7D0052084F8E40007
:201BE000F5F786F938BDC0463D400C403C500C40D6AB01000416002038B51B4C012094F821
:201C0000391494F8AF5484F869010F2927D06070202005F091FE1348012DC4F828020CD0F4
:201C200094F8391494F8405204EB4101B1F82C21691C5143490096310CE094F8391494F80C
:201C4000405204EB4101B1F82C21691C5143490001F2A32104F5087004F09CFE38BD03F0CB
:201C60008BFE38BDAD1901001001002010B58188ADF1200D202918BF27212AD180680446C0
:201C80000078002100B10121641C8DF8151014F8010B10228DF8140021466846FDF768FF5B
:201CA0001034204645F0C8FF231D049013F8010B19468DF816000A680DF1170422604B68D9
:201CC0006360087A207205496A46182044F08CFAC1B2382005F06EFD08B010BD51960000A6
:201CE0002DE9F047DFF86490DFF85CA0DFF86080054600264FF0FF30192734462860E0B28F
:201D000005F0DCFBB8B1837AABB1017A0126022915D04946DAF8002040690978D26811FB92
:201D2000072104F025F841462B680A68B0FBF2F0834288BF2860641C032CE0D301E000205A
:201D400028603046BDE8F0876C340020FA320020A03500201A491B48F8B52D2751F8202F09
:201D60004E6840F8202F8D684660CC6885600B69C4604E6903618D694661CC6985617F1E6A
:201D8000C461EBD1203151F8047B203040F8047B51F8046B40F8046B51F8045B40F8045BA4
:201DA00051F8044B40F8044B51F8043B40F8043B51F8042B40F8042B09680160F8BDC04699
:201DC00088870100E07F002130B504460D4642F20900ADF12C0D09A902F0E2F89DF82400A6
:201DE00008B342F20B000DF10E0102F0D9F800230094BDF80E00029300040190684602F0D5
:201E000025FE044604A942F2030002F0C9F804F02FFC024604A9B4FBF5F06843241AE0B29B
:201E200002F0D0FA06E042F20D0003A902F0B8F89DF80C000BB030BD70B51A4E96F8585461
:201E4000044608460021FEF711FE0F2D334615D093F8392493F86511AA4208D0491C6FF0BA
:201E60000F06A9408A01A2EB8102921907E0491CA9408A01A2EB8102A03A00E0002283F8F7
:201E80006441012C1CBFC3F86021C3F85C0107D1D3F83C144018C3F85C015218C3F8602138
:201EA00070BDC046100100202DE9F04107461748174C001D06786068804780461549A26810
:201EC000087886281CD1104D05F11E021088401C10808720087005F0F3FDA168404688478E
:201EE000082004F033FDE879B04207D127B90020FEF762FABDE8F0811B20F9E7E920F7E702
:201F000040469047BDE8F081481D0020FC330020D8180020BD3500202DE9FC470C46054662
:201F200045F094FD164F8146786816468047804603F0EAFA8246B2002146484645F08EFDE0
:201F4000504605F09FF802E02D1D241DADB23046411ECEB278B128466946042245F05EFD42
:201F600068462146042204F027FD0028ECD00548012141700170B96840468847BDE8FC87FB
:201F8000D8180020901E00202DE91E4142F2050001A902F005F842F20100694602F000F84E
:201FA0009DF8040010B3DFF848800099D8F88021E1B19DF80400904203D891420BD900206D
:201FC00002E09DF804100120891A642288F894014A43C8F8BC2108F5DC74204604F040F90D
:201FE000204601F027FE012088F89801BDE81E81C00E0020C8B50146184AC87AC8B9B2F866
:202000004E70906D4FB3801F801DC67826B1B1F81F2083889A4202D07F1EF5D1C8BD8A7F20
:20202000C270CA880280B1F81F208280097B8170C8BDB2F84C70506D7FB121382130867FB4
:202040004EB1B1F81F20B0F81F309A4203D1212245F0FCFBC8BD7F1EF0D1C8BDC00E00202D
:20206000012898B528D1164800680068014601208847012820D004F07FF9134C012104F191
:20208000D800017005F0ECFC800917D20D4800683222B2FBF0F707B90F46083C04F1300085
:2020A00005F00AFE04F13000394605F001FE04F1300005F0FFFD01E002F076FB002098BDBC
:2020C000E0010010A03500200C160020001F06B480B280B5082802AFADF1080D26DBB0F55E
:2020E000005F23DA00F18851091F0B686A46136049685160BDF80010CA0B10D33A7801F07A
:20210000FF018A420BD17988BDF80220914206D1B988BDF80420914208BF012007D0BDF834
:202120000610401A083880B20828D8DA002002B0BDE8804002B070471FB5014604208DF877
:20214000000048788DF80100B1F89A000DF10203ADF80C009031184605F08EF804F0C0F9FB
:20216000C0B14FF6FF7453200DF10E01ADF80E40F2F7B0FA0A4890F83914A0F84C440F29A9
:2021800008D00F2180F8391404F098FB03F0F4FB05F058F96846FBF793F900901FBDC04625
:2021A000100100202DE9F843DFF85C90044609EB440000F16805B0F86800884645F0D8FA15
:2021C000074612480678B7B12A883846002145F059FB00253C70494664187D70627D381D9B
:2021E000414645F033FB3046394645F0B7F940B92846BDE8F8838DF8004068461A21FEF7F1
:2022000047F81A20BDE8F883FC9D01001001002038B5194C94F8690194F8401294F8AF54A5
:2022200040B9606860B9012084F86901202005F083FB05E0481CC0B2042884F8400215D080
:20224000012D07D094F839244FF47071914001F2564106E094F839244FF47071914001F25A
:20226000636104F5087004F0A7FF38BD202002F0B1FFFCF7CBFF38BD100100201849194813
:20228000F8B51F2751F8202F4E6840F8202F8D684660CC6885600B69C4604E6903618D6919
:2022A0004661CC6985617F1EC461EBD1203151F8046B203040F8046B51F8045B40F8045B9F
:2022C00051F8044B40F8044B51F8043B40F8043B51F8042B40F8042B09680160F8BDC04674
:2022E00090830100E07F00212DE9F843174C04F1800007688046632037B300261D25397D61
:2023000035291CD140463946324645F095F9787E30F07F0005D194F88B00401E84F88B004B
:2023200004E094F88A00401E84F88A007D7057F80C9C3846FDF79CFD4F46002002E03E4635
:2023400057F80C7C002FDAD1BDE8F8831001002038B5144DD5F8600101680120884701287D
:202360001ED0D5F82401C4680F483C2101220023A047002808BF002013D0286880470B48D4
:202380000C4A0B4D016893681068D160A0EB9000C91A05FB01F3190C814228BF081C10602D
:2023A000012038BD8000001000A00C403020094040420F006035002038B5124D00242046D6
:2023C000AC800146AC6105F041FD28612046014605F03CFD686102F095FD0C480A490C4C9A
:2023E0000860606880470C4905460A48C1600B490161FDF7D3FAA16828468847F0F704FE2D
:2024000038BDC046580B00205C1E0020D5320100D81800204811002009680100111B010074
:2024200070B505F051FC01461348007802281AD0084605F04BFD11480068006B8047104A2F
:20244000002305F053F80F4A12684FF090557A2600232D184FEA020446EB0106ED1846EB6D
:202460000406341C05E005F037FB0446084605F02DFD204670BDC046B03500208C01001004
:2024800000093D0084350020F8B50D46044605F01BFC0646E8B205F011F88025071C1ED02D
:2024A000B87AE0B110480078022806D03846FEF7D3FE00F049FD832511E097F909000B4989
:2024C0004FF4A06202EB002202F47F4220461143002203F03BFB05463846FEF7BDFE3046FD
:2024E00005F0F4FC2846F8BDB035002001000804F8B50646B1680A687568906B20F4FA60F8
:2025000090630968086B20F40070086305F0DCFB104C0746207820B1022003F0ABF900203E
:202520002070384605F0D2FC05F0CEFBA96B11B905F0CCFCF8BD0021A96305F0C7FC696B03
:20254000286BEF686A6B401A2863296B3B4630469847F8BDB3350020F8B5844640F6FF7490
:202560001CF8013B002210E0481B401E10F8015B7F1E01F8015BF9D103E01CF8010B01F81C
:20258000010B521C5B08082AEADA5808F5D21CF8010B1CF8015B05F00F07FF1CC5F30315BB
:2025A000122F45EA001508D11CF8016B300A24BF1CF8010B60F3DF16BF19AC42D4D1F8BD98
:2025C00010B58188ADF1200D182918BF272123D1846820788DF81400641C03A8214604F06B
:2025E000E3FB0834204645F038FBADF81600A11C11F8010B8DF8180011F8010B002200B1E1
:20260000012268468DF8192004F09EFD05496A46182043F0E9FDC1B2072005F0CBF808B043
:2026200010BDC0466F7B01002DE9F0410446A56E1F461646884605B1A84704F1600003C8E4
:2026400006400F4008BF002E1FD041462046802202F066FD04F1700181E8C00078B104F170
:20266000700191E8600000F1180797E8060000F11803B243A94383E80600A16E416000204D
:20268000A06604F1400005F035FBBDE8F08170470246F8B5084611464C68203822D0401E17
:2026A0001DD0401E18BF6FF001001FD18D6805F00BFB0F4E07463068006901462868884767
:2026C000B0F1FF3FF7D100256564E564206CA563401EA064384605F0F9FB2846F8BD00217B
:2026E000084601E00121002084F82D10F8BDC046D001001010B54FF0FF3004F0B1FF0446F3
:202700000E480F49006881420ED10E480E49002205F0E0FA0D490220087003F0C5F818B9F2
:2027200001F094FDFCF770FB0948204204D009484FF0005105F0E6FA10BDC04684340020D1
:2027400085290000C434002095930000B0350020020000406C3300201FB5044694F89A0041
:2027600038B304F18F0101A845F0E8FA03208DF80C00114890F86F140091B4F89820B0F874
:20278000523401A92046FDF727FB0146DC290DD0DD290BD0E42909D0F32907D0DE2905D0CE
:2027A000DF2903D0E82918BFDB2902D12046FDF76FFD00901FBDC0461001002010B5044607
:2027C000012002F007FD208900280CBFEB2000201249607091F80F02C20824BF20F0040095
:2027E00081F80F02820809D2400813D32B202070EB236370204600F06FF90BE091F80F02BD
:2028000000F0FD0081F80F02217C6078C1F3001104F0D0FD204603F0C9F810BD100100202E
:202820000146124810B50078E0B911480278134B4068920001FB0204A3F110000068C06B7D
:202840008047211AA1F54871090806D3094A011B891A090828BF00F5487409482146F9F7DA
:202860003FFE10BD04490120087010BD3E1F0020701D002000093D00BC3500205018002092
:2028800059F3000030B5174C054605F12801ADF1140D04F2424045F023FA08B3EF230920BB
:2028A0008DF801306B688DF800005A781978181D01EB0221ADF802102A890178082A8DF8C9
:2028C000041014BF94F87E04C07805F11C018DF805000DF1070005F0DDF96846FAF7F0FDD2
:2028E00005B030BD1001002010B504460320ADF1180D04F128018DF8020000208DF80300C3
:2029000001A845F01BFA6068007804F11C018DF80C000DF10D0005F0BDF904F1280003F01B
:20292000DFFD58B14FF6FF7453206946ADF80040F1F7D0FE044920460A3108800DF10200C7
:20294000FAF7BEFD06B010BD5205002070B5134E706918B106F1140005F0DAF9134C6068AF
:202960008047316A0A680025157109683162A16888470B4A0B49107810B90846007858B133
:20298000157008460570FBF7FDFB07480078012802D02846F0F7C2FC70BDC046FC330020AE
:2029A000B9350020BB3500203D1F0020D81800202DE9FC41144EADF80400706880478046AA
:2029C0006946722003F0B0FC104D114F298800240FE0009AE00000EB0410801803883A8838
:2029E0009A4204D101A9022244F030FF2988641CA4B2A142EDDC502001A9F1F76BFEB1683E
:202A000040468847BDE8FC81D8180020681E00206205002030B50446606800252062ADF1C6
:202A2000140DA5657820A4F84C0094F82C0025650F2807D004F12C0120460122F6F7C8F942
:202A400008B116E0284694F83C10FF2901D1A16D21B104F13C012046FBF704F848B92B46AF
:202A600001208DF80C30032101AA00902046EFF7FFFB05B030BD70471CB5154C6368191C44
:202A800025D0207888B1FF2803DA401EC0B220700870628847201021F5F746FF207820B178
:202AA00004F10C0045F018F91CBD04F10C0045F015F908210523074AADF800106068ADF8EE
:202AC00002301168019068468847002060601CBD5C1C0020D8180020F8B5164B93F85E10D5
:202AE00003EB8101D1F8B440017801F07F014A000170A5181219527803EB8206D6F8B470EA
:202B000027B183F85E20017804EB41052A78141103EB8403D3F86C712FB90C2909DA182119
:202B2000FDF7B6FBF8BD02F00F0257F8221001B18847F8BD1001002038B50546FDF7E4F947
:202B4000134CE0698047012812BFB4F85A04B4F85A04401C688294F88A0068B994F83904B2
:202B60000F2809D104F5DC752846FEF777FC4FF47071284604F020FB064D6868804794F80D
:202B80008A10491C84F88A10A968884738BDC04610010020D81800200146114810B5007827
:202BA000D0B910480278104B4068920001FB02041868C06B8047211AA1F54871090806D33D
:202BC0000A4A011B891A090828BF00F5487408482146F9F785FC10BD06490120087010BD8F
:202BE0003E1F0020701D00204018002000093D009DAB0000BC35002070B5134D11496878D5
:202C00000C880830444312480068104EC06B80477168401A31788900B0FBF1F10D4802788E
:202C20003C209040B1FBF0F242436878891A00F10803B1FBF3F25A43891A401A001908305A
:202C400070BDC046521D0020781E0020701D002040180020680500201549124838B50C4653
:202C600000786068804721460F4D124CEA780C3C23789A4206D10D4A89681278D20802D2B4
:202C800088470AE08968884704F06EF82078FBF71BF8012804BF2078E87004F0A3FB012035
:202CA00038BDC046BD350020781E0020BA350020D8180020381C002038B5164C04F53B70CB
:202CC00005461C30FEF7CAFB02F066FA042003F03DFE94F8EE02032802D194F8ED02A0B1B9
:202CE00005F14501E120F1F7F5FC05F14601E720F1F7F0FC94F87F0494F83313884204D027
:202D000005F14701E820F1F7E5FC2846FAF7D8FB38BDC046100100202DE9F8431D46164636
:202D20008946804604F0D0FF044600F0DDFE07462946424648469FB138723A600C48786094
:202D4000384600F0FBFEF86006B17E600949086808B93868086000F0F7F897F9095001E0EB
:202D60006FF00105204605F0B1F82846BDE8F883FFD700006C34002038B5044642F2080053
:202D80000DF1020101F00CF99DF8020040B19DF8020002281ED1204602F00CFB054606E074
:202DA00042F20C00694601F0FBF89DF8005094F8200068B9284601F0B9FB0020A4F87C50F3
:202DC00094F8223020702BB1102004F0C5FD38BD0120207038BD704770B5F9F797FFEEF7E1
:202DE0004FFE124D68688047064603F09DFF104C94F96E0404F07AFC01F0BCFB03F098FBC2
:202E000003F0AAFB02F0D4FBA9683046884794F86F0401F08BFB04F255415220F1F75AFC51
:202E200004F048FE08B900F019F970BDD81800201001002070B50C4620B141680122A24031
:202E4000114201D1022070BD0D4E104B914300254160305D43F82450FF2804D009490968B4
:202E600051F8201001E044F020410748F9F7C0FF20464FF0FF3104F0CDF8284670BDC04636
:202E8000483400201C300020007FC767303200201548134A1349E4300078801E0A2807D8AA
:202EA000DFE800F019140F06140F06140F0607C0FEE710688008FCD250688008FCD2F4F754
:202EC00017B808688008FCD3F4F712B808688008FCD2F4F70DB810688008FCD3F4F708B8B7
:202EE00054600C4058600C40041600203EB5401E4FF000040AD0401E04D0401E1CD1F3F7BF
:202F0000F7FF19E000F012FA044615E0684604F082FE01940B4D8DF80040084902940122A9
:202F20006B4605F1780001F029FA054A2C21234605F19C0001F08AFF20463EBD912E01002C
:202F4000851B01000416002013481CB5007802281ED001281FD004281DD004F0B5FE0446B8
:202F6000684602F0B5FA00280C480BD0009931B904F0A2FE0A48042104F0C4FE04E004F08F
:202F800008FB01E004F098FE204604F09FFF1CBD192004F09DFE1CBDB035002024340020D4
:202FA0006C33002070B51348134D06782868ADF1200DA0B1002444F0FDFC0DEB04020021D8
:202FC000CB00491C20FA03F3042902F8013BF7DB241DE4B2202CEEDB296868468847022E52
:202FE00006D1064991F8500140F0040081F8500108B070BDBF050020101F00207C1300200C
:2030000010B50446012002F0E5F81248FEF726FA208900280CBFEB2000200F49607091F8CA
:203020000F02C20824BF00F0FB0081F80F0280080BD391F80F0200F0FD0081F80F02217C49
:203040006078C1F3001104F0B5F9204602F0AEFC10BDC046F40200201001002038B5104CCC
:203060004FF470000025E0600F48A56000686560C06B80470B49C0F1FF3008600B49C8689D
:20308000657008B90A48C8600A480570012001F03DFD0F2002F0B4FEE068FFF77DFD38BD8D
:2030A000701D00200830044040180020FC1B002095350100BC350020DFF854C08CB5FF2011
:2030C0009CF867119CF88B708CF86401012908D09CF839049CF85814884217D003F064FA97
:2030E0008CBD00218CF8671187B19CF86F148DF803009CF87E748DF800109CF87F148DF8CC
:20310000017068468DF8021004F065FD8CBDC046100100201449154898B53C2751F8202F21
:203120004C6840F8202F8B684460CC6883600B69C4604C6903618B694461CC6983617F1EA6
:20314000C461EBD1203151F8044B203040F8044B51F8043B40F8043B51F8042B40F8042BF0
:203160000968016098BDC046448D0100E07F0021154909681F280ADC1F2819D00D380FD080
:203180000A380FD0001F0FD0C01E0FD01AE0253810D0001F10D0401E10D0801E10D011E070
:2031A000086870474868704788687047C8687047086970474869704788697047C8697047D3
:2031C000086A7047002070474817002070B5124C6068F8B1124D68688047064694F88B2003
:2031E0000E4861680078904206DCA96830468847F120F5F733F970BD04F1800044F0FAFA3B
:20320000002394F88B00A9686360401C84F88B003046884770BDC04610010020641E0020F2
:20322000D8180020F8B5134C60680D468047124A8446A168B2F84C70506DB7B10024213859
:203240002130867F6EB1B0F81F20954209D1002282774FF6FF72A0F81F20604688472046DE
:20326000F8BD7F1E04F10104EAD1604688474FF6FF70F8BDD8180020C00E0020F8B5074671
:20328000C81D01F00705C610002F4FF0010000FA05F0A0F1010C14BF0029002019D0002055
:2032A000BEB17F1E3346024617F8011F941BB4F1FF3F08D10DB10CEA010104E001F1FF0418
:2032C000401C2140C0B20029F8D15B1E02F10102EAD1F8BDF8B5054616460C460C2003F029
:2032E0000FF80746082003F00BF8DFB1D0B144604580B86076B900210B4C0170606939466A
:2033000004F0DCFDA08840F00800A080E06904F0D1FDF8BD03F0E8FB384603F0E5FB204613
:2033200003F002FCF8BDC046580B002038B5134D95F8E100002410B91148007860B104F0E0
:20334000C3FC95F8E310002906BF012185F8E310012404F0BBFD0CB1002038BD022002F0F7
:20336000EFFC0E20FAF772FF03F084FA01280EBF0120002085F8E20038BDC0460416002096
:20338000D6AB01004EF68851CEF2000108684FF0F00340EA034008600C4885460C4885441A
:2033A0006F4607208743BD460A486F4607600A48002803D07946491D8E460047FCF710F96D
:2033C00004F088F804F03EFDFEE7C046003B0120000500002C1F0020457B010038B5FF20C6
:2033E000124D134C85F86401201D006880470346D5F88000014650B14A7E32F07F001CBF9F
:2034000002F0EF024A7651F80C1C0029F4D1A1681846884795F8390495F85814884201D016
:2034200003F0C2F8082004F097FA38BD10010020D818002070B50546124C687E94F8AF64A9
:2034400000F0EF0068762846FCF75EFD294604F1800044F0CFF9022E02D12846F7F740F97B
:20346000094D6868804704F18A021178491C1170A968884794F839040F2802D1082004F0A0
:203480006BFA70BD10010020D818002000B58188ADF11C0D162918BF27211CD181680DF1A2
:2034A0000B000B4604F0F4FA0833184644F0D5FBADF81400991C11F8010B002200B10122B8
:2034C00068468DF8162003F03FFE05496A46182042F08AFEC1B2512004F06CF907B000BDB2
:2034E000797B010070B51048104C007860688047104E0F4DF1782A78914207D10E4AA16826
:203500001278D20803D28847012070BDA168884703F02AFC2878FAF7D7FB012804BF287875
:20352000F07003F05FFF70BDBD350020D81800202C1C0020781E0020BA35002002461148BD
:2035400008B5007801281CBF0F48027018D10F4890F87F0402F024FC4168006802FB0103FA
:203560000B4A4FF47A70B3FBF0F189B200FB1130A2F85E1040037D23B0FBF3F0A2F8600050
:2035800008BDC046BF050020C2140020100100207C13002070B5124C606880471149002515
:2035A000064648784D70A168820807D2C00814D3304688472846EFF7B1FE70BD304688476D
:2035C00009480078012802D00120EFF7A7FE606880470646FAF744F8A1683046884770BDF8
:2035E000D8180020701D00203D1F00202DE9F041054600202860114800780E46012802D038
:203600000120EFF78BFE0E4C606880473768804630463FB16A687968914203DC38463F68DC
:20362000002FF8D1056030682F60854201D100F009F8A16840468847BDE8F0813D1F00208C
:20364000D8180020B0B5144C00252846A26A216BA56390420CD05268914209DD01F0C4FF8D
:203660000146A06A42689142C8BF4160A063216BE76A37B118B142687B689A4201DD3846FE
:20368000A06328B14068814202DD01F0C9FFB0BD03F06EF9A563B0BD1001002070B505466E
:2036A000114808260623ADF1180D0278104CADF808600E48ADF80A3001788DF80C20686885
:2036C0008DF80E1000218DF810102168059002A88847ADF800600520ADF8020021680195FA
:2036E0006846884706B070BD580B0020181E0020D818002038B501460C684D682068002874
:2037000008BF4FF0FF301FD004F0DEFA2168002954BF491E0021216004F0D8FB206890B953
:2037200004F12C0004F0CEFA04F1480004F0E0FA04F1640004F0DCFA6868FAF7F7FB04F1D6
:20374000180003F0A1FA002038BDFEE738B5134C054694F8201094F8230081421DDD94F87E
:203760002110A94219DD636A3BB1294604F5BA72984794F8230094F8211084F8220010FBF6
:203780000151E06901EB81010918087884F82300D1F8011004F5BA70884738BDC00E002031
:2037A000C8B5064611484768FFB1416891F82F1049091AD30768C7B1016891F82F1049096E
:2037C00013D201684268C968D26891420DD1371C06D07F1E09D14168C16000274760C8BD18
:2037E00003484FF4004104F08DFAC8BD343500206C3300202DE9F041124E8046706A3546F0
:203800000746A0B1687D00240AE057F824302BB1184603F049F906F115000078641CE4B26B
:20382000A042F2DC384603F03FF90020686205F11C004246202102F0A7FC04202875BDE86F
:20384000F081C046D4330020B0B5054610480768C7B1B968087B012400F00F00022818BF12
:20386000002011D1F8680B4AC36812788868192712FB073102F07CFA074928600968B0FB0B
:20388000F1F001E00020044628602046B0BDC04634350020FA320020A0350020084608B5C6
:2038A00000F0005100F00400084316D00B4800680068014601208847012808D0084800688F
:2038C0003221B1FBF0F1074803F063FE08BD064804F0AEF8054804F04FF808BDE00100107A
:2038E000A0350020243400208529000074350020134910B5044691F80F02ADF1180D40F0EC
:20390000020081F80F02012003F03EFA607890B9211D02A803F0B0FC03F040FD014601208F
:20392000009004F110030193E38902AA0520F2F7C7FC607010B1002103F03CFD06B010BD11
:203940001001002000B58188ADF11C0D162918BF272119D181680DF10B000B4604F098F8A2
:203960000833184644F079F9ADF81400991C11F8010B8DF81600684603F0E6FB05496A466A
:20398000182042F031FCC1B2502003F013FF07B000BDC046657B010000B58188ADF1240DC0
:2039A0001E2918BF272119D1836818788DF80B005B1C13F8010B19468DF80C00684603F08D
:2039C000C3FB11220DF10D0003F10B01FCF7D0F8054918206A4642F007FCC1B2442003F0FB
:2039E000E9FE09B000BDC046837B010010B5124CD4F8E41281B1606850B961600020C4F8E0
:203A0000E4020220F2F73CFA022003F0BDF903E004F5397001F056FC607860B194F839043A
:203A2000D4F8E0120F2806D00448C4F8C80204F5307002F0AFFF10BD10010020B53E0100BE
:203A4000F8B506460F48104C0578201D006880470746012D06D10A49087820F00F0040F05D
:203A60000100087009480068094D8369286832464FF0FF319847A16838468847F8BDC0466B
:203A8000F1130020BF050020D818002040180020381C002010B5044600211C22ADF1200DE9
:203AA0006846FDF795FE60788DF80000A0788DF80100E0788DF8020020791122611D8DF828
:203AC000030001A8FCF754F8A07D8DF8150008B1A06906900348006881696846884708B01A
:203AE00010BDC046201E00202DE9F041DFF8488098F848600025012404FA05F31E4215D0F2
:203B0000E8B203F0DBFC88B1877A7FB998F84A1098F84820457283F0FF038472491C88F8E6
:203B20004A10134088F84830BDE8F0816D1C032DE2D30020BDE8F081B032002010B5027AE3
:203B4000012A17D0022A18BF00201DD190F909300E484FF4A06221F470614FF6FC7402EB5D
:203B6000032202F470620A4342F4005204EA0201084310BD0A2490F90930416100F11002E5
:203B800004825B1D1046937010BDC04601000306F8B504460D4608461122002143F072FE62
:203BA00094F800C0BCF1000F1AD0641C00214FF0010EE078A37843EA0023207809E0C6100A
:203BC000AF5D00F00702401C0EFA02F2C0B23A43AA558342F3DA491C241DC9B28C45E8DC52
:203BE000F8BD80B502465378107840EA0320C7130F7007BFC0F3062300F0FF00C0F3C32370
:203C0000C0F30A004B70802848800DDA02280BDB012B0CD0022B0AD0042B08D0052B06D0A9
:203C2000062B04D0072B02D00022104600E0921C4A6080BD2DE9B841114C0546201D006832
:203C40008047804602F090FF6F7E0146002F08BF686806D068682A69AF68401A8018C01941
:203C600068602961E96805F1140201F09BFD012768686F76A168A86040468847BDE8B881EB
:203C8000D8180020114810B50078F0B1104C233C94F82A12642011FB00F0C4F8A00104F584
:203CA000CE70FFF7C7FFB4F8760194F82A22D4F87C11401C80B28918A4F8760100B900219A
:203CC0000020C4F87C11FFF741FD10BD65050020E30E002038B504460F4910481430098823
:203CE0000068A14213DD0E4D6868804703466946722002F019FB0099E00000EB041009186E
:203D00000091A968184688470098001D38BD641AA1B200EBC10038BD681E0020C00E002024
:203D2000D818002070B5114C0025DD214FF43C7204F17806ADF1400D3046E560FDF748FD8B
:203D40003C2208236846294604F098F84FF43C70074908906A462B4607960220069004F1F7
:203D6000280004F087F810B070BDC046580B0020E97C0100042810B51AD10E4C204603F03D
:203D800093FDA8B1204603F091FF0B4909684843B0F5967F0CD2204603F08EFF052001F06D
:203DA000CFFF0649012008700548042103F0AAFF002010BD24340020A03500208134002010
:203DC0006C33002038B5104C114D607838B90F492846F4226538FBF7CBFE012060704FF050
:203DE0000451C1F88854002081F8CD03012481F8B443022381F80134032281F8022404251B
:203E000081F8DE5338BDC0461C1A0020D47E01008940002110B5114C22685168496839B16A
:203E200010B1F6F724FE226850684068804722685168886808B9C86878B103F093FC2168A9
:203E40004868806808B1804721684868C06800B180470348503802F0C5FC10BD6C3400205E
:203E60005100070610B50446012001F0B3F92078212804BFEB2060700D4991F80F02C208DE
:203E800024BF20F0040081F80F02800805D22B2020702046FEF720FE10BD91F80F0200F097
:203EA000FD0081F80F026078002103F083FA10BD1001002010B5114C6078D4F8E012E0B1CB
:203EC0000F484031C4F8B80204F52C7002F062FD03F02AFC48B9F3F7F9F9C4F8E40260B115
:203EE000017E41F04001017610BD002394F84004C4F8E432401C84F8400410BD10010020AE
:203F0000ED39010010B58188ADF1180D162918BF272118D1846820788DF80800641C684663
:203F2000214602F041FF0834204643F096FEADF80A00A11C03A803F007F905496A4618203F
:203F400042F052F9C1B20D2003F034FC06B010BDC77B01000146104808B500784FF4C8522A
:203F6000802803DD8428B8BF4FF41642052909D001F016FF0949C07B0988022814BF02F5DC
:203F80007A720A4402F57A624FF47A6002F5FA62B2FBF0F008BDC0468F050020B6100020B2
:203FA000F8B50E4602F0B8FF05464FF6FF70A84208BF682013D00C4C606880470849094AB1
:203FC0000746680000EBC5004018017889184278304643F03BFCA168384688470020F8BD45
:203FE000E0A50100BC100020D8180020014608B5D0381DD0401E19D0401E15D0401E11D07D
:20400000401E0DD0401E09D0084603F03BFCFF280EBF0020074911F8200008BD052008BD7A
:204020001C2008BD182008BD042008BD082008BD0C2008BD7D9E01001FB5044620788DF864
:204040000000607861688DF801000DF1020043F0D6FD218943F0FBFDA17A00F8011BE17AD4
:2040600000F8011B217B00F8011B617B00F8011B216943F0C4FD842010216A46FCF74EFB4D
:2040800000901FBD80B502F09BFF01460F4802680429C2F340674FF0FF3016D1C2F3033124
:2040A000083911D0491E0AD0891F0ED1100E04D3900E2CBF0E200D2080BD0B2080BD002F69
:2040C00014BF0A20092080BD0C2080BD94120050F8B516460C46054603F0F6FD2B461F689A
:2040E00084460022214630460A6027B9196008B1012101700CE008B11446047000E03F68EE
:2041000038680028FBD1B94208BF141C01D039600124604603F0DAFE2046F8BD00B5002128
:20412000ADF12C0DADF800108188022918BF272007D1806843F091FD6A460DF1030101F07D
:2041400077FE8DF80200002806BFBDF80000401C0120ADF80000BDF800100DF10202422076
:2041600003F0C6FC0BB000BD38B50F49104C888B401C88836068804705460C4801788629A1
:2041800003D0A1682846884738BD8721017003F097FCA16828468847082002F0D7FBE92037
:2041A000FCF70AF938BDC046481D0020BD350020D818002098B5024650684178CF111ED093
:2041C0001389D06400214478C4F3C3040F2C08D0047809190019891C801C89B28B42F2DCD3
:2041E00001E0891C89B28B4206DB5068178940185060781A108100E00021A2F8501098BD7D
:2042000080B507468020EFB1B97A01291AD197F909000D4A0121113001FA00F0C34342F816
:20422000043C13681843106097F909008140C8B202F0D0FFF868002101F0F6FE812804BF91
:204240000221B97280BDC0460C100440F8B5104E00241125E0B203F031F9071C14D0B87A20
:20426000012811D13846FFF7CBFF81280CD097F9090096F8491005FA00F0084386F84900EF
:204280000448002103F03EFD641C032CE2D3F8BDB0320020A0330020F8B506460F4D104FC1
:2042A0007388002417E0A20002EBC402921951689068D26852B9AF420BD00A7855F8222015
:2042C0000346491C08461946904701E0FBF750FC7388641CA4B2A342E5DCF8BD50B101005F
:2042E0005CB1010070B544680D4604F5827003F0E3FC0D4A667F207F0C49A3691268801980
:20430000C01D80B204F5827445436943B1FBF3F010186330B0FBF2F1491C204603F0C8FC11
:20432000204603F0C7FC70BDA035002040420F003EB5054615F8060C03281DD12B68186924
:20434000009058690190986902906C6859689A681868DB68A0472968086015F8080C43F05A
:20436000D9F90446012043F003FA011C04D042200870204643F0F2F83EBDFEE7F0B51546A2
:204380000E4604461F1CADF1240D08BF002308D0684600212422082303F050FDB8686B4662
:2043A0000690204631462A4603F044FD034804490268204609B00A60F0BDC0468CAC01006F
:2043C000A0350020F8B503468C46171C4FF000001BD006460146C6B91CF8014B082584F0B0
:2043E000010202F001028918C9B24A1E9A4208D0401C6D1E4FEA6404C0B2F0D18742EADC43
:20440000F8BD87424FF00106E5DCF8BD0E49086820F0020040F4087008600C48032140F8C5
:20442000041C41F230018160012101605022826001604FF4CA62826001604FF48652826030
:20444000016003480160704700000460586004400041044038B50E4B1B680D461446AB4250
:2044600004D30C4951F82510884201D0022038BD03F02AFC084B103B1A68AC400121A940B0
:204480008A4314431C6003F021FD002038BDC046A01E002030320020E020024070B5104D2C
:2044A00095F83904B5F85E440F280FD0D5F8606101F09AF80019864208D895F839144FF4DE
:2044C000707088402418A41B04F5707405F5F2752846FCF7C3FF2146284602F06DFE70BD79
:2044E0001001002010B50F4C104601214FF0E04221700221014012EA03000B4A08BF002959
:2045000004D0114691F90000401E087092F9000018B90020EEF702FF01E092F90000002022
:20452000207010BD3D1F0020361E0020B0B50F4C0546606880470E490D700A490A4A0F7892
:204540001FB91778A1682FB907E01778A16837F07F0702D088470120B0BD8847FEF7C2FF23
:20456000B0BDC04650040020BD350020D81800202C1C0020104898B5877890F8AF44002F7C
:2045800014BF802100210A4BB3F85C004FF67F72022C02EA000241EA020140EA0100A3F8E4
:2045A0005C0004D10349087867F3C710087098BD20180020CC1400201001002010B5044668
:2045C0000F480078ADF1180DC0B1012000238DF8000004F128018DF801300DF1020043F008
:2045E000ADFB6068007804F11C018DF80A000DF10B0003F04FFB6846F8F762FF06B010BD6B
:204600003D05002038B5EB2002F043FE0D48002404700A480078862802D12046FFF7A4FDD8
:20462000074D6868804708490A6A13681C7112680A62A968884702F0DBFD38BDBD3500202B
:20464000D8180020BB350020FC3300201FB5144600900A79487940EA02208A7942EA00224C
:20466000C87940EA022001900A78487840EA02208A7842EA0022C87840EA02200290684672
:2046800000F0E4F9B0FBF4F16143401AC0B200901FBDF8B5051C0E4606AF04D0012D0CBF3D
:2046A0000624002400E002240EB9A41CA4B2012A06D0022A0ED15889C01D04EBE00408E044
:2046C0003878002814BF022101210020FAF7F4FC2418A4B22046F8BD70B50D46044603F087
:2046E000F3FA6668A1682B468E4204D103F0EEFB4FF0FF3070BDE1682568491CB1FBF6F29A
:204700007243891A4B55A2686369E160521CA260934238BF626103F0D9FBA06870BD7047D8
:204720000F4800B50068ADF1240D69467030F3F763FF10B99DF80B0008B900200DE06846B6
:2047400001F0A9FF9DF808104FF47A73B0FBF1F24A43801A091A03FB01F009B000BDC046A0
:2047600014010020F8B502F08DFB0D460746FF2F08BFF42011D0094C60688047084A0646D1
:20478000B800084B115C80184278C918284643F05DF8A168304688470020F8BDD818002045
:2047A00020A101003C05002038B50D4DD5F860014268002101209047D5F8600101680120E6
:2047C000884708B1286880470648074CD5F86C310068083C606018688047206138BDC046C0
:2047E0008000001030200940683500202DE9F84303F086FADFF830900C4D0024012680460E
:2048000006FA04F018EA000F06D059F8240018B107680FB12146B8472868641CE4B284427E
:20482000EED9BDE8F883C04630320020A01E0020B0B503F049FA05460B48017801290FD070
:204840000A49024601230878137048B1084C0746206880680146204688470C347F1EF7D16B
:20486000284603F033FBB0BD3C1F002023AC010004AC01002DE9F0410E4C201D0068804733
:20488000064600F041FE8046002043F0DFF8084D686002F0B1FB0746404602F0F3FB17B177
:2048A000012068702870A16830468847BDE8F081901E0020D818002010B50F4C94F80F0268
:2048C000ADF1180DA8B940F0010084F80F02012002F05AFA02A801F017FE0120009004F535
